:020000040000FA
:1000000000400020157A0100517A0100537A010066
:1000100000000000000000000000000000000000E0
:10002000000000000000000000000000557A010000
:100030000000000000000000577A0100597A01001A
:100040005B7A01005D440100797E01005B7A01006A
:100050005B7A010000000000E5F400005B7A01001B
:1000600041CE00006D6A0000A9F400005B7A010037
:100070005B7A01005B7A01005B7A01005B7A010028
:100080005B7A0100D18301005B7A01005B7A010099
:100090005B7A01007DB2010059B201007DCF000002
:1000A0008DCF00005B7A010000000000000000001E
:1000B0000000000000000000000000000000000040
:1000C00010B5064C2378002B07D1054B002B02D02E
:1000D000044800E000BF0123237010BDA4020020EB
:1000E0000000000090D70300084B10B5002B03D090
:1000F0000749084800E000BF07480368002B00D10B
:1001000010BD064B002BFBD09847F9E7000000001C
:10011000A802002090D70300A402002000000000E5
:10012000164B002B00D1144B9D46402292029A1A86
:10013000924600218B460F461348144A121A2CF09F
:100140002FFB0F4B002B00D098470E4B002B00D0FD
:1001500098470020002104000D000D48002802D01F
:100160000C4800E000BF22F095FA200029002AF098
:100170006DF921F067FFC046000008000040002034
:100180000000000000000000A4020020A00B0020DE
:100190000000000000000000C46005614661876146
:1001A0004146C161494601625146416259468162F8
:1001B0006946C16271468160124B1A68026018601C
:1001C000002070470F4B1A6812681A6070470D4B79
:1001D0001A68002A01D127F0EDFF506010681860FE
:1001E000D468156956699769D1698846116A894644
:1001F000516A8A46916A8B46D16A8D4691688E46CD
:1002000001207047400A002010B502F04DFB1EF09F
:100210007BF80022084B1DF06BFA084A084B1CF0D3
:1002200033FE1EF0C3F80323020002209A43054B5D
:100230001043C01810BDC04600806640182D4454BD
:10024000FB2109400000808010B502F02DFB1EF05C
:100250005BF8094A094B1DF04BFA0022084B1CF0D1
:1002600013FE1EF0A3F80323020002209A43054B5D
:100270001043C01810BDC046182D4454FB2109403E
:10028000008066400000808010B502F00DFB011C6C
:100290001CF01CFA024B002800D1024B180010BDC4
:1002A000442403003C24030010B502F0FDFA44008E
:1002B00064080849201C1CF009FA002805D10549EA
:1002C000201C1BF089FA002801D0034810BD034808
:1002D000FCE7C046FFFF7F7F3C240300442403006B
:1002E00010B502F0E1FA034B034002201843024B21
:1002F000C01810BDFCFFFF7F0000808010B502F029
:10030000D3FA440064080849201C1CF0DFF90028D7
:1003100007D10549201C1BF055FA002801D10348DC
:1003200010BD0348FCE7C046FFFF7F7F4424030065
:100330003C2403001FB50023019302F0B5FA01A984
:100340001EF02EFB032203000220934306490343C1
:100350005B180293019B934303435B1802A9039329
:1003600006F054FD05B000BD0000808070B50D00A2
:1003700002F09AFA041C280002F096FA1CF0BEF96A
:100380000100201C1EF0E8FA0323020002209A4319
:10039000014B1043C01870BD000080801FB50023C2
:1003A000019302F081FA01A91EF0ACFA03230224A2
:1003B0009843074B2043C0180290019824F0FDFE9B
:1003C00002A90390200006F021FD04B010BDC04634
:1003D0000000808070B50D0002F066FA041C280051
:1003E00002F062FA011C201C1EF068FD03230200CB
:1003F00002209A43014B1043C01870BD000080805A
:1004000070B50D0002F050FA041C280002F04CFAFE
:10041000C00FC30760004008184303230224984319
:10042000014B2043C01870BD0000808070B50D00E6
:1004300002F03AFA041C280002F036FA011C201CD3
:100440001EF0C4FC0323020002209A43014B104318
:10045000C01870BD0000808010B502F025FA1EF0B3
:1004600059F80323020002209A43024B1043C0189C
:1004700010BDC0460000808010B502F015FA1EF0D5
:1004800051FC0323020002209A43024B1043C01880
:1004900010BDC0460000808010B502F005FA1EF0C5
:1004A000EDFB0323020002209A43024B1043C018C5
:1004B00010BDC0460000808010B502F0F5F91EF0B6
:1004C00053FB0323020002209A43024B1043C0183F
:1004D00010BDC0460000808010B502F0E5F91EF0A6
:1004E00005FB0323020002209A43024B1043C0186D
:1004F00010BDC0460000808010B502F0D5F91EF096
:1005000071F90323020002209A43024B1043C018E2
:1005100010BDC0460000808010B50349034815F0A7
:1005200001FDFFF754FEC046E8450300003203001A
:1005300070B5060008680D0002F0B6F90021041C31
:100540001BF040F9002801D0FFF7E6FF201C1EF049
:100550001DFD041C012E06D1032302209C432043D1
:100560000C4BC01870BD686802F09EF90021051C94
:100570001BF028F90028E7D1281C1EF007FD011CFC
:10058000201C1BF0F7FB0323020002209A431043B8
:10059000E6E7C0460000808010B502F085F91EF045
:1005A00019FC0323020002209A43024B1043C01897
:1005B00010BDC0460000808070B50D0002F074F9D7
:1005C000041C280002F070F9011C201C1EF05AFDCA
:1005D0000323020002209A43014B1043C01870BD50
:1005E0000000808010B502F05FF90021041C1BF0B0
:1005F000DFF8002801D0FFF78FFF201C1EF0D6FE89
:100600000323020002209A43014B1043C01810BD7F
:10061000000080800048704740D7020080235B05BF
:100620001869034B1B7843438020C002C01A7047EF
:100630002F09002080235B051869034B1B78434377
:100640008020C002C01A70473009002070B5084DE4
:10065000C4012B680021181924F033FC2868054BCD
:1006600000197F3000781B788342F0D270BDC046FD
:10067000C00200202E09002010B5C3790400002B11
:1006800008D0064A037981791068DB01C01801306F
:1006900024F017FC0023237210BDC046C0020020C6
:1006A00010B50349034827F0E8FFFFF790FDC04667
:1006B0006D4603000032030010B5124B01001A68AA
:1006C0004379DB01D31818007F300478FF2C08D160
:1006D0000879C00112185278FF2A0FD08879904209
:1006E0000CD08A799B180132D2B258787E2A01D078
:1006F0008A7110BD00234C718B71FAE701204042D2
:10070000F7E7C046C0020020FC2270B592021378C1
:100710004D2B01D08022D2028026802076053469BC
:10072000336964421440E41AC0023169001B1AF0B4
:1007300079FE284B284918703369E21852185D4237
:100740001540264B264A27499A1A52183169954274
:1007500030D38020C002401B1AF064FE224B641B81
:100760001870E411214BE4B21C70A1200123002574
:100770001F4A20491360C0004D604B68002BFCD01D
:100780001358DBB2A342F7D21B4901330B7001238C
:100790005360FFF743FF03780500184CFD2B0BD186
:1007A00080235B051869164BC009C018C0012818C2
:1007B000206070BD6D18C9E7FFF73CFF0378803DEE
:1007C000FD2B01D12560F4E7FFF734FFFD2124F074
:1007D00078FBF7E730090020FF87FFFFA402002025
:1007E000000000209CD703002F0900202E090020C4
:1007F00000D00040FCD0004031090020C0020020A1
:10080000FFFFFF01F7B5254B254F1A78254B140044
:100810001B7839680133E001405CFF2839D001348E
:10082000E4B29C4200D101249442F4D180230026FA
:100830005B051B69DB090093E30101933B68E2015F
:100840009D182A78280053425341F61824F04FFB94
:100850000023002815D1134B01341B78E4B2013377
:100860009C4200D101240D4B1B78A342E4D1072EFA
:1008700011D923F0EDFBC6E7DA01AA5C002AEAD120
:100880000133009A9342F7D13868019BC01824F0D5
:1008900024FB2000FEBDFF24FBE7C04631090020F9
:1008A000C00200202E090020F7B507000D0001242A
:1008B0000E4B1B7801930E4B1E68019B9C4202D984
:1008C000FF242000FEBDE10171180B78FE2B09D139
:1008D0008B78AB4206D103312A0038002BF036FF6B
:1008E0000028EED00134E4B2E7E7C0462E0900202C
:1008F000C002002010B5054A03791068DB01C0185A
:1009000081780022033002F005FD10BDC0020020F6
:10091000F0B585B002900D001600039378294BD8EE
:10092000FFF7C2FF0400002E3ED0FF2801D0FFF7E2
:100930008DFEFFF767FF0400FF2805D11F492048FF
:1009400027F09BFEFFF743FC1E4FC0013B68019060
:10095000FE21181824F0B5FA3B68019AE9B29818FC
:10096000023024F0AEFA3868019B2A00C018033028
:10097000029906F06DFB0C2025F077FD039A030029
:10098000002A17D0104A1A600E4A1C7112685C7156
:10099000E4011419A278DE7102329A7101221A72EE
:1009A0006A46127B5A7202E03300FF28E3D1180036
:1009B00005B0F0BD054AE6E70023F8E78A460300E4
:1009C00008300300C002002050E2020008E30200E9
:1009D00007B501A903F04CF90199FFF765FFFF285E
:1009E00005D10549054827F048FEFFF7F0FBFFF762
:1009F0002DFE03480EBDC046A0460300083003008C
:100A0000D0DB0200F7B50192027A05000091002ABE
:100A100001D1FFF745FEC479002C06D1214A1768A1
:100A20000279D201D25D002A04D1092201201A6084
:100A30004042FEBD69797E22C901791808007F30E5
:100A4000AB790078D21AFF2809D12879C00138186B
:100A50004078FF2819D0C01A824200D902000198BC
:100A6000061B964200D91600002E19D0009A0133B9
:100A70001019C91832002BF078FEAB799B19DBB244
:100A80007E2B04D0AB71A419D4E70022E7E7002342
:100A9000AB716B79DB01FB187F331B786B71F2E76D
:100AA0002000C6E7C0020020F0B585B00393037AAA
:100AB00004000192002B01D1FFF7F2FDC379002B56
:100AC00034D02D4A03791268DB019B5C002B2DD0BA
:100AD000019B02910093009B002B2CD07E22A379D6
:100AE000D71A009A974200D917006079224E013335
:100AF000C001C01833683A001818029906F0A8FA25
:100B0000A379DB19DBB27E2B33D10023A371FFF76E
:100B100079FE0500FF2811D12079FFF797FD00230A
:100B200023721C23039A13601D3B03E00923039ADD
:100B300013600A3B0193019805B0F0BD60793368FA
:100B4000C001181829007F3024F0BBF93368ED018B
:100B50005819617924F0B5F962793368D2019B188C
:100B60007F331B786371029BDB190293009BDB1BB5
:100B7000B0E7A371F7E7C046C0020020002170B5BE
:100B8000080024F00EF9012405000C4B1B78A34249
:100B900001D2280070BD0A4AE3011068C01803782A
:100BA000FE2B08D181780022033002F0B3FB010054
:100BB000280004F0E9FD0134E4B2E6E72E09002044
:100BC000C002002073B501A903F052F80199FFF7A4
:100BD0006BFEFF2805D10F490F4827F04EFDFFF7A8
:100BE000F6FA00257E260D4B1C68C301E3185978E0
:100BF0009B780233DBB2C201A2187F321078FF2843
:100C000004D1C81A401924F0D8FA76BDF31AED18A9
:100C10000023F0E7A046030008300300C0020020D4
:100C200010B5024B024A24F060FB10BD79060000AB
:100C3000B90600007FB50B00012803D10021186818
:100C400001F018FD102102A828F025FB0A4902A88E
:100C500025F0AEFF039B0193002B06D1042804D19D
:100C6000064827F0FDFCFFF7B2FA02A9044802F09B
:100C70001BFB07B000BDC046C8CB0300202D0300FE
:100C800084320300002313B5044A046A0905009363
:100C9000890C8A58A16B23F0C0FA13BDA8D70200B3
:100CA000F0B587B000931B7804000F0002927C2BF4
:100CB00005D18268525C002A01D09A2A14D11A0008
:100CC0006B3A022A2DD8A568E8190378032B5ED168
:100CD00004A9666823F06DFBAB19984206D16760E2
:100CE0000499200023F0C9FA07B0F0BD0378032B64
:100CF0004DD105A923F05DFB009B1B786B2B04D124
:100D0000049B059A13430493E6E76C2B03D1049BE1
:100D1000059A5340F7E76D2BDED1059B049A1340EB
:100D2000F1E76E2B04D0022219009143702966D19D
:100D3000A368D81901930378032B28D1636804A909
:100D4000039323F036FB0600019B039A9B189E42F7
:100D5000C5D0B378B01C7578032B18D105A923F042
:100D600028FB0600372D15D1059A1F2A0FDC4149B3
:100D7000049B114199420ADBC021090611418B42B3
:100D800005DB93400493049A53005340DCD5029D45
:100D900000224FE0392D08D1059B1F2B01DD1F23B9
:100DA0000593049B059A1341ECE72F2D03D1049B77
:100DB000059A9B18E6E7302D03D1049B059A9B1AF0
:100DC000E0E7312D09D10599049802F081F9002856
:100DD000DDD1059B049A5343D4E7332DD7D0059931
:100DE000352D06D10029D2D0049823F073FD04904C
:100DF000C9E70029CBD0049823F07CFDF7E7752BD9
:100E0000C5D1A368D8198378032BC0D145780230A7
:100E100023F0DEFA2F2D01D1049060E7302D06D1AA
:100E2000404243000490584000D458E7AFE7C04325
:100E3000F2E73200561CED09FBD16368DB1B01931E
:100E40000135DB09FCD1023252193900200028F0AB
:100E5000C2FA0400009B029A1B7831001A33037017
:100E6000013023F05CF9701C2018019A290023F04E
:100E700056F939E7FFFFFF3FF0B597B00890C02063
:100E8000002540230AAC80000F0016002570636027
:100E9000A56025F0F7FA2561E0606561A561E5616F
:100EA0002762E562A84218D1C349C44827F0E5FB90
:100EB0000023060013930D9825F0FEFA002E00D1B2
:100EC000E0E10023BA6B3968300015F09BF8380078
:100ED00024F0F8F93000FFF77AF9321E03D004222B
:100EE000022E00D0033A0026B549009692005258CF
:100EF0002000B96B330023F090F9102025F0B5FAEB
:100F00001021040028F0C7F90AADAB68002B00D10E
:100F100094E12A78002A00D090E1013B0C32AB60CA
:100F20005343EA68A649D318DA785D6892005258AC
:100F300002921A689B681202120A0393029B05929E
:100F40005B7806930F23069A13400493002D01D17A
:100F5000636803933023069A1340102B27D0202B6D
:100F600066D0002E00D042E10123069A1A40099271
:100F7000099A02992A405300CB1880215B884901C5
:100F800007931B0B1B038B4200D048E13B000799E2
:100F900040331B780905090D8B4200D026E1002A59
:100FA00000D11EE1380024F0FDF90135E0E7002D05
:100FB0000BD180213800029B6A009A184901403009
:100FC000049BAB4205D801269EE7002EF1D10026F6
:100FD0009AE753881E0B36038E4214D106781B0500
:100FE00002321B0D9E4221D121000AA823F054F9A0
:100FF0000028ECD13B0040331B78062B00D035E1B4
:101000007049714852E7049A6B1C9A4206D9039AB8
:10101000059900920AA8029A23F0FFF8029B6D003E
:101020005D1969880AA8FFF72DFED0E70135C7E7EB
:10103000002E0BD0029A6B009B5A1B0B032B48D13E
:101040000121200028F08FF900230370029B6E001D
:101050009E19049BAB4240D8002380201E00400113
:10106000049A934269D3A368039A981800230693BD
:10107000A2686368D31898426DD3029B1B781F2B1C
:1010800001D02E2B00D10126029B597840230B4022
:1010900018004342434149B25B421E40002900DA36
:1010A00001260025039B0495D0180795069B9D42B9
:1010B00058D1002E02D1079B012B63D00499200048
:1010C00028F0BDF9029B059A03992000FFF7E8FD7F
:1010D0007DE7012D00D876E78CE7802173884901F0
:1010E0001A0B12038A4226D13A0040321278DBB240
:1010F0009A421CD1082A07D1B96CF86C08F07CFB25
:101100000100200023F07FF8002D0AD1029B5B78BC
:101110007F2B06D90E9B2000591C06930E9123F0BD
:10112000ACF8380024F03EF90135023691E7002D85
:1011300000D148E75EE76B1C69E702995A008A18FC
:101140005288110B0903814203D1D2B2072A00D978
:101150000126013384E7069B01210133069323F026
:1011600001F885E7049A037801320492002B04D039
:10117000079B0133079300230493012122F0F2FF20
:10118000013593E7A268039B944663441D00069BC8
:101190009E4200D11BE72B78002B07D1A3680122C8
:1011A000E91A200028F057F90136F0E7280001215C
:1011B00022F0D8FF0500F7E7AF460300542F0300E5
:1011C000A8D70200D74603001C2E0300012D00D132
:1011D000F9E601232A001A402ED0049A032A0DD0E2
:1011E00008E721000AA823F057F8DEE60135049B42
:1011F000022BEBD10023012D00D1E4E6069A691EF3
:10120000D20705D5029A9288120B012A00D16908EB
:10121000012900D056E7002B00D1D8E652E7039A07
:10122000059900920AA86B1C029A22F0F6FF079912
:101230000AA8FFF727FD67E61300DFE72B78002BEE
:1012400000D031E63B0040331E78002E00D0D1E6BE
:101250006368002B00D1CDE62B692000591C23F0D8
:101260000CF8A3686B62EB69AB6224E6022B01D138
:101270000949C6E60B3B09480949012B00D815E688
:10128000084913E6380024F01DF8089A13AB13CB75
:1012900013C2089817B0F0BDE946030004310300FB
:1012A0001D4703004447030000237F2803D8034B56
:1012B0001B5C9B07DB0F18007047C0465C470300B0
:1012C00000237F2803D8034B1B5C1B07DB0F180090
:1012D0007047C0465C47030000237F2803D8034BB8
:1012E0001B5C5B07DB0F18007047C0465C470300C0
:1012F00000237F2803D8034B1B5C5B06DB0F180021
:101300007047C0465C47030000227F2808D8054B81
:101310000132195C0C23194202D15F38424242412A
:10132000100070475C47030000237F2803D8034B5D
:101330001B5CDB06DB0F18007047C0465C470300F0
:1013400000237F2803D8034B1B5C9B06DB0F180090
:101350007047C0465C470300BFF34F8F024A034B00
:10136000DA60BFF34F8FFEE70400FA0500ED00E0FE
:101370000120024B1B685B0018437047D80800200F
:101380000120A922044BD2001B6898649B58034A91
:10139000136083401843704704000020C4020020FB
:1013A00001220F4B10B51A600E4A51680029FCD07B
:1013B00000215160A122D200985801225A601CF0ED
:1013C00061FF0022084B1CF093F91CF0EFFF032390
:1013D000020002209A43054B1043C01810BDC046BE
:1013E00000C00040FCC000400000D03F00008080F2
:1013F00010B5C30708D483070ED10368094A934286
:1014000002D0094A934207D101F0EAF9002801DD30
:1014100012F04EFD054810BD01F046FA1BF06EF9C2
:10142000F4E7C046A0F002004C240300D0DB020029
:10143000F0B50F000A2485B001901C491C4824F027
:1014400019FEFA200025800012F032FD019BAB420C
:1014500003D0386801F0C4F90500280021001AF013
:1014600051F903AE3031B170280021001AF064F850
:1014700021001AF047F930317170280064211AF008
:101480005BF821001AF03EF9002530313170705DB3
:1014900024F0DAFD0100064824F0ECFDFA200135C5
:1014A000800012F005FD032DF1D1C6E774DB0200C8
:1014B00024000020054B002805D00023022802D17B
:1014C000012349000B4318007047C0463C24030029
:1014D00010B5024924F0FDFF10BDC046C25B0300F9
:1014E000F0B5204B8BB004AC20C9013800930194B7
:1014F00006230DF05DFBE0681B4EB04225D10527A9
:101500001A4BDF572069B04223D1194B5B795BB28C
:1015100003936069B04220D10522164B9A560123ED
:1015200004355B42009303993B00280016F0A2FDAE
:101530000023A2686168280016F022FD28000499A3
:1015400016F056FD30000BB0F0BD23F06CFB070029
:10155000D8E723F068FB0390DBE723F064FB02008D
:10156000DDE7C0467CDC0200D0DB0200ECE50200D7
:10157000FCE50200F4E5020070B586B00600012229
:10158000080003A901F0E6FA039D2C00049A631BEE
:1015900001929A4205D92178301D16F053FE01348C
:1015A000F4E7014806B070BDD0DB0200F0B51400CE
:1015B00089B001220600080002A901F0CBFA200040
:1015C0000024022205A9029F01F0C4FA059D039B95
:1015D00001939C4206D2395D301D16F033FE28552A
:1015E0000134F4E7014809B0F0BDC046D0DB020089
:1015F000F0B5050087B048680C000F6801F0F0F8FE
:10160000010002A827F05EFE0026032D03D1A0688A
:1016100001F0E6F806000024039B01939C4209D2E6
:10162000049B381D31001D19019316F00BFE013487
:101630002870F1E702A9024801F036FE07B0F0BDBC
:1016400008E00200F7B5314FB43701972F4A30490F
:10165000FC32536C8B4200D8F7BD0325043B536426
:101660001A682A4B511CAC331E680C008B08F35CC3
:101670002C4064002341881A2B400131022BF4D006
:101680000326019B12011B6800019A181F49830859
:101690000093009B002BD9D00F23106818422BD148
:1016A0001C4B1B68984227D30C00B8342468A04216
:1016B00022D20F24C01AC31723400C001B181B1181
:1016C0001D00AC34246898082418207835406D003B
:1016D00084462841304001280ED13700AF403D00FC
:1016E00067463D4325700D00FC356C6C0A4FBC42CB
:1016F00007D2201D68642360009B0432013B0093E5
:10170000C7E70B00BC331860F6E7C046380A002074
:10171000F80A0020EC0A0020780B00200F239943E0
:1017200070B506000D00081A412119F07BFE104C1F
:1017300002002300B033186023002100AC331E6088
:101740008301EB1AB4310B6023003000B833002161
:101750001D602BF025F822000023FC32D364A22266
:101760005200A352443A4733FF3AFF33E25270BD6E
:10177000380A0020A222034952008B5A01338B52AF
:101780007047C046380A0020A222034952008B5AF3
:10179000013B8B527047C046380A0020A223034AFF
:1017A0005B00D05A431E9841C0B27047380A0020EF
:1017B000F7B50024032500900191019B9C4200D1C4
:1017C000F7BD009AA300D3580F2213422DD11A4A15
:1017D0001100B43109688B4227D31000B83000687B
:1017E000834222D20F20591ACB17034010005B18F6
:1017F0001B111F00AC3000689908401801782F4079
:101800007F008C463941294001290ED12E00BE406F
:1018100037006646374307701700FC37786C074E71
:10182000B04206D2021D7A640360FFF70BFF013459
:10183000C3E7BC321160F8E7380A0020780B0020BB
:1018400010B5FFF797FF064800220300BC331A606B
:101850000300044AFC3328215A64FFF7A9FF10BD96
:10186000380A0020F80A0020F8B503262C4C002581
:101870002200BC321368AB420FD1022219000327A9
:1018800094462200B03212689200914226D300237F
:10189000FC34E364FFF778FFF8BD23001560214AAC
:1018A000FC335A642300B0331B689B009D42DDD299
:1018B0002200AC321268AB08D35C2A0032405200DE
:1018C00013413340032B07D12200FC32536C191D06
:1018D00051641D60FFF7B6FE0135E3E72000AC3030
:1018E00000688A08801802780D0016003D406D00DF
:1018F0002E413E40022E09D0032E0BD0012E07D1DF
:101900003B00AB409A430270012301E0002BF7D16A
:101910000131B6E76346AB409A4302700023F7E714
:10192000380A0020F80A0020274AF0B513001100F9
:10193000B833B43109681B6803265B1A11000360D1
:101940000023B0310C681900AC3215684360836025
:10195000C36003614361A400A14206D143681B0137
:10196000436083681B018360F0BD0F008A08AA5C96
:1019700037407F003A413240012A0CD8012B0ED16A
:10198000C7680137C7604769BB4200D94361012A74
:1019900010D0002A09D0022A10D00131DCE7022B36
:1019A000F1D1076901370761EDE78368013383608F
:1019B0001300F2E7436801334360F9E742680133FB
:1019C00001324260E9E7C046380A0020A223F7B599
:1019D000424F5B00FD5A0F300409002D02D0002554
:1019E0002800FEBD002CFAD0A3235B00F95A4A421E
:1019F0004A4101923A00B03212683B0094463A00E4
:101A00003026FC33AC32DB6C1068634507D3019B96
:101A1000002BE4D111F052FC01230193EAE70321EA
:101A2000C25C0A422AD10135AC4228D89B00591B1E
:101A30004C1C012D04D13D005A1CFC359208EA646F
:101A4000A208801826000322012516407600B54022
:101A50000678023135433E000570AC3601928B4268
:101A60002CD23A00B4321568210101336D181A1BCB
:101A70001201002128002AF093FEB1E700250C2175
:101A80000A4205D10135AC4203D89B000133CEE7B1
:101A90000025324205D10135AC4203D89B00023308
:101AA000C5E700253F218A4305D10135AC4203D863
:101AB0009B000333BBE700250133A6E70D00326826
:101AC00088081018019A0131154002226D00AA40C1
:101AD0001500027815430570C1E7C046380A00209A
:101AE000A22330B5214A5B00D35A002B3CD10F21F1
:101AF000084239D11300B4331B68984234D3140020
:101B0000B8342468A0422FD2C31AD8170840C0188E
:101B10001300001103250400AC331B6881085B5CD3
:101B20002C40640023412B40012B1DD11300FC33BA
:101B3000DC6CA14200D2D9640321AC321468830862
:101B4000E31804000D000C406400A5401C7801302F
:101B5000AC431C7014688308E35C04000C40640010
:101B600023410B40022BE9D030BDC046380A00208B
:101B7000A223F0B5002685B00700614802925B0001
:101B8000C25A0D00B24206D1B74207D1390028002F
:101B9000FFF71CFF0600300005B0F0BD002904D19E
:101BA0003800FFF79DFF2E00F5E70F243B001600DD
:101BB0002340F0D10200B43212681E009742EAD3EB
:101BC0000100B83109688F42E5D2B91ACA1722401C
:101BD0005218121100920200AC321268009C01925D
:101BE000009A019992088A5C0321214049000A4128
:101BF00003210A40012ACED129000F310909B03052
:101C00008C460168033689000391210014000131DC
:101C1000039A914212D201988A08825C08003040EF
:101C2000400002413240022A02D101340131EFE783
:101C3000002A03D10133E2189445F7D8644501D155
:101C40003E00A8E7644521D9009B032663441900A0
:101C5000009B0800E218AC239C46294B9C44634639
:101C600005001B6884081C19330035406D00AB402B
:101C7000257801309D4325709042F0D1204B890892
:101C8000FC33DA6C9142DBD2D964D9E71B199C454D
:101C900023D8032502261A49009BAC31E318019191
:101CA000009A6244934209D36346191B090120013B
:101CB0000A00381800212AF073FDC1E701991800C5
:101CC00009689A088A1831002840400081400800BD
:101CD0001178013308431070E2E7029E002E00D114
:101CE00059E700212800FFF771FE061E00D152E7D8
:101CF000220139002AF039FD3800FFF7F1FE4AE7EA
:101D0000380A0020F0B50E4C421E27681100002052
:101D1000BE09FB0F73407B403E097D087340BF083E
:101D20007B406B40DB072B4301251F0040002B400D
:101D30001843E940ECD18242E8D32760F0BDC046A9
:101D4000C802002070B50123A12400250B4A0C48CD
:101D50001360E4000421002345604668002EFCD097
:101D600016591B02013933430029F5D1002BF1D05C
:101D700004490B600123536070BDC04600D0004091
:101D8000FCD00040C8020020014B18607047C046DC
:101D9000C802002010B504000C2024F066FB034BA1
:101DA000446003600223037210BDC0463CDE0200A3
:101DB00010B50400102024F058FB044B0360237A74
:101DC0000371636883600023C36010BD00DE0200FE
:101DD00010B50400102024F048FB044B846003601D
:101DE000034B43600023C36010BDC046C40603001C
:101DF000F945020010B5043024F025FA004810BD62
:101E0000D0DB0200002803D0012808D0002005E024
:101E100007224B680448934300D1044870474B683D
:101E2000DB085B001843F9E7442403003C2403006B
:101E300010B50349034826F020FCFEF7C8F9C04658
:101E400001480300942E030070B515001A001C0011
:101E50000AF0E2F9002802D04368002B0BD12B1EB8
:101E600004D1074B022C01D1FFF7E2FF012C00D176
:101E70004360180070BD022CFBD100224260F8E7DD
:101E8000D0DB0200F8B504000D000B7A124A9B006B
:101E9000995824F01EFB1149200024F01AFB280059
:101EA000FFF786FF01260700380022F0AFFB051E72
:101EB00004D10B49200024F00CFBF8BD002E03D107
:101EC0000849200024F005FB01222900200000F031
:101ED000B7FB0026E8E7C04678DE02003948030079
:101EE0003F4803003C48030030B5002585B001A9F8
:101EF0000400019522F06BFBA84205D10A490B486A
:101F000026F0BBFBFEF763F9636802A9083B636038
:101F10000368029343680393042328C0022004F05B
:101F200075FF05B030BDC046DC470300942E0300AA
:101F3000F0B513681400012287B00F680D000092FD
:101F4000D908022306000CF001FE022E12D1032351
:101F5000686803401DD101682B4AC968914218D1B5
:101F60002A68904206D0059305A9686822F02FFBE5
:101F7000061E06D1002563689D4233D3234807B06F
:101F8000F0BD381D012231680AF046F973684360DC
:101F9000EAE70DF0B5FF039003980DF0FDFF002870
:101FA000E8D00DF0ADFF05000DF0F6FF029028001F
:101FB0000DF0F2FF060028000DF0EEFF029B002B53
:101FC00003D0002E01D0002805D01149114826F079
:101FD00054FBFEF7FCF8381D012202990AF01CF9A7
:101FE0004660D9E7A368EE009959002909D0042971
:101FF00007D0381D01220AF00FF9A3689E197368F3
:1020000043600135B7E7C046F9210000D0DB02008C
:10201000094803000032030073B50C0015001B28AB
:102020000DD000231F2808D1081D002229000AF026
:10203000F3F81A4B002800D1194B180076BD032382
:10204000194208D1174922688A4204D12B4002D193
:1020500029689142F1D0AB07EED1134B2A689A421E
:10206000EAD16A686368534007229343E4D101933D
:1020700001A9200022F0ABFA061E01D1074BDCE7D4
:10208000281D002231680AF0C7F80028D4D0416822
:10209000706800F053FB0028EAD1CDE74424030028
:1020A0003C240300C0DE020084DE0200F7B50B68AA
:1020B0001C4A04000D00934203D05A681A4924F0C8
:1020C000D3FA1A49200024F004FA002301270193CF
:1020D00001A9280022F07BFA061E0CD11449200029
:1020E00024F0F7F92B680F4A934203D011492000DE
:1020F00024F0EFF9F7BD002F03D10F49200024F0A1
:10210000E8F901223168200000F09AFA0B4920001A
:1021100024F0DFF901227168200000F091FA002715
:10212000D6E7C04684DE0200FB470300FF470300FA
:10213000CB830300C14A03003C48030082D2030062
:1021400010B504000C2024F090F9034B44600360A8
:102150000023037210BDC0463CDE020010B504002F
:102160000C2024F082F9034B4460036001230372C6
:1021700010BDC0463CDE020010B5043000220AF05B
:102180004BF8002805D10449044826F076FAFEF7FA
:102190001EF8406810BDC04601480300942E03009D
:1021A00010B5024B08C024F02FF810BD84DE0200E9
:1021B000F8B5070048680E000DF0A2FE040000F01C
:1021C00029FC0C4D022F00D9B568002809D122F056
:1021D00047FA060020000DF0DFFE011E03D130009B
:1021E000F8BD4010F3E7331D012218000AF014F87F
:1021F0004560EFE7D0DB0200F0B5070089B00020B2
:102200001E000D00019222F02BFA0E4B0400076015
:102210009F4203D10423027913430371019B2B4393
:102220000DD03368AA00B218019905A8039404934D
:1022300023F0FCFF681C05AA03A9FFF779FE200024
:1022400009B0F0BDC0DE020010B5002A03D122F0B3
:1022500049FA08480AE0042A09D10430002209F0AA
:10226000DBFF002801D1FFF7E3FD406810BD22F03D
:102270002FFAEEE7D0DB020073B50600194D0C0013
:10228000280020F061FF3100174820F099FE174820
:1022900020F05AFF164820F057FFFF239B00E61856
:1022A00021787F2901D0B44206D1280020F04CFFCC
:1022B000104820F049FF73BDA37850290CD80E4A6E
:1022C000505C0E4A525C01936378009303000C4803
:1022D00020F076FE0434E3E762780A4820F070FECE
:1022E000F8E7C04616490300434903004B49030081
:1022F000D4480300815303007ED003002DD0030097
:102300006C4903008F490300F0B51D008BB00790A6
:102310001B481600089120F017FF2900194820F0EB
:102320004FFE194820F010FF184820F00DFF002440
:10233000AC4204DB124820F007FF0BB0F0BD089B55
:10234000375DA0000799181803788278095D049713
:1023500007689B063F037F0E0397C7789B0E099380
:102360003B09029300883F07C004400E3F0F0190D5
:1023700012090097099B064820F022FE0134D7E796
:10238000164903006348030090480300C248030055
:10239000F4480300F0B505008BB008680C0001F0AC
:1023A00051FC049004A822F0A8F900270126049B00
:1023B00003900693069B197800291ED1380004F07B
:1023C00025FD0122009007A9606800F0C3FB079B70
:1023D000089A05939B1801920293022D22D9A068B6
:1023E00000F0FEF900281ADA089BC01817D52D490D
:1023F0002D4826F042F9FDF7EAFE0800FEF76CFFD3
:10240000002806D006A822F08AF9069B1B78732BB9
:1024100000D13000069B3F1801330693CAE7059BA5
:10242000181805900024BC4202D300980BB0F0BDF0
:10243000049B18780028F8D0FEF74EFF01250028ED
:1024400003D004A822F06BF905000598029A4319FD
:102450009A42CCD3049B1B78732B09D0009BA60017
:102460009E190195019B0436002B10D164190AE0D6
:10247000290000F067FF059B009A5D19A31C9B00D3
:10248000059501349850049B01330493CBE7049BDA
:1024900005AA1978039807F09FFA019B7060013B29
:1024A0000193DFE7B049030000320300F0B589B0C3
:1024B000039101921E0001F0C5FB049004A822F0D4
:1024C0001CF900240290B44201D309B0F0BD049B72
:1024D00018780028F9D0FEF7FFFE0125002803D068
:1024E00004A822F01CF90500039B019A5B199A428B
:1024F00005D21D491D4826F0C0F8FDF768FE049B73
:102500001B78732B10D064190E9BA700DF19002DC8
:1025100025D0049BAA0052421978BA5803AB0298FE
:1025200007F0BAFA013DF2E70E9B671CA400E058E1
:10253000012205A900F00EFB069CAC4200D92C003C
:102540002200059903982AF010F9039B2A1B1819F9
:102550003C0000212AF024F9039B5D190395049B9C
:1025600001330493AFE7C046B049030000320300D3
:10257000F0B50E0089B0039001CE0F0022F0E5F80F
:102580004410210004A826F09DFE069D2200002193
:1025900028002AF005F9039B0096013B2A1929001F
:1025A0003868FFF783FF04A9024800F07DFE09B0F8
:1025B000F0BDC04608E0020030B50C0089B005004F
:1025C0000222606805A900F0C5FAA06800F008F9C9
:1025D000002809DA069B0393C01805D509490A4863
:1025E00026F04BF8FDF7F3FD0599069AEB1E8A18C5
:1025F000091820000C3000902068FFF757FF0348AF
:1026000009B030BDB049030000320300D0DB020046
:10261000074BC2070AD4074A074B0240062A05D0D7
:102620000322064B0240022A00D0036818007047BC
:10263000A0F00200070080FF84320300442B030057
:1026400070B50D00040016000BF068FE2800FFF7BF
:10265000DFFF8368002B04D0320029002000984758
:1026600070BD42680249200023F0FEFFF8E7C04633
:10267000054B030010B50A0001000248FFF7E0FF18
:1026800010BDC046F8100300F7B5050008000E00A5
:1026900025F0F7FF002812D001AA6946300013F098
:1026A000E9FC009B002B0AD01649280023F011FFFB
:1026B000009C154BE71EE418A400002F09DA310036
:1026C00028000222FFF7BCFF2800104923F001FF79
:1026D000F7BD019A0E4913195B681259280023F0BF
:1026E000C3FF019B1B199A68002A06D107492800DD
:1026F00023F0EFFE033F0C3CDFE70649280023F000
:10270000B3FFF7E7C34A0300FDFFFF3F494903005A
:10271000E74A0300FC4A030010B50400FFF778FF06
:10272000054B0069984203D0431E9841C0B210BDCA
:10273000200026F045FDFAE7096C010070B50500A0
:102740000C0001208D4203D0214B9D4201D100207D
:1027500070BD9942FBD001231D4204D01942F6D12D
:102760002B000D001C002A001A4B1A40062A05D027
:10277000AA0711D1184A296891420DD12340062B8E
:1027800005D0A307E3D1144B22689A42DFD1210080
:10279000280001F019FADBE72340062BD7D0A30766
:1027A00003D10D4B22689A42D1D02800FFF730FFA9
:1027B0008369002BCBD0220029001B2098470028DA
:1027C000C5D0064BC01A42424241D0B2C0E7C04613
:1027D000D0DB0200070080FF8432030044240300A2
:1027E000104B10B5984219D00F4A0123904217D0D0
:1027F000184201D0184110BD830706D10B4B026867
:102800009A4202D106F034F8F5E721F0DAFF0849E0
:102810000200084813F086FBFDF7D9FC0020EAE728
:102820001800E8E73C24030044240300A0F0020061
:102830008A4A03008831030010B5C30705D4830713
:1028400006D1054B02689A4202D122F0F3FC10BD7A
:10285000FFF7C6FFFBE7C046A0F002000F4B70B5C4
:102860000D000124984204D100230B6023001800BE
:1028700070BD0B4B984201D10C60F7E70300234079
:1028800002D040102860F1E78207F0D1054A0168C4
:102890009142ECD105F0ECFFF4E7C0463C24030084
:1028A00044240300A0F00200184B10B5984228D031
:1028B000174B984227D0C30703D5401019F03EFFAD
:1028C00010BD0323184206D1124A0168914202D179
:1028D00022F0B9FCF4E70340022B09D10E4B034070
:1028E000062B05D0FF23DB05C01803239843E7E739
:1028F00021F067FF09490200094813F013FBFDF7B7
:1029000066FC0020DCE7FE208005D9E73C240300BC
:1029100044240300A0F00200070080FF704A030077
:102920008831030010B583070CD103680A4CA34219
:1029300002D122F0A6FA10BD084CA34202D122F027
:1029400047FAF8E721F03DFF05490200054813F07A
:10295000E9FAFDF73CFCC04690EC0200C0E9020039
:10296000204A03008831030013B50C0001A9FFF7CA
:10297000D9FF019BA34206D022000349034813F06C
:10298000D1FAFDF724FC13BD434A030000320300D3
:10299000F7B505000C0017001E00D3070ED5571021
:1029A0000197019B002B1FDA1B190193002E1DD0EC
:1029B000002B15DA002301930198FEBD01A9100038
:1029C000FFF74CFF0028ECD138006C6821F0F9FECD
:1029D000220003000B490C4813F0A4FAFDF7F7FBA3
:1029E0009C42E9D20194E7E7002EF9D1019B002B2C
:1029F00001DB9C42E0D86A680449054813F092FA6A
:102A0000ECE7C046E6490300883103000A4A0300A8
:102A1000582E030010B50400830710D10D4B026837
:102A20009A420CD10C4B0340062B06D1C00822F071
:102A3000CEFD43000120184310BD8068F9E7200057
:102A4000FFF7E6FD4369181EF6D0210001209847E4
:102A5000F2E7C04608E00200070080FF164B70B5A1
:102A6000040000209C4203D0144DAC4201D101204F
:102A700070BD134B00209C42FAD0012626408642AE
:102A800003D06010431E98410DE02000FFF7C0FD09
:102A90004369002B09D0210030009847002804D05A
:102AA000401B43425841C0B2E2E72000FFF7B2FFAB
:102AB0000028DCD00138E5E73C240300442403006F
:102AC000D0DB020010B50400FFF7A4FF002809D1F5
:102AD000200021F076FE04490200044813F022FA97
:102AE000FDF775FB10BDC046A24A03008831030004
:102AF00070B504000D001600FFF78AFD036A002B75
:102B000005D03200290020009847002818D10D4D2B
:102B10002000002E08D121F054FE02000A492800AE
:102B200013F000FAFDF753FB042E04D121F049FE07
:102B300006490200F3E721F044FE05490200EEE7F2
:102B400070BDC046883103000A4B0300354B0300BB
:102B5000564B030010B521F04AFE002805D1034969
:102B6000034825F08AFDFDF732FB10BDC149030083
:102B700088310300F0B58BB0079310AB10CB0090F9
:102B800001911B78062A12D8012A08D93F230B701D
:102B90000B0001330193002301990B7001E0002A1F
:102BA000F9D101209042804140420BB0F0BD009924
:102BB00000292ADA019B01995F1C2D230B708021CB
:102BC00009068C46009B63440093019BFF210993F7
:102BD000009BC90518000840884224D12021079B8A
:102BE000F81C0B401900009B5C024E23002C13D1F3
:102BF0004B4049227B7046234A4059403A70B97095
:102C000000230370019BC01ACFE7019F002BDCD08B
:102C1000390001370B70D8E741240B4361403B700A
:102C20007970BB70ECE7002C00DA06240199013AB8
:102C30007D1A551B2022079911430291672942D121
:102C4000002C00D1D5E1002B7BD0A84A934200D9BB
:102C5000D5E0A749009818F0C9FD431E984100230C
:102C6000002630300393203305900493A14B039A40
:102C70000099D05818F0B0FD002808D0049B039AA2
:102C8000F6189D4B0098D15819F064FA0090049BF7
:102C90005B100493039B04330393182BE6D1153385
:102CA0000493009A914B934260D39149009818F095
:102CB0009DFD002854D0002E01D12B230493FE2328
:102CC0009B05009352E0002BBFD1029B662B38D1AD
:102CD000631C9D4200DCAC1E029B651C0393002319
:102CE0001E0004930593E343DB171C40039B652BF5
:102CF00000D0F1E0651C00230693069B9D424EDD4B
:102D0000009819F0FBFC7B1C0893030030333B70E8
:102D1000059A069B934205D1002C03D0BB1C089357
:102D20002E237B7019F00AFD011C009819F032FB6C
:102D3000724919F00FFA069B009001330693089F21
:102D4000DBE7631D9D4200DCAC1F029B652B00D0BE
:102D5000ADE0002503933A3B049305952E00C2E7AE
:102D60000098664919F0F6F901360090029B662B2F
:102D700003D0672B37D1042E35DC6B461B7D3B70AF
:102D8000029B672B01D1731EE418631C9D4200DC7B
:102D9000AC1E002C12D16623013703930494029BCE
:102DA000662B00D0B0E0012E00DDEDE05449009824
:102DB00018F01CFD002800D0ACE0E5E02E23250033
:102DC00030227B70BB1C013E1F00002E74D0002DF2
:102DD00005D1049501235B42059367334CE01A70DB
:102DE000013D0133EFE76B1F9C4270DB029A672ABB
:102DF00064D01300AC1F00250393059573E70023EF
:102E000000260393203304933B4B039A0099D05838
:102E100018F0D8FC002808D0049B039AF618354B0C
:102E20000098D15819F096F90090049B5B10049318
:102E3000039B04330393182BE6D13049009818F014
:102E4000D5FC002805D000982E4919F083F90136E9
:102E50000090029B662B11D1AE4212DAA319013306
:102E60009D4203DCAD1BAC1E00D56C1E0023351942
:102E70000493013505966633039334E7029B652B73
:102E800009D16B1F9C4200DBAC1F2B230025049350
:102E900005953A33F0E7029B672B12D1231D9D4223
:102EA00000DC6C1FA6420CDA731CE41ADEE7002576
:102EB000029B0495039350E704968BE71C00029B4A
:102EC00099E7029B002503932B23049395E70025A4
:102ED000029B0595039309E7039B672B00D00AE744
:102EE000251E00D007E701252C0004E7FFFF7F3FE8
:102EF000F8FF7F3F90DF0200A8DF020000002041C2
:102F00000000A040CDCCCC3D3B49009818F06EFCB1
:102F100000282CD030217B1E1A782E2A60D0100079
:102F20003038092853D901330193019B1B78302B8A
:102F300014D1019A52782E2A09D10399662906D014
:102F400001994B70049B0A702D2B4BD1013E013728
:102F50003B00019A9A4247D331231370274B009AC2
:102F60009A4204D8039B663B5A425341E41A029B9F
:102F7000672B09D1002C07DD3B00013F3A78302A4E
:102F8000FAD02E2A00D01F00049B002B1AD020223A
:102F9000079B0A2113401A00452313433B706B46DD
:102FA0001B7C30007B7018F0C7FA0A2118F0AAFBCE
:102FB0003031B97030000A2118F0A4FB3C1D3031CB
:102FC000F970270000233B70099BF81AEDE5392AB8
:102FD00002D001321A70A7E7019A19709342A4D067
:102FE000013B99E70136B2E75A1E117819701300B8
:102FF000AFE7012427E6C0460000A040FFFF7F3F67
:10300000F0B5802787B02C4D02907F422C78002CA1
:103010001CD063B2002B10DA6E1C6D787C40E4B2D9
:10302000002D13D0013CE4B2FF2C0DD004AB981D51
:103030000121057010F0F2FEF4E704ABD81D012168
:1030400004702E0010F0EAFE751CDFE70627013F32
:10305000002F2ED0029810F02BFF0124BC42F6DA8C
:103060000025052D22D0154E22002900300009F040
:1030700067F86B4601901B79002B15D0631E1A0070
:1030800029003000039309F05BF8031E0CD12200E5
:103090002900300009F01CF8FF22019B2900134091
:1030A0003000621E09F014F80135DAE70134E4B2A9
:1030B000D4E707B0F0BDC046834B030024000020D6
:1030C00010B5C820FFF79CFF004810BDD0DB020000
:1030D00070B506000D00002814DD002907DD154835
:1030E00018F02AFA0124864209DC002407E00100D6
:1030F000C020000618F020FA01248542F5DAE4B277
:10310000200070BD002907DDC020000618F014FA69
:1031100001248642F3DBE8E70024A042F0D001005E
:10312000044818F009FA0123854200DB231CDCB2B5
:10313000E6E7C046FFFFFF3F032230B50240012112
:10314000002A04D1084C03680D00A3420AD00B00EA
:1031500003401D1E06D1002A04D1036803481B1A30
:103160005D425D41280030BD4C240300A0F0020008
:1031700010B50400FFF7E0FF012300280AD1023355
:103180002340022B05D105480440063C601E8441C3
:10319000E0B203000120184010BDC046070080FFC8
:1031A00010B521F00EFB03490200034812F0BAFEED
:1031B000FDF70DF8214C03008831030010B5040021
:1031C000102023F052F9044B84600360034B4360EA
:1031D0000023C36010BDC046C4060300E54B0200D7
:1031E000F7B504000E00019301208B180A0000219E
:1031F0000093009B934212D82725002900D0053D5B
:10320000224F2A003900200023F02EFA009B9E4214
:1032100014D32A003900200023F026FAF7BD1378D2
:10322000272B08D0223B5D426B41DBB20132002BE1
:10323000DFD02725E4E700230100F7E73278954245
:1032400005D12A001249200023F00EFA1AE0114994
:103250005C2A14D01F2A09D97F2A15D0019B002B84
:1032600002D053B2002B07DB3900ECE70A490A2AE7
:1032700005D00A490D2A02D0092A05D108492000A3
:1032800023F027F90136C1E70649DCE71C500300AB
:103290001B5003001F500300225003002550030061
:1032A000285003002B500300194B70B506000D0089
:1032B00098420ED14968A86806F06CFA041E08D03E
:1032C000280026F013F8E000002306242B6020439A
:1032D00070BD102023F0C9F86968040081600660A1
:1032E000A86806F039FA6B686060591C2B6899422F
:1032F00009D1AB68E3600023E268A1682000535461
:10330000AB602B60E4E7A86823F0C5F8E060F2E763
:103310008432030070B504000D00002A05D006F0C9
:103320006BFAC3000620184370BD06F033FA00287C
:10333000F7D12A002100024821F022FBF4E7C04621
:103340008432030010B50A000100024821F018FB86
:1033500010BDC04608E00200094B10B50340062B23
:1033600001D1C00810BD830708D1064B02689A42FC
:1033700004D18168C06806F03FFAF3E7FFF710FF59
:10338000070080FF84320300064B10B50340062B74
:1033900003D1C00822F025F910BD8368C0680B6016
:1033A000FAE7C046070080FFF0B50F00002689B09D
:1033B000110005001C0038000096032332000BF0BA
:1033C000C5FB0E20B7420FD0012F0FD102AA10214A
:1033D00004A813F0A1FD216802A83200FFF730F91C
:1033E00004A92800FFF760FF09B0F0BD206883073B
:1033F0001BD1134B02689A4217D104A9FFF7C4FFEF
:10340000104B060020680340062B0CD1C00822F0A8
:10341000D9F804001020049F23F027F80560876086
:10342000C6604460E0E74468F4E704A90122FFF7BE
:1034300091FB002205990498FFF76CFFD4E7C04682
:1034400008E00200070080FFF0B58BB00490086828
:103450000D0006920793FFF7DBF806006868FFF798
:10346000D7F8864202D06868FFF79AFE08A9286854
:10347000FFF78AFF040009A96868FFF785FF089A2B
:103480000590A3180393049B2700022B19D9AB685E
:103490001E498B4206D0012130000091210012F01C
:1034A000B1FE0700049B032B0BD0EB68174A934235
:1034B00007D00122210000923000089A12F0A2FEEB
:1034C0000390039B059AD91B069B38000093099B28
:1034D00021F037FA002809D1079B0138002B0FD0C3
:1034E0000B490C4825F0C9F8FCF771FE0A4B9E42C7
:1034F00008D10100200021F008F8440001202043F9
:103500000BB0F0BD041B6400F8E7C046D0DB02003E
:10351000445003000032030084320300F0B58DB044
:1035200004000391FFF774F804A906002000FFF7D8
:103530002BFF0190039883071ED10368314A934201
:1035400017D106AA05A921F09CFC00242500059BA3
:103550009C4220D32900002508A825F0B3FE0A9C30
:10356000059B9D4236D308A93000FFF79DFE0DB0A4
:10357000F0BD254A934208D023480022C3680121A8
:103580000293029C03ABA047039006AA05A90398E7
:1035900021F01EFCD9E7069BA700D859FFF738F8A1
:1035A000864205D019491A4825F067F8FCF70FFE46
:1035B000002C01D0049BED18069BD859154B0340F5
:1035C000062B05D1C00822F002F82D180134BEE701
:1035D0008068FAE7002D06D02000049A019929F0AE
:1035E000C4F8049BE418069AAB00985807A9FFF7A3
:1035F000CBFE079A0100200029F0B7F8079B0135A0
:10360000E418ADE790EC0200C0E902005850030056
:1036100088310300070080FFF0B5070087B0086815
:103620000D00FEF7F5FF04A906002868FFF7ACFEC1
:1036300005A904006868FFF7A7FE03902000022F89
:1036400007D901230093AB68049A2100300012F0DF
:10365000D9FD059A041B049BA418064D9C4205D86D
:10366000039929F073F8002800D1034D280007B012
:10367000F0BDC0463C2403004424030073B50D0094
:10368000060069462868FFF77FFE01A90400686804
:10369000FFF77AFE0100022E02D908480DF0DCF98E
:1036A000019A0098064D824206D8801A201829F007
:1036B0004DF8002800D1034D280076BD325003009C
:1036C0003C24030044240300F0B58FB00790106839
:1036D0000C001600FEF79CFF0690012C31D070689C
:1036E000FEF796FF069B834202D07068FFF758FDF5
:1036F0000DA97068FFF748FE0D9B089009930DA96E
:103700003068FFF741FE0D9B0B900493079B012B44
:103710001CD1049B5D1E01235B420A9300242700F9
:10372000049B03940593059B002B13D1039B002B53
:1037300023D1214B069A0E209A4200D01F480FB089
:10374000F0BD072309931E4B0893D8E701230025FA
:103750000A93E3E70B9B09995A19012308980093F0
:1037600021F0EFF8002816D1039B002B19D1079BFD
:10377000002B09D12F00049B5C1E049B0134E21B2B
:10378000934212D13068DAE7079B2C00012B0AD054
:1037900001232F0003930A9BED18059B013B059322
:1037A000C1E72C00F7E7039FE7E70B9B0698D919C1
:1037B00021F0E6F8C3E7C04684320300F8DF0200D8
:1037C000C1500300F0B589B0049008680D00FEF701
:1037D0001FFF07006868FEF71BFF874202D068687A
:1037E000FFF7DEFC06A92868FFF7CEFD060007A953
:1037F0006868FFF7C9FD069A0590B3180393049B08
:103800003400022B19D9AB681D498B4206D0012127
:1038100038000091310012F0F5FC0400049B032BEA
:103820000BD0EB68164A934207D001223100009278
:103830003800069A12F0E6FC0390079B0025002B47
:1038400012D1039B2000191B20F06EFE01304500B1
:103850000120284309B0F0BD0599200028F076FF2B
:10386000002808D101353400079A039BA618B342FB
:10387000F2D26D00ECE7200020F03EFE0600F2E7F9
:10388000D0DB0200F0B58BB00E0007000392FEF70C
:10389000BFFE05003000FEF7BBFE854202D03000BF
:1038A000FFF77EFC05A93800FFF76EFD06A90400AE
:1038B0003000FFF769FD069B0200002B05D11A4975
:1038C0001A4824F0DAFEFCF782FC19498D4227D110
:1038D0000E210791089109910399002922DD07978C
:1038E000039920000091059921F02BF8002811D0B0
:1038F000071B3A002100280021F042F8059B069999
:10390000DA1B521A7918079061182800089621F0DE
:1039100037F8099007A9032003F078FA0BB0F0BD3F
:103920000449D6E70997DBE79D5003000032030006
:1039300084320300F8DF020010B50100014821F0D5
:1039400030F910BD4945020010B50100014821F0D1
:1039500028F910BD5B450200F7B50600080001A973
:10396000FFF712FD019B0500002B01D11348FEBD9E
:10397000134B04009E4207D10027019A631B9A4211
:1039800011D8002F07D1F1E70E4B9E42F4D0019AD7
:10399000631B9A4201D80C48E9E72078B04701340C
:1039A0000028F4D1E2E72078FDF78AFC002803D054
:1039B0002078B047071ED9D00134DEE73C2403004D
:1039C00029130000411300004424030010B5010036
:1039D0000148FFF7C1FF10BDA912000010B501009A
:1039E0000148FFF7B9FF10BDC112000010B501007A
:1039F0000148FFF7B1FF10BDD912000010B501005A
:103A00000148FFF7A9FF10BD2913000010B5010000
:103A10000148FFF7A1FF10BD41130000F0B585B0CC
:103A200006000C001700FEF7F3FD694605003000A4
:103A3000FFF7AAFC0600042F23D1A30716D1124BCF
:103A400022689A4212D101AA210000980AF094FF3C
:103A5000002802D10D480CF0FFFF0199029A2800BE
:103A6000521A711820F08CFF05B0F0BD002322001F
:103A700000992800FEF78CFF335C01205B0018439F
:103A8000F2E70020F0E7C04608150300674C03008A
:103A900070B51D008AB0002968D01868344C030046
:103AA0002340062B05D083071FD1324B02689A4270
:103AB0001BD10239012953D806A9FFF765FC06007E
:103AC00028680440062C0ED1C00821F07BFD0400BC
:103AD0001020069D22F0C9FC274B85600360C6605C
:103AE00044600AB070BD4468F2E7012938D8012269
:103AF000104210D04410210006A825F0E3FB089BDB
:103B0000220000211800019328F04AFE06A91A4855
:103B1000FFF7CAFBE5E703A920F069FE002805D0FE
:103B2000049A0399144820F02BFFDAE72868FEF77F
:103B300071FF1021002800D0411006A825F0ABFB32
:103B400028680CF0DDF9040020000CF025FA0028AC
:103B5000DCD0FEF745FEC1B206A825F027FCF3E74E
:103B60000649074824F089FDFCF731FB0548B8E712
:103B7000070080FF8432030008E002004D4C030080
:103B800088310300F8DF020073B50400080001A9C2
:103B90001600FFF7F9FB0500042E06D10300019A79
:103BA0000749200022F060FD73BD0649200022F085
:103BB00090FC0123019A29002000FFF711FBF3E795
:103BC000AD50030051590300F7B502001C4B05002E
:103BD0000C001A401E00062A19D10B40062B04D1F6
:103BE000441A60426041C0B210E0C00821F0EAFC13
:103BF00007002640062E0CD1E00821F0E3FC002F40
:103C000009D0002807D0874205D00020FEBD4768B4
:103C1000EFE76068F3E769462800FFF7B5FB01A905
:103C200005002000FFF7B0FB009A019B01009A42BB
:103C3000EBD1280028F08AFD44426041D3E7C0461A
:103C4000070080FF084B07B50340062B08D0830709
:103C500004D10268054B92699A4201D0FFF7A0FA9D
:103C600001A9FFF791FB0EBD070080FF294200006C
:103C70000A4B13B503400C00062B08D0830704D170
:103C80000268074B92699A4201D0FFF789FA01A9AD
:103C9000FFF77AFB019B236016BDC046070080FF3B
:103CA00029420000F0B59BB00B900C000792102148
:103CB0000EAA12A8099313F02FF9079B9C4208D370
:103CC0000B9A12AB13CB13C21B6813600B981BB07B
:103CD000F0BD21787D2914D1631C0593079B621CDC
:103CE000934208D961787D2905D112A825F05EFBA1
:103CF000059C0134E1E7B549B54824F0BEFCFCF76A
:103D000066FA7B2904D012A825F050FB0594EFE752
:103D1000079B651CAB4243D961787B2904D112A86B
:103D200025F044FB0595E3E72B007D2903D02129ED
:103D300001D03A291FD100252E001A78212A23D03C
:103D40000022049200211A7805913A2A31D15A1C96
:103D50005B7805927D2B30D01300012207998B42AE
:103D60001ED219787B291FD101320133F6E7079A59
:103D700001339A4214D01A787D2A03D0212A01D027
:103D80003A2AF4D11E00D8E707995A1C914209D962
:103D90005A780492723A012A04D802339942D1D84F
:103DA0008C49A9E78C49A7E77D29DED1013A002A91
:103DB000DBD1059A0593069205E0079B059A93428D
:103DC000EED900230693059B1B787D2B01D08349F8
:103DD00092E7002D45D0002328781693FDF77CFA52
:103DE0002C00002822D0099B1B680893002B01DDC2
:103DF0007B4981E716AA3100280020F08AFD209A2D
:103E0000169B013A04009A4202D87649764874E734
:103E1000219A01339B009F580122099B52421A604C
:103E2000B4422ED271480CF017FE0134B44204D2D1
:103E300023782E2B01D05B2BF7D1611B01222800A8
:103E4000FFF768FA002205000100229808F0E4F963
:103E5000002804D12900664824F008FC4FE7476891
:103E6000DEE7099B1B68002B01DA624944E7209AD0
:103E7000013A9342C9D2013321999A005758099ABD
:103E80001360069B002B16D1049B002B58D010AA60
:103E9000102116A813F040F8049A3900733A531E03
:103EA0009A4110A8D2B2FEF7CBFB16A95248FFF7F1
:103EB000FBF9070002E0049B002BE8D101235B42E1
:103EC0000D931093069B002B00D1B6E00AF026FA62
:103ED000229B059A0293219B06990193209B16A889
:103EE0000093099BFFF7DEFE16A825F04EFA002688
:103EF000179B0400C3180A9303780493B34213D0AA
:103F00003E4D1900280028F099FDB04200D06FE125
:103F10006678002E17D03100280028F08FFD002889
:103F200000D067E106000490237808932B2B0CD077
:103F30002D2B48D00425202B08D00025089506E01D
:103F400073230493A3E70496EEE702250134237854
:103F5000232B02D1133B1D4301342378302B07D18F
:103F6000049B002B01D13D330493002E00D1303649
:103F70000DAA0A99200020F0CCFC037806902C2B87
:103F800004D10C3B1D43030001330693069B1B78B1
:103F90002E2B06D1069810AA01300A9920F0B9FC00
:103FA0000690069B1C78002C07D02100144828F0AE
:103FB00045FD002800D022E10400069B1B78002B61
:103FC00022D0104998E60025C0E7C0467B4D03008B
:103FD00000320300BC4D0300A34D0300D44D030089
:103FE000F84D0300424E0300582E03005B4E0300C1
:103FF000942E0300784E030084320300C24E030067
:10400000C74E0300D74E030016A825F06FF9049B96
:10401000002B08D13800FFF7ABF83C2304930028AD
:1040200001D002330493002E00D12036089B002BD0
:104030000CD0732C06D174495EE6069D2C002E0030
:104040000895E7E7632C01D1704955E6049B3D2BA9
:104050001FD05E2B1FD03C2B01D13B3B1D433800B2
:10406000FFF76AF800282DD0632C50D026D8472CB3
:1040700013D8452C26D2002C40D0252C22D0380035
:1040800020F09FFB220003006149624811F04AFFC3
:1040900035E64023E2E78023E0E7582C53D0622C3A
:1040A000EDD1002303930D9B02220293612301961D
:1040B000009539000EA808F0E9FF19E6672C17D81B
:1040C000652C1BD33800FFF753F800286CD0002C68
:1040D00056D06E2C54D0472C3FD8452C41D2252C9D
:1040E00050D0380020F06DFB220003004A49CCE795
:1040F0006F2C1AD0782C26D06E2CC0D100230393BD
:104100000D9B01960293009561230A22D1E73800A6
:10411000FEF766FB0D9B16A90870012201932B0088
:1041200000960EA808F056FFE2E5EB0602D58023C4
:104130009B001D43002303930D9B01960293009562
:1041400061230822B5E70022230003920D9A173B52
:104150000292019600951022ABE72300653B022BEB
:10416000BFD83800FEF7A0FB109B220002930D9BE6
:10417000011C01932B0000960EA822F02DFAB7E542
:104180006724EEE738008024FEF78EFB234917F002
:10419000E1FF109B640002930D9B2C430193011CD3
:1041A000009623006622E7E7049B3D2B01D11C49C2
:1041B000A2E5002C01D0732C13D116A93800FFF70B
:1041C00057FD109B0100169A002B00DA1092109BED
:1041D0009A4200D916930D9B00960193169A2B00D4
:1041E0009FE7380020F0EDFA220003000D494CE76C
:1041F000013499E633000234049E049394E6069B4E
:1042000001330693D9E6C046F04E03001C4F03006D
:104210004F4F030000320300804F03000000C842EC
:10422000B44F0300E94F0300F0B5A1B004000D0046
:104230000D920A2800D0E6E1073C0692144038D1DE
:104240001368BD4A93422ED10FAA10A9069820F0F8
:1042500018FE0694109B11A908930F9B2800099340
:10426000FFF792F800230A900C93AB0706D1B34AEC
:104270002B689B1A59425941CBB20C9314AA1021B6
:1042800018A812F049FE119A002794460A9B0A9C2E
:1042900063440593059BA34212D8089BBB4200D1FF
:1042A000A7E1A749B1E0A74A934202D10F94109425
:1042B000D0E70DAB0F930123109300230693C9E7BA
:1042C0002178252904D018A825F070F80134E1E7F9
:1042D000059B661CB34205D89B499C4824F0CDF948
:1042E000FBF775FF6178252904D118A825F05EF841
:1042F0003400EBE7002528290ED1A01C06003378F6
:10430000292B1CD1311A0122FFF704F8010006986D
:10431000FDF732FF0500013600233400402200265D
:10432000302104200B9320330793059BA34219D916
:1043300023782D2B0AD12C3B1E430134F5E7059B36
:10434000B34201D88249C8E70136D8E72B2B01D107
:10435000293BF1E7202B01D10643EEE7232B49D07F
:10436000302B44D000231293059BA34245D8012350
:104370005B421393059BA342AED923782E2B15D114
:10438000059B601C8342A7D963782A2B4FD1089ADA
:104390003B00BA4238D9099A9B009858FEF720FA98
:1043A000013713900234059BA34295D9002D07D104
:1043B000089A3B00BA4227D9099A9B009D580137B9
:1043C0002278672A5DD8652A00D3D1E0582A75D0B3
:1043D00035D81300453B022B00D8C9E00A9B5D4944
:1043E000E41A00941300594811F09CFD78E7164335
:1043F0000791A2E710230B939FE723782A2B0FD175
:10440000089A3B00BA4202D85349544866E7099AD1
:104410009B009858FEF7E4F9013712900134A6E7A3
:10442000200012AA059920F074FA04009FE70023E7
:1044300013AA0599139320F06CFA0400B3E7632ADA
:1044400049D0642ACAD103222B001340022B0AD17F
:10445000434B2B40062B06D0FF23DB05E818904387
:1044600004F0CEF90500139B0A220393129B0096D9
:104470000293079B01936123290014A808F006FE0C
:1044800024E7732A16D8722A00D381E0692ADAD089
:104490006F2AA3D10B9B002B02D084239B001E43C9
:1044A000139B00960393129B08220293079B019390
:1044B0006123E1E7752AC6D0782A8FD11300139AB9
:1044C000173B0392129A0292079A01920B9A164393
:1044D00000961022D0E7224B2B40062B05D0AB07CD
:1044E00016D1204B2A689A4212D11CA92800FFF746
:1044F000BFFB1C9A0100012A01D01B4985E7129BD2
:10450000019320230093330014A808F063FDDDE637
:104510002800FEF711FE00280BD02800FEF760F9F6
:10452000129B1CA9087001932023012200933300E1
:10453000EAE70E4969E7C04690EC020008E0020095
:10454000464D030084DE0200984C03000032030055
:10455000AA4C0300114D0300C04C03008831030036
:10456000070080FF84320300E74C0300004D030086
:104570002800FEF799F9139B22780293129B011CE5
:104580000193079B14A80093330022F025F89DE6C1
:1045900016AA10211CA812F0BFFC23781A00723A48
:1045A00050425041C2B2722B09D00C9B002B06D056
:1045B000AB0704D1544B2968994200D10422290049
:1045C00016A8FEF73DF8139A1D9B002A00DA1393F4
:1045D000139A9A4200D91A00129B1E990193202324
:1045E00014A80093330008F0F5FC1CA824F07EFE0C
:1045F0006CE60C9B4448002B00D1444818A9FEF7F8
:1046000053FE050019E00800FEF702F816A906009F
:104610002800FEF7B9FE0700072C22D118A90D9833
:10462000FEF71CF90025A84207D01899A94207DC1B
:10463000364B0E359E4200D0354D280021B0F0BDDE
:10464000169B1CA8594324F03DFE1E9B169A059309
:1046500000930121189B380022F058F91CA9300062
:10466000CDE70D98FDF7D4FF86420FD11CA90D9818
:10467000FEF78AFE1C9D05901D2C16D8192C3AD2E7
:10468000052C21D0122C1FD00025D6E71E4B00256B
:104690009E42D2D101221CA90D9820F0A8F8A84270
:1046A000CBD01C9B1D9D0593E6E71F2CECD101236D
:1046B000059A009316992B00380020F042F9154D09
:1046C0000028BAD1144DB8E7169B1CA8E91824F0AD
:1046D000F9FD1E9B169A39001800069328F045F83C
:1046E000169A1E9B94460693634418002A00059967
:1046F00028F03BF8B2E70095059B169A3900200098
:1047000022F038F9DBE7C04608E0020084320300FB
:10471000F8DF0200442403003C24030070B50C00C1
:104720008AB0050004A920681600FEF72DFE0023BC
:104730000593049B0100C218029605AB06A80194DC
:104740000095FFF7AFFA06A90248FEF7ADFD0AB0E3
:1047500070BDC04684320300F0B5050087B008681C
:104760000C00FDF755FF0090012D2AD96668022D37
:1047700028D0A068FEF734F805000021080020F0DA
:1047800010FB04A901902068FEF7FEFD049B0400C5
:10479000C7183F4B9E423FD1A7422CD92078FCF747
:1047A00083FD002811D1A74225D9002D0FD121006A
:1047B0003A1B009820F0E4F80100019800F0E4FFB3
:1047C00019E0334E01256D42D7E70134E4E72600B6
:1047D0003078FCF769FD002802D10136B742F7D1E5
:1047E0002100321B009820F0CBF80100019800F066
:1047F000CBFFB74202D8019807B0F0BD3400207853
:10480000FCF752FD002802D00134A742F7D1EB1784
:104810005B1BDB0FED1AC6E73000FDF7F9FE009BCE
:10482000834202D03000FEF7BBFC05A93000FFF741
:104830001FFA059B0390002B17D11649164823F049
:104840001CFFFBF7C4FC3E002100321B009820F047
:1048500097F80100019800F097FFB742CBD9059B6C
:10486000F418EB175B1BDB0FED1A2600059B029378
:10487000002DE8D0029BF3189F42E4D3029A0399DB
:10488000300027F063FF0028DED00136F0E7C04695
:10489000D0DB02009D50030000320300F0B50D0094
:1048A0008BB0022803D8FFF757FF0BB0F0BD0868A4
:1048B000FDF7AEFE08A9049028686C68FEF764FD59
:1048C0000090A868FDF78CFF431C0700002118002A
:1048D000059320F066FA354B05009C4202D134481E
:1048E0000CF0BAF809A92000FFF7C2F9099B06905D
:1048F000002B05D12F49304823F0BFFEFBF767FCA2
:10490000089A3C009446009B63440293BB000393C7
:10491000099B0193019A029B9E1A002C0BD0009BCD
:10492000B34208D8019A0699300027F00FFF0028FB
:1049300022D0013EF1E7EB68BE009C19009A029B71
:1049400000999A1A049820F01BF82060002F11D0CB
:10495000059BDC1BEB68A70099193A00180027F0AB
:104960000DFF6B6800211A1BEB689200D81927F025
:1049700017FFAC60280098E7039AEB6894466344FD
:104980000793029B04989A1B019B013FD21AF118CE
:104990001FF0F6FF079B02961860E3171B1BDB0F47
:1049A000E41A039B043B0393B2E7C046D0DB02004A
:1049B000B25003009D50030000320300C379024847
:1049C000002B00D101487047442403003C2403001D
:1049D00010B5FBF751FE014810BDC046D0DB020008
:1049E00010B50868FBF748FE004810BDD0DB020098
:1049F00073B50D00022838D1012601A96868FFF7B8
:104A000037F976423400019BC318834211D101A9C2
:104A10002868FFF72DF97342734162426241DBB2AD
:104A2000D2B20199FBF774FF002822D11149124834
:104A300017E00278722A01D0772A06D1611C0ED1C4
:104A4000723A544254410130DFE7622A01D0742A9D
:104A500005D1711C03D1743A56425641F3E7074918
:104A6000074823F00AFEFBF7B2FB0126764234002A
:104A7000CDE776BDA046030008300300C850030010
:104A80000032030010B50124037905499B005A58F0
:104A90000448224200D10448A243CA5010BDC04677
:104AA000CC020020442403003C24030010B5040081
:104AB0000FF018FA0C4988420AD020000FF054FA7F
:104AC000A02204216379D205C133FF339B009950A2
:104AD000A223A022DB00D205D0586379D84001235D
:104AE000184020F06AFB10BDE428030070B503797C
:104AF000064C05009B001859400820F05EFB01227F
:104B00002B799B0019590A401A5170BDCC02002024
:104B100010B504000FF0E6F9084B984202D02000CF
:104B20000FF0EEF9A0226379D205C133FF339B0069
:104B300098580007800F20F040FB10BDE4280300C8
:104B400013B50A4904000FF00FFA052168466156B3
:104B500012F084FF684612F0A7FFA0230021044A48
:104B6000DB00D15020F029FB16BDC046DC28030035
:104B70000070004070B504000FF0B4F9124DA84267
:104B800011D0124B98420ED020000FF0D7F9290017
:104B900020000FF0E9F9A0220C216379D205C1337E
:104BA000FF339B009950A0220C216379D205C133B9
:104BB000FF339B009950200009F040FA044B002875
:104BC00000D0044B180070BD14290300FC2803001A
:104BD000442403003C24030070B5A222A025D20087
:104BE000ED05AA581F23CA401100174C0340E05698
:104BF000421EC90700D5421C022A0BDC00218A4252
:104C00001CDB124DEE5C30008E4201D00220E954D4
:104C1000E25470BD072A09DD0C2A12DC0B4903207F
:104C2000CD5C002DF4D10238C854F1E707490320C8
:104C3000C95C4D1EA94149420840E9E70A00080045
:104C4000E6E703200C22E3E7600200204C0200208C
:104C500070B505000800FDF7C3FD0400431005D042
:104C60001249134823F009FDFBF7B1FA28000FF0B1
:104C700039F9104988420AD028000FF075F9A022AE
:104C800003216B79D205C133FF339B009950A022D9
:104C900001236979D2058B40002C04D0A121C900E1
:104CA0000548535070BD0549FAE7C046225103003C
:104CB00000320300EC280300D0DB02000C050000EA
:104CC00070B505000800FDF78BFD0B2303410400C0
:104CD000DB0705D40D490E4823F0CFFCFBF777FA2C
:104CE00028000FF0FFF80B4B984202D028000FF07D
:104CF00007F9FF22A40092001440A0226B79D2058C
:104D0000C133FF339B0004489C5070BDF450030036
:104D100000320300E4280300D0DB0200032370B557
:104D20000B4004000800022B03D11C4B0B40062B48
:104D300028D1FDF755FD1A4B05009D4205D91949AB
:104D4000194823F09AFCFBF742FA20000FF0CAF84A
:104D5000164988420AD020000FF006F9A02203214C
:104D60006379D205C133FF339B00995060792900E4
:104D700005F07CFC002D03D10D4920000FF0F4F864
:104D80000C4870BDFDF790FD19F0BEFA00220A4BE9
:104D900017F06AFD19F042FACDE7C046070080FF20
:104DA000FF03000001510300003203002C2903001F
:104DB000DC280300D0DB02000000E03F10B503490F
:104DC000034823F05AFCFBF702FAC046E550030003
:104DD0000032030010B50800FDF702FDFA239B0026
:104DE000584305F00FFC002801D0FFF7E7FF01480A
:104DF00010BDC046D0DB020010B50800FDF7F0FC86
:104E000005F000FC002801D0FFF7D8FF004810BDD6
:104E1000D0DB02001F22037901201340014AD35C3A
:104E2000584070474C02002010B5FFF7F3FF034BCA
:104E3000002800D1024B180010BDC04644240300D6
:104E40003C24030070B5CA4D28000FF04BF8C94C44
:104E5000A04205D028000FF045F8C74B98420BD16F
:104E600003210020FFF7B8FE022805D1C3490B68D3
:104E70009A1C012313430B60C14D28000FF032F838
:104E8000A04205D028000FF02DF8BB4B98420BD163
:104E900002210120FFF7A0FE022805D1B7494B6887
:104EA0009A1C012313434B60B64D28000FF01AF8EB
:104EB000A04205D028000FF015F8AF4B98420BD157
:104EC00001210220FFF788FE022805D1AB498B683B
:104ED0009A1C012313438B60AB4D28000FF002F89E
:104EE000A04205D028000EF0FDFFA34B98420BD145
:104EF00004210320FFF770FE022805D19F49CB68EB
:104F00009A1C01231343CB60A04D28000EF0EAFF4A
:104F1000A04205D028000EF0E5FF974B98420BD138
:104F200005210420FFF758FE022805D193490B699B
:104F30009A1C012313430B61954D28000EF0D2FFFC
:104F4000A0420BD028000EF0CDFF924B984205D026
:104F500028000EF0C7FF884B98420BD11121052085
:104F6000FFF73AFE022805D184494B699A1C0123B8
:104F700013434B61884D28000EF0B4FFA04205D0CA
:104F800028000EF0AFFF7C4B98420BD10C2106207D
:104F9000FFF722FE022805D178498B699A1C01236C
:104FA00013438B617D4D28000EF09CFFA04205D07D
:104FB00028000EF097FF704B98420BD10B21072071
:104FC000FFF70AFE022805D16C49CB699A1C012320
:104FD0001343CB61724D28000EF084FFA04205D030
:104FE00028000EF07FFF644B98420BD1122108205D
:104FF000FFF7F2FD022805D160490B6A9A1C0123D4
:1050000013430B62674D28000EF06CFFA04205D0E1
:1050100028000EF067FF584B98420BD10A21092057
:10502000FFF7DAFD022805D154494B6A9A1C012387
:1050300013434B625C4D28000EF054FFA04205D094
:1050400028000EF04FFF4C4B98420BD106210A204E
:10505000FFF7C2FD022805D148498B6A9A1C01233B
:1050600013438B62514D28000EF03CFFA0420BD041
:1050700028000EF037FF474B984205D028000EF06D
:1050800031FF3D4B98420BD11A210B20FFF7A4FDB5
:10509000022805D13949CB6A9A1C01231343CB62FC
:1050A000434D28000EF01EFFA04205D028000EF050
:1050B00019FF314B98420BD114210C20FFF78CFDC6
:1050C000022805D12D490B6B9A1C012313438B60D9
:1050D000384D28000EF006FFA04205D028000EF043
:1050E00001FF254B98420BD117210D20FFF774FDCE
:1050F000022805D121494B6B9A1C012313434B63B2
:105100002D4D28000EF0EEFEA04205D028000EF036
:10511000E9FE194B98420BD116210E20FFF75CFDDA
:10512000022805D115498B6B9A1C012313438B630D
:10513000224D28000EF0D6FEA04205D028000EF029
:10514000D1FE0D4B98420BD115210F20FFF744FDE6
:10515000022805D10949CB6B9A1C01231343CB6369
:10516000174D28000EF0BEFEA04231D02AE0C04606
:10517000CCE50200DC280300E4280300CC02002078
:1051800014E6020024E602002CE6020034E60200E7
:105190003CE60200FC28030044E602004CE6020064
:1051A00054E602005CE60200D4E50200DCE5020001
:1051B000E4E50200ECE50200F4E50200FCE5020093
:1051C00004E6020028000EF08DFE204B98420BD121
:1051D00010210800FFF700FD022805D11C490B6CC7
:1051E0009A1C012313430B641A4D28000EF07AFE1B
:1051F000A04205D028000EF075FE144B98420BD14A
:1052000000211320FFF7E8FC022805D11049CB6CE0
:105210009A1C01231343CB640F4D28000EF062FE4D
:10522000A04205D028000EF05DFE084B98420BD13D
:105230001E211420FFF7D0FC022805D104490B6D74
:105240009A1C012313430B6570BDC046E42803007C
:10525000CC0200200CE602001CE60200A0230C2277
:105260000249DB055A5024315A5070474407000068
:1052700010B50400FDF7CCF9084B98420BD0084B51
:10528000984208D0074B984205D00749074823F0B9
:10529000F4F9FAF79CFF200010BDC046B8E6020002
:1052A00054E5020090E50200D55003008831030068
:1052B0007822054B054890331B681A80743A5A804F
:1052C0001A715A717047C046380A0020D0DB0200BC
:1052D000084A10B5130090331B689979002908D04B
:1052E000116B0029F9D0002199711B69587905F0DB
:1052F000BDF910BD380A002013B5084C903423685E
:1053000018881FF05AFF2368009058881FF055FF37
:1053100069460190022001F079FD16BD380A00208F
:1053200010B50D4C002803D00868FFF7A1FF04005A
:1053300020000A490EF018FE6079002105F096F968
:1053400020000EF0FBFD0022054B064890331B6841
:105350001A619A7110BDC046CCE502000429030011
:10536000380A0020D0DB02001FB50C4B02AC0093C2
:105370000194022309F01CFC029A002A03D0084B76
:1053800090331B685A806268002A03D0044B903324
:105390001B681A80034804B010BDC04650E80200E4
:1053A000380A0020D0DB0200F0B5264B89B004ACEF
:1053B00000930194042309F0FBFB234F04223B00DC
:1053C00090331B6804981A715A71204B0340062BC6
:1053D00006D0830730D102681D4B92699A422BD1C7
:1053E000012303940293002590373B6818690EF05F
:1053F000A5FD3B6860681D61FFF73AFF154906008F
:105400000EF0B2FD144A3B6812689D719A60227BCF
:105410000299DA719981DD81039A012900D112681C
:105420005A6101221E619A71237A002B01D0FFF785
:105430004FFF0A4809B0F0BD03AA02A9FDF772FAAE
:10544000D1E7C046F0E70200380A0020070080FFDD
:105450002942000004290300D8080020D0DB020004
:10546000F0B5294B89B004AD01950093042309F0F0
:105470009FFB6B68A868049E0393FFF7F9FE234F18
:10548000040090373B6818690EF058FD00223B6815
:105490001F4920001A610EF067FD607980212D7B85
:1054A00005F0E4F8002E1DD1607905F067F9039B43
:1054B000002B14DB0022154B164990331B6809683A
:1054C00003989A710918DA719A81DA815A61023265
:1054D00099601C619A71002D01D0FFF7F9FE0E480A
:1054E00009B0F0BD31000D4815F09CFF05F08AF8B9
:1054F0000028DCD0607905F041F90949094823F01A
:10550000BCF8FAF764FEC04620E80200380A002022
:1055100004290300D8080020D0DB020040420F001D
:10552000375103000032030010B5182020F09DFF12
:10553000074B9033186078230380743B43800371DA
:1055400043710023837103614361024810BDC0466B
:10555000380A0020D0DB0200F0B56D4C87B0260081
:1055600090363368002B40D09A79002A3DD0694D9F
:105570009A6829688A4238D89A79022A0BD11B691D
:105580000021587905F072F82B6832680A3393606D
:105590000123937129E09A79012A26D19A89D98920
:1055A000914204DBDD79002D19D00021D9815869A1
:1055B000012A02D0DA8992008058574A904216D1C7
:1055C0001B6900215879903405F050F8246853483D
:1055D000218815F0B1FF0123A060A37105E09D7142
:1055E00018690EF0ABFC33681D6107B0F0BD05A96A
:1055F000FEF73EFB9034236801901B6980215879A7
:105600000293059E05F032F8019B24681F781F2342
:10561000218842481F4015F08FFF618815F08CFFEC
:105620007D1EEDB20390012E5AD9019B5B78232B8E
:105630004DD0622B50D1002D4BD0023FFDB26A1EDF
:10564000514251414A42022E4ED00121022301987B
:10565000C05C3A2803D00F273840207101332079ED
:1056600084469E420ED90198C05C3A280AD1581C43
:10567000864207D9019F0233385C0F2738409E428B
:1056800035D86071092D3DDC6346043B9A1852B24F
:105690006F00234B002900D1224BD85B002A2EDB60
:1056A000104104F0AFFF1A4B039990331A685379F5
:1056B00059430B000A3B0A2B00DA0A2315490968F3
:1056C000CB189360D3890133D381022361E7002291
:1056D000B9E72A000625B6E7002101230A00B6E74C
:1056E000002101230A00BAE733000121B7E70A26A7
:1056F0007043019E6071F65C3E408019C1E75242E2
:105700009040CEE7029B0021587904F0AFFFCAE732
:10571000380A0020D8080020D0DB020060EA000030
:10572000B0450300A2450300002803D0012807D09C
:10573000002004E08B680448002B00D10348704728
:105740008B685B001843FAE7442403003C24030001
:1057500000228168F0B5CB0F094C5B185B100E1965
:105760009A4201DB0748F0BDC568B11A9400890070
:105770002C196D5827682560C46801326750EFE71F
:10578000FFFFFF3FD0DB020070B583680D0041686A
:1057900004008B4212D3C900C06820F07CFE63680D
:1057A0000A495A00A3686260D21A013352189B005A
:1057B000E0609200C018002126F0F2FFA368E268C2
:1057C000591C9B00A16002489D5070BDFFFFFF3F28
:1057D000D0DB0200F8B5070016004C10836803D533
:1057E000E418E243D2171440A34200D21C000B4934
:1057F0003800FFF7C9FFBB68094A591E9B189B0078
:10580000181FFA688C4203DBA40016510348F8BD48
:1058100015580139D5500300F2E7C046D0DB02002D
:10582000FFFFFF3F70B50025040085601021C068B0
:1058300020F031FE04232900E0606360102226F08E
:10584000AFFF014870BDC046D0DB020030B50C0090
:1058500085B0104B02AD043100930138022301954D
:1058600009F0A6F923680C4C996801290FD9D8686A
:105870000A4B029AC91889004118A24200D100229D
:105880002D79074B002D00D1064B1FF0E0F92000C9
:1058900005B030BDBCE80200D0DB0200FFFFFF3FD7
:1058A0003C2403004424030070B50C680B00A1687D
:1058B0000200002905D11A491A4822F0DEFEFAF743
:1058C00086FC2068012A27D05A680023FDF760F87B
:1058D000E168A26886008B19013A1D680436A2604F
:1058E000121A92008919180026F048FF0021A368B7
:1058F000E0689A001150616804290BD95B00994255
:1059000008D949088900E06820F0C5FD6368E060B7
:105910005B086360280070BD01225242D5E7C04693
:1059200045510300582E030007B500900191022055
:1059300069461FF0F2F9694601900220FFF7B4FFB3
:1059400000480EBDD0DB020070B50E000D49050009
:10595000002420F0BEFDB3689C4204D328000A490D
:1059600020F0B7FD70BD002C03D00849280020F0BE
:10597000B0FDF168A300012259582800FCF760FE31
:105980000134E8E7EFCB03007ED603003C48030078
:1059900070B5032604000D000E4029D1174B0A688C
:1059A0009A4225D183688A6899184368994210D928
:1059B00004318900C06820F06EFDAA68A368E06029
:1059C0009B181A1D9B006260C0181022310026F03F
:1059D000E7FEA368E9689800E3681818AB689A00C6
:1059E00026F0C3FEAB68A268D318A360044870BD5C
:1059F000290020001FF09AF9F8E7C046C0E902002C
:105A0000D0DB020010B50400102020F02EFD044B66
:105A100084600360034B43600023C36010BDC04635
:105A2000C4060300334C02000B4B70B50500036045
:105A30000C000800042900D204206860AC608000DB
:105A400020F013FD6A68E860121BA40092000019A0
:105A5000002126F0A5FE70BDC0E902007FB50C0054
:105A6000150012283CD005D8052819D007283CD0AD
:105A7000002432E00300193B042BF9D893070DD121
:105A8000284B12689A4209D1AB6800938A68EB6888
:105A9000C96808F0ABFF244C00281ED1234C1CE041
:105AA00003231340E4D11F4A2968914238D1A368E7
:105AB000AA6898181FF052F90600A368E1689A00D6
:105AC000C06826F052FEA068F36880001818AB6822
:105AD000E9689A0026F049FE3400200004B070BD49
:105AE00011002000FFF754FFF7E703A91000FCF7AF
:105AF000B5FE0028BCD0039B002B01DA00230393E2
:105B0000A368039858431FF029F90500C3680421CE
:105B10000093A268E068039B20F0F8FE2C00DCE70D
:105B20001C00DAE7C0E90200442403003C2403001F
:105B3000F0B5040087B017000326002A29D10E40D3
:105B40001FD1544B0A689A421BD103AA806808F0FF
:105B500013FF0499039BA268E0685D1A521A89003A
:105B6000920041189B00181826F008FEA368AA00AE
:105B7000E818E368800052421818310026F010FE41
:105B80006BE00491022003A90394FFF78DFE4248C5
:105B900012E0042A2DD1314221D13E4B0A689A42AB
:105BA0001DD103AA806808F0E7FE002806D103AAE9
:105BB000E168A06820F0BDFE07B0F0BD039B04982B
:105BC000C01A1FF0CBF805008368E1689A00039BB8
:105BD000C0689B00C91826F0C8FD2800ECE7002328
:105BE0000A002068A168FCF7D3FEE3688000C05873
:105BF000E2E70E4048D1274B0A689A4244D103AAF3
:105C0000806808F0B9FE049B0398BA68C51AAD18FD
:105C10000193002D25DDA368E9186368994207D92F
:105C20008900E06820F037FCA368E0605B196360DE
:105C3000039BA268E068D21A9900EB189B004118F8
:105C40009200C01826F09AFD039BF9689800E3685B
:105C50001818BB689A0026F088FDA3685D19A56036
:105C600095E7E3688000F9681818920026F07DFD3A
:105C70000499B868A268039FE368521A381889002B
:105C80009200591880006EE73A0020001FF0A7F834
:105C90007DE7C04608150300D0DB02000123064A59
:105CA0001370064A1060064A06481160064A1370CF
:105CB0000022064B1A707047990B0020CC09002077
:105CC000D8090020442403003209002033090020B1
:105CD00000487047D0DB0200F0B595B005AC3C221F
:105CE0000021200026F05CFD00250EF065F800285C
:105CF00004D1042D0BDC704815B0F0BD0EF068F82F
:105D0000C0B2605501350D28F3D03D2DEDD10622EE
:105D10006A49200026F0B1FE002806D1684B664A89
:105D20006849186820F081FFE5E7052266492000F0
:105D300026F0A3FE051E15D10A21614B02001E6844
:105D40006248FDF7E7FA0700200026F08FFEC11F2A
:105D5000112002AB2A00C018FDF7DCFA390002005E
:105D60003000DFE706225A49200026F086FE051E95
:105D700010D1534B0200092156481C68FDF7CAFA9E
:105D80002A00022106005448FDF7C4FA310002003F
:105D90002000C7E705225149200026F06EFE051EAF
:105DA00005D1474B02001E680D214D48C9E7062268
:105DB0004C49200026F061FE051E0BD1404B02002D
:105DC0000C2149481C68FDF7A5FA2A0006000421A9
:105DD0004648D9E70A224649200026F04EFE021E18
:105DE00008D10C21364B43481C68FDF793FA324A20
:105DF0000100CDE70A224049200026F03EFE021EA7
:105E000004D12F4B05211C683C48EEE70A223C498F
:105E1000200026F032FE021E04D1294B08211C6806
:105E20003848E2E705223849200026F026FE051E04
:105E300005D1234B02001E680A21344881E707225E
:105E40003349200026F019FE002827D10A2200211C
:105E500002A826F0A5FC0725635D6E1C7C2B18D1DB
:105E6000174B02A81B68019326F000FE00220100D8
:105E700002A8FDF74FFA0700200026F0F7FD0338CF
:105E8000411B0022A019FDF745FA390002000198D4
:105E900048E7073D02AA53553500DDE708221D49B2
:105EA000200026F0EAFD021E00D024E7044B0E215C
:105EB0001C68194899E7C046D0DB0200A1510300D5
:105EC000D009002059510300605103003B640300D6
:105ED000665103005B6403006D51030070510300C1
:105EE00076510300845103008B5103009851030045
:105EF0009D510300A8510300B5510300C051030098
:105F0000C6510300D1510300DA510300F5510300DB
:105F1000E0510300E8510300F151030010B5054CB6
:105F2000200026F0A3FD002201002000FDF7F2F979
:105F300010BDC046DC09002010B505481DF040F832
:105F4000044B1B6898681CF0ABF9034810BDC046B1
:105F50007C5303007C000020D0DB0200F8B52A4D02
:105F6000002107003C22280026F01AFCFA21A92370
:105F70008900264EDB00264C8F4231DD254A3068F1
:105F8000C250380015F0D8FA20600122002433688E
:105F9000214F1A603C700DF00FFF002803D00DF068
:105FA00017FF285501340DF007FF00281FD12B19CA
:105FB000013B1B780D2B1AD1012233685A603B78C4
:105FC0002800002B0BD00022144B3A701A60336863
:105FD00013481900FC31CA640132DA605A60F8BD16
:105FE0001F2078433268D05001232360CDE73B78EF
:105FF000002B05D00B4B1B6898681CF051F9DEE7AD
:106000003C2CC8DDF6E7C046EB0900201800002054
:106010002403002018790000340900202003002008
:10602000BB5303007C00002010B505481CF0C8FFDE
:10603000044B1B6898681CF033F9034810BDC04638
:10604000A25303007C0000204424030010B505483F
:106050001CF0B6FF044B1B6898681CF021F903483C
:1060600010BDC046835303007C000020D0DB02003B
:10607000104BF7B5060018680F00FDF7E3FD0E4B57
:1060800004001868FDF7DEFD05003000FDF7DAFDBD
:1060900006003800FDF7D6FD33002A0000902100ED
:1060A00006481CF08DFF064B1B6898681CF0F8F83A
:1060B0000448FEBDC8090020D40900200052030096
:1060C0007C000020D0DB020010B5FDF7BBFD010015
:1060D00004481CF075FF044B1B6898681CF0E0F83E
:1060E000024810BDAF5303007C000020D0DB02004B
:1060F00070B50D00FDF7A6FD04002800FDF7A2FD18
:106100002100020004481CF05BFF044B1B689868E8
:106110001CF0C6F8024870BD935303007C000020B9
:10612000D0DB020070B5154E040030001CF048FFB3
:10613000134B1B6898681CF0B3F8124B1B78002BAC
:1061400002D0114B180070BD2000FCF749FBFFF78F
:1061500005FF040026F08AFC310005000200200043
:1061600026F08BFC0028ECD02A000849200026F0FD
:1061700084FC074B0028E5D0064BE3E7A151030060
:106180007C0000203309002044240300BB5303009B
:10619000D0DB02003C24030070B5040019481CF059
:1061A0000FFF194B1B6898681CF07AF8174B1848BA
:1061B0001E78002E14D12000FCF712FBFFF7CEFE54
:1061C00005221449040026F058FC05002000002D8B
:1061D00007D126F04BFC2A00C11F601DFDF79AF87D
:1061E00070BD26F043FC0C4D02002900200026F073
:1061F00044FC021E02D107212800EFE732000321F0
:106200000648EBE72C5203007C00002033090020F5
:106210004424030060510300BB5303008362030066
:10622000F8B50400FCF7DCFA010018481CF0C8FEC1
:10623000174B1B6898681CF033F8164B16481D78EE
:10624000002D13D12000FCF7CBFAFFF787FE0400E6
:1062500026F00CFC114902000700200026F00DFC7E
:10626000021E04D102210E48FDF754F8F8BD0D4E70
:106270003A003100200026F000FC021E02D1072166
:106280003000F1E72A0003210748EDE7225203001E
:106290007C000020330900204424030066510300E1
:1062A0006D510300BB5303008362030070B505000A
:1062B00019481CF085FE194B1B6898681BF0F0FF0D
:1062C000174B18481B78002B25D12800FCF788FABB
:1062D000FFF744FE14490522040026F0CEFB011E00
:1062E0000ED1124D0F22280026F05AFA200026F077
:1062F000BDFB611DC21F280026F037FA09480AE0DD
:10630000200026F0B3FB0A490200200026F0B5FB6E
:106310000028DAD1074870BD8C5303007C000020B0
:10632000330900204424030070510300DC090020DD
:10633000BB530300D0DB0200054B10B51B780100F6
:10634000002B04D0034822F098F9F9F740FF10BD64
:106350003309002088310300F0B5070087B03E48BC
:106360000D00FFF7E9FF3D4B1868FDF76BFC3C4B58
:1063700004001868FDF766FC06003800FDF762FCB3
:1063800032000300210037481CF01AFE364B1B6810
:1063900098681BF085FF2800FCF722FAFFF7DEFD66
:1063A000040026F063FB314907000200200026F0BC
:1063B00064FB0028EFD007222D49200026F05DFB6A
:1063C00003AD061E0FD1C8201EF0F7FE039020007B
:1063D00026F04CFB010032000939E01DFCF79AFF62
:1063E0002900686017E023490322200026F045FBBE
:1063F000011E19D10A22280026F0D2F90323E25CFB
:106400007C2A0DD1280026F037F91EF0D6FE1A4B53
:106410000190029301A9022000F0F8FC07B0F0BD42
:10642000D91E6A540133EAE720003A00134926F0E6
:1064300024FB041E07D112481EF0BFFE2200039069
:106440000E211048CAE7CC2040001EF0B6FE002204
:10645000039008210C48C1E780520300CC090020BA
:10646000D8090020B05203007C00002066510300D0
:10647000C752030072510300D0DB0200B951030080
:10648000E7030000CF520300DE520300F0B5060020
:106490008BB041480F001400FFF74EFF3F4B1868C8
:1064A000FDF7D0FB3E4B03901868FDF7CBFB0500D2
:1064B0003000FDF7C7FB06003800FDF7C3FB3300D3
:1064C00000902A00039937481CF07AFD364B1B6870
:1064D00098681BF0E5FE2000FCF782F9FFF73EFD0F
:1064E000050026F0C3FA314906000200280026F014
:1064F000C4FA0028EFD007222D49280026F0BDFA63
:1065000007AC071E0FD1C8201EF057FE07902800C9
:1065100026F0ACFA01003A000939E81DFCF7FAFE52
:106520002100606017E023490322280026F0A5FA25
:10653000011E19D10A22200026F032F90323EA5C59
:106540007C2A0DD1200026F097F81EF036FE1A4B5B
:106550000590069305A9022000F058FC0BB0F0BD91
:10656000D91E62540133EAE728003200134926F0AD
:1065700084FA051E07D112481EF01FFE2A0007905C
:106580000E211048CAE7CC2040001EF016FE002263
:10659000079008210C48C1E7E7520300CC0900200E
:1065A000D8090020185303007C0000206651030026
:1065B000C752030072510300D0DB0200B95103003F
:1065C000E7030000CF520300DE520300F0B50600DF
:1065D0008BB041480F001400FFF7AEFE3F4B186828
:1065E000FDF730FB3E4B03901868FDF72BFB0500D1
:1065F0003000FDF727FB06003800FDF723FB3300D2
:1066000000902A00039937481CF0DAFC364B1B68CF
:1066100098681BF045FE2000FCF7E2F8FFF79EFCAF
:10662000050026F023FA314906000200280026F072
:1066300024FA0028EFD007222D49280026F01DFA61
:1066400007AC071E0FD1C8201EF0B7FD0790280029
:1066500026F00CFA01003A000939E81DFCF75AFE51
:106660002100606017E023490322280026F005FA84
:10667000011E19D10A22200026F092F80323EA5CB9
:106680007C2A0DD1200025F0F7FF1EF096FD1A4B55
:106690000590069305A9022000F0B8FB0BB0F0BDF1
:1066A000D91E62540133EAE728003200134926F06C
:1066B000E4F9051E07D112481EF07FFD2A0007905D
:1066C0000E211048CAE7CC2040001EF076FD0022C3
:1066D000079008210C48C1E732530300CC09002081
:1066E000D8090020625303007C000020665103009B
:1066F000C752030072510300D0DB0200B9510300FE
:10670000E7030000CF520300DE520300F0B506009D
:106710008BB041480F001400FFF70EFE3F4B186886
:10672000FDF790FA3E4B03901868FDF78BFA0500D1
:106730003000FDF787FA06003800FDF783FA3300D2
:1067400000902A00039937481CF03AFC364B1B682E
:1067500098681BF0A5FD2000FCF742F8FFF7FEFB50
:10676000050026F083F9314906000200280026F0D2
:1067700084F90028EFD007222D49280026F07DF962
:1067800007AC071E0FD1C8201EF017FD0790280088
:1067900026F06CF901003A000939E81DFCF7BAFD52
:1067A0002100606017E023490322280026F065F9E4
:1067B000011E19D10A22200025F0F2FF0323EA5C12
:1067C0007C2A0DD1200025F057FF1EF0F6FC1A4B55
:1067D0000590069305A9022000F018FB0BB0F0BD50
:1067E000D91E62540133EAE728003200134926F02B
:1067F00044F9051E07D112481EF0DFFC2A0007905D
:106800000E211048CAE7CC2040001EF0D6FC002222
:10681000079008210C48C1E733520300CC0900203F
:10682000D8090020665203007C0000206651030056
:10683000C752030072510300D0DB0200B9510300BC
:10684000E7030000CF520300DE520300A122002123
:106850000920284BD2001B6870B599500832985017
:106860008022F830D202FF301A502348C024195039
:10687000A9212248C9005850C12189005A501F221D
:1068800001211F4B64001B785BB2D8B202409140DB
:106890001C4A1151002B18DA0F230340083B1A4CF5
:1068A0009B089B001B1903242040A040FC3484401B
:1068B000DD69A5432C00C025854028002043D86110
:1068C000C0235B00D150116070BD9C080D4BA4002B
:1068D000E41803230340FF20C025DB009840AD00EF
:1068E000665986433000C0269E40330003436351FF
:1068F000E6E7C046180000200405000018790000F3
:106900007402002000E100E000ED00E010B5012479
:106910000A4B1C700A4B18600A4B19600A4B1A602C
:106920000A4B1C70FFF792FFA922094B09491B680B
:10693000D200995008485C601C6010BD990B002083
:10694000D0090020C8090020D40900203309002004
:10695000180000206A180000D0DB0200F0B5002506
:10696000374B384E1D70384B93B01D703378009004
:1069700001911700354CAB4227D00D201CF070FB65
:10698000236898681BF08CFC3570FA260335B60036
:106990002F481CF015FB2368013D98681BF080FC14
:1069A000300014F0E7FB002DF2D103AE3C222900A9
:1069B000300025F0F5FE0DF0FFF9002805D00DF0B0
:1069C00007FA705501353D2DF5D1FFF73FFF0098CF
:1069D000FDF738F905000198FDF734F929000200A8
:1069E0001C481CF0EDFA236898681BF059FC38002D
:1069F000FBF7F6FEFFF7B2FA17490522040026F06E
:106A00003CF8011E0ED1154D0F22280025F0C8FEBE
:106A1000200026F02BF8611DC21F280025F0A5FEDE
:106A20000F480AE0200026F021F80E49020020005D
:106A300026F023F80028DAD10B4813B0F0BDC04689
:106A40003309002075020020320900207C0000205C
:106A5000A15103001552030070510300DC0900200E
:106A600044240300BB530300D0DB0200174B70B576
:106A70001D78174C002D0BD0FFF72EF9236800214D
:106A80001A00FC32D16401225A60DA601A6070BDCB
:106A90002368104A1900FC31CC6C012C09D1C120AB
:106AA00080001858400304D51068CD640130106090
:106AB000DC601068084A12689042E8DB012207484F
:106AC0005A6002700020C864DA60E0E733090020F1
:106AD0001800002020030020240300203409002097
:106AE00073B501A9FDF7C4F8019B06001849502BA6
:106AF00016D8802040001FF0B8FC164C0500231D5E
:106B0000D8670023019A93420FD15B222800EA54F0
:106B100007F05AFC2B0000280BD104340E49E06723
:106B20000E4821F0AAFDF9F752FBF15CE95401335C
:106B3000E9E75A1B0133591E09789B29F9D129002D
:106B400007481DF01DFF00230434E36776BDC046EF
:106B5000D2530300380A0020E1530300003203003F
:106B600084320300F0B58BB00600080011001A0053
:106B700010AB1F78334B05AD01950093052308F04A
:106B800017F8912000011FF070FC2F4B04A9D86763
:106B900002AB1B7B476043702B792C4F03702B7A21
:106BA000040083702B7BC3702B7C30003B60FDF7AF
:106BB0005FF80025264B03900C201D601FF055FC4C
:106BC000244B0600036006F04FF8B06006F04CF866
:106BD000214B224A1860224B11001D70214B70601E
:106BE0001D70214B30001D602B0005F013FF2000AD
:106BF000049A039921F049FC20000EF02BFB0400BD
:106C0000A8420AD105F014FE0F4B1848DC67184B58
:106C1000196821F032FDF9F7DAFA0122154B1A70E2
:106C200006F01CF80028FBD1134B0433D8673B68EF
:106C3000002B04D00C4B114819681CF0C1F907480F
:106C40000BB0F0BDD4EB02003C0A0020A4030020EE
:106C50002C03002034EC020028030020D0DB0200CB
:106C600037090020350900203003002000320300DE
:106C70007000002036090020380A0020C3530300AA
:106C800000220D4910B50B78DBB2934210D10B4AAC
:106C90001478002C02D001240C701370084B1B7860
:106CA000002B07D0074A136820331360064B1A687D
:106CB000100010BD8268FBE735090020360900206E
:106CC000370900202C03002028030020D2235B007A
:106CD0005843134AF0B51368000C984206D2114C81
:106CE0002368013323601368203B13601F230500D2
:106CF00001270D4E9D431468A5420BD803401A1D71
:106D0000202A00D92022094C2468934204D3084B3E
:106D10001860F0BD3770EEE7E51829710133F4E72C
:106D20002C03002030030020370900202803002016
:106D30003403002070B50E001049040000251FF038
:106D4000C8FB73689D420AD3012B03D10C49200074
:106D50001FF0BFFB0B4920001FF0BBFB70BD002DD7
:106D600003D0094920001FF0B4FBAB00F318012247
:106D700099682000FBF764FC0135E2E7018A030013
:106D8000F8530300C14A03003C48030070B50D00EE
:106D900001281ED0002803D0022807D0002004E0DC
:106DA0004B680E48002B00D10D4870BD00260D4CDD
:106DB0006B689E4203D3012064002043F5E7B300D3
:106DC000EB189968022008F039FF401024180136AA
:106DD000EEE74B685B001843E7E7C0464424030036
:106DE0003C24030088EC020010B5040010201FF0C2
:106DF0003CFB044B84600360034B43600023C3608F
:106E000010BDC046C4060300434E020070B5060024
:106E10000D000C48002E0FD0B41CA40020001FF061
:106E200024FB094A030002604660002D04D00022C2
:106E3000083C944201D1180070BDA8589918886088
:106E40000432F6E788EC020090EC0200F0B5040092
:106E500085B00D00160007284CD003D8052824D093
:106E6000002144E00300193B042BF9D80800FBF78C
:106E7000CFFB3000FBF7CCFB2C4B426A9A4205D08B
:106E800030002B4922F0B9F9061E0CD0330029003E
:106E900072680831009208336A68200007F0A6FD86
:106EA0002449002823D1244921E01000FBF7B0FB3E
:106EB0001F490FF0ABFF011E19D06B6872680021EB
:106EC0009818FFF7A3FF070029006B6808379A009E
:106ED00008310400380025F048FC31006868736808
:106EE000800038189A00083125F03FFC2100080086
:106EF00005B0F0BD03A91000FBF7B0FC00218842EB
:106F0000F5D0039888420FDD6B685843FFF77EFF8A
:106F1000040023002800083300930830039B6A68AC
:106F200004211FF0F3FCE1E70449E0E7E96D00000C
:106F300090EC0200442403003C24030088EC02008F
:106F400030B5040085B0042A2DD103250D4020D191
:106F5000164B0A689A421CD101AA406807F00CFD42
:106F6000002802D1124809F077FD019B0298290000
:106F7000C01AFFF74BFF050021006B6808319A002B
:106F8000019B08309C00091925F0EFFB280005B093
:106F900030BD0A00002361682068FBF7F9FC02306D
:106FA00080000059F3E70020F1E7C0460815030010
:106FB000674C0300F0B50C001100002285B01E00E4
:106FC00000920123200007F0C1FD184D002C1DD0B8
:106FD0003568AB0703D1164B2A689A4216D01020A9
:106FE0001FF043FA0400306808F08AFF00250426E9
:106FF0000390039808F0D0FF071E0AD12800210053
:10700000FFF704FF050020001FF056FA280005B026
:10701000F0BDAE4205D8F10020001FF03CFA04009C
:107020007600AB001F510135E3E7C04688EC020053
:1070300090EC020010B504000C201FF016FA034B70
:107040004460036001235B42836010BD04ED0200D5
:10705000F8B50D000400160005F094FE2B00032780
:1070600023433B4219D1BE4217D9B2082900200060
:1070700014F054F93100B94360183E406918002EED
:1070800002D0320025F0B8FA80220549D2008B5890
:10709000002BFCD005F066FEF8BD29002000EEE7CD
:1070A00000E00140F0B5836999B05A1E06339B0099
:1070B0000492C218079102920F210122C3180433CF
:1070C00003930369019006A81A4009180A70032265
:1070D00093430A930CA8F9F75FF8031E01D000F060
:1070E0003FFD019A5568D468079A002A00D184E2CE
:1070F0002A785E2A00D180E20798079309F0C4FB42
:1071000004000AE0D24B63600434D24B1A6B002AAD
:1071100000D171E200221C6B1A63F9F753F80D9449
:1071200000F01EFDCC4BEEE7CC4BECE77F216B78FB
:107130005B06DB173A78DB01100052B208400343CC
:107140000137002AF6DB01225B001343DBE7002353
:107150007F213A78DB01100052B20840C318013792
:10716000002AF6DBDB000622EFE703220337974312
:1071700008CFC8E70023C6E700237F213A78DB0168
:10718000100052B20840C3180137002AF6DB9B00FA
:107190005B42029A9858002800D0EEE2B049B1480C
:1071A00021F06BFAACE700237F213A78DB01100075
:1071B00052B20840C3180137002AF6DB029A9B003E
:1071C0005B42985821F024F9E5E700207F223B78C4
:1071D000C00119005BB2114008180137002BF6DB23
:1071E000251D08F0CFFC60605EE000207F223B7828
:1071F000C00119005BB2114008180137002BF6DB03
:10720000251D08F08DFCEEE700217F223B78C901A7
:1072100018005BB2104041180137002BF6DB2068E4
:107220001FF01BFD206070E700217F223B78C90121
:1072300018005BB2104041180137002BF6DB22002A
:1072400001CC08F011FE60E7251D08F0B3FCCAE789
:10725000251F042221682868FBF74AFC286023E0E8
:1072600000237F213A78DB01100052B20840C31896
:107270000137002AF6DB9B005B42029A2168995095
:10728000E3E000237F213A78DB01100052B208408E
:10729000C3180137002AF6DB9B00029A5B42216883
:1072A0009858251F21F0B6F82C002EE700207F22E9
:1072B0003B78C00119005BB2114008180137002B60
:1072C000F6DB2168251F08F089FCEDE700207F220E
:1072D0003B78C00119005BB2114008180137002B40
:1072E000F6DB2168251F08F091FCDDE700217F22F5
:1072F0003B78C90118005BB2104041180137002BE0
:10730000F6DB231F1A68206808F0D6FD083CFCE66F
:107310002200231F083A126821681868FBF7E8FB6F
:107320000C3CF2E600237F213A78DB01100052B2D8
:107330000840C3180137002AF6DB029A9B00D31AD3
:107340001A68002A00D129E700221A60DDE600252C
:107350007F223B78ED0119005BB211404D190137D6
:10736000002BF6DB029BAD005D1B286821F050F876
:10737000002800D112E70021286821F04BF8C4E66C
:1073800000207F223B78C00119005BB21140081831
:107390000137002BF6DB08F02DFCB6E600207F223B
:1073A0003B78C00119005BB2114008180137002B6F
:1073B000F6DB08F037FCA8E62368A4E62368A360A0
:1073C000231F1B68636008349FE6231F1968226827
:1073D0002160BAE7221F1368216823602300083B5D
:1073E00018681060196090E67B783A781B021343A6
:1073F0001D4A9B18EF1888E67E783B782068360295
:107400001E43FBF72BFBEF1C251F2C00002800D18F
:107410007BE6164BF618BF1977E67E783B78206836
:1074200036021E43FBF71AFBEF1C251F2C00002819
:1074300000D06AE6EDE77E783B78360220681E438E
:10744000EF1CFBF70BFB0028E3D1043C5DE6C046D4
:107450003C240300380A0020D0DB0200442403004F
:10746000FA530300902F03000380FFFF0080FFFF0B
:107470007E783B78360220681E43EF1CFBF7EEFA5D
:107480000028C6D0E1E7260027682200380017212F
:10749000083608F0E9FC38003200162108F0E4FC58
:1074A0000021320008001FF0C9FBAB786A781B028C
:1074B00013430A9A0F210C320A920A9AEF1CFB1806
:1074C0001360022206ABC9180A9D0B781A43231DCC
:1074D00013436B6000230A9A0B709360A060340022
:1074E00013E625002668AC4B083D9E4208D1666035
:1074F000A6602A00002103201FF0A0FB2E60D3E627
:10750000012131402CD07610231F012E11D12600ED
:107510001A680C3E0592A04A00211A6003202260DE
:10752000626032001FF08AFB059B336003232B60EF
:10753000ECE626002A68103E05921A6800210692A1
:10754000954A03202A601A60226032001FF076FB01
:10755000059B069A336023000C3B1A600523E6E77F
:107560002B682E602600103E2360320003201FF09F
:1075700065FBFBF773FA00280DD00122864B06A9A4
:1075800033600A9B5B6813400E32521813700A9BDB
:107590000C3B0A93A3E7236833602300043C226872
:1075A0000C3B1A6080E67B783A781B0213437B4AD7
:1075B0009B18EB186360EB78083423600F267F215B
:1075C0000220012506AA2368B6180B4205D1221F06
:1075D0001768002B00D0A3E698E60A9A013B526890
:1075E000024270D0220008C20523636014000A9B87
:1075F0001F680A9B0C3B0A933D00019B6F1C5D605A
:107600002B78180010385A2800D907E313F0F6FE3B
:107610007AFD8AFD8CFD06038EFD06039FFDADFD00
:10762000B2FD0603B4FDCBFDDDFDEDFDFCFD0CFE62
:107630001CFE20FE28FE39FE4EFE5EFE6EFE80FE23
:107640008AFE9FFEB8FEC6FE060306030603060377
:10765000D4FED6FE1DFFDDFEE2FEECFEF4FE05FFCD
:1076600013FF30FF0603060306033BFF69FF6300B9
:1076700063008000A300A700B700B700CBFF06039C
:1076800006030603060306030603060306030603B2
:10769000C800DA00EC00FE000D0116012B013D01CF
:1076A0004F016C0182013002570282026F02060311
:1076B0009701A201AD01BA01C601E201FC01190264
:1076C000DA02EF0200030A9A52682A4032700A9ADC
:1076D0000C3A0A9279E77B783A781B0213430A9AAC
:1076E000EF1C0C320A920A9AFB1813602B780A9A44
:1076F000403B584258410F21430006A8091808781A
:1077000003432343536000230A9A0B709360FCE405
:1077100020680EF04FFC251F002804D0F8F752FD1A
:107720002B680D931CE223681B4A2C00934200D166
:10773000EBE45B10DBB2012B00D03FE702220A9B97
:107740000399994200D8A3E1F8F73CFD0020019B82
:10775000DC6019B0F0BD206808F0D2FB62E57E78ED
:107760003B7836021E43019BEF1CDC60206808F06A
:10777000EDFB002801D1043C4DE66060C4E4012229
:107780000A9B06A95B6813400E32521813700A9BBD
:107790000C3B0A93B9E4C046D0DB02000380FFFF34
:1077A00000207F223B78C00119005BB2114008180D
:1077B0000137002BF6DB8300E41A04342100FFF7C5
:1077C00025FB2FE500207F223B78C00119005BB22A
:1077D000114008180137002BF6DB8300E41A04344B
:1077E00021001DF0DEFA1DE500237F213A78DB0140
:1077F000100052B20840C3180137002AF6DB9B0084
:107800005B4221681859FDF7BFFF1EE600207F226A
:107810003B78C00119005BB2114008180137002BFA
:10782000F6DB251D1CF01CFFDDE42500231F083DB1
:107830001A68216828681CF04BFF35E500237F217A
:107840003A78DB01100052B20840C3180137002A11
:10785000F6DB01339B00221F5B4212682168185936
:107860001CF036FF52E500207F223B78C001190052
:107870005BB2114008180137002BF6DB8300E41AD5
:107880000434210000F012FECCE400237F213A787A
:10789000DB01100052B20840C3180137002AF6DBA2
:1078A0009B005B42216818591DF0BCFBCDE500230D
:1078B0007F213A78DB01100052B20840C31801372B
:1078C000002AF6DB251F022B05D1DC4A2168286837
:1078D00006F0E6FBC2E42600083E2268296830680C
:1078E00006F0DEFB3060FAE500257F213B78ED01F4
:1078F0001A005BB20A4055190137002BF6DB220053
:107900002900206808F072FECD4B5D19AD006419A6
:10791000FFF7FBFB00257F213B78ED011A005BB2EE
:107920000A4055190137002BF6DB22002900206898
:1079300008F0B0FEFF222B0A13401540E5E70322B2
:10794000FB1C93430022186811001F1D251D1DF00C
:10795000B2FB48E40322FB1C9343251F22682968DD
:1079600018681F1D1DF0A7FB78E40322FB1C93433E
:1079700019795F1D8A00A41A0434220018681DF0CA
:10798000B5FB4FE40322FB1C934318798021C243CB
:10799000490092005F1DA4180143EEE700207F21FB
:1079A0003B78C0011A005BB20A4010180137002B67
:1079B000F6DBFF25FF220100C3096D0011402B40BB
:1079C0005B189B00E41A000A0240231D206808F09F
:1079D0009DF927E400217F223B78C90118005BB2A2
:1079E000104041180137002BF6DBFF22CB09520073
:1079F0001340CAB29B189B00E41A083C22000020E6
:107A000008F0C4FCFFF70EFC00237F203A78DB016E
:107A1000110052B20140CB180137002AF6DBFF21DA
:107A20001800FF250840DA096D002A40451C52194C
:107A30009200A41A1B0A194022001FF0FFF8FFF75A
:107A4000F1FB00217F223B78C90118005BB2104096
:107A500041180137002BF6DBFF22CB0952001340FF
:107A6000CAB29B189B00E41A0C3C22000120C7E715
:107A70000F2206ABD2181378002B00D15EE601214D
:107A80000A9B5B680B4013700A9B0C3B0A9355E6FC
:107A90000A9B5B6813420ED003220A9B21685B6835
:107AA00093431C0059609A600A9B08341F680A9B24
:107AB0000C3B0A93A0E50A9B0C3B0A933FE66B78CC
:107AC000022B03D1043C2068FFF718FB002BFAD1EE
:107AD0000A9B039A934203D25A495B48FFF760FB23
:107AE0009868002801D0FFF709FB0C3BF1E7079EDF
:107AF000231F0593002E1CD0079E00213200079102
:107B00000BAB201F006808F053FE012815D12F0091
:107B10000B9B2360F8F756FB019B06AA5F60DC60B5
:107B20000F239B181A780A9B01201343019A1361B3
:107B30000FE60BAB32002168E3E700282FD10B9B47
:107B4000043C002B00D13D4B2360002E4CD03F491C
:107B5000300020F09CFD002846D0F8F733FB0D964E
:107B60000D9B3B4918680FF051F9002800D1AEE099
:107B7000019B5A68002A00D1A9E01378432B00D05A
:107B800092E0937850781B02D11C0343019ACB18E2
:107B90005360D3680593043BD360FFF79BFA022838
:107BA0000FD12B490B9820F072FD002805D00B98BF
:107BB0000EF098F9043C2060C7E7F8F703FB0B9B35
:107BC000AFE5059C00207F223B78C00119005BB225
:107BD000114008180137002BF6DB251F2A682168A1
:107BE00008F070FEFFF73AFB059CFFF78EFA0021C4
:107BF0007F223B78C90118005BB210404118013761
:107C0000002BF6DB250001CD08F06EFEFFF7EBFA46
:107C10002068251F1FF02DF8FFF746FBAF2B05D876
:107C20000120803B5B000343FFF76DFABF2B11D8A7
:107C3000B022D31A9B00FFF7ACFAC046D0DB02009B
:107C4000FFFFFF3F4054030080300300A42D0300DA
:107C5000C8300300CF2B04D8C022D31A9B00FFF7F3
:107C60000CFBD62B06D8D03B1800216807F0E6FFA6
:107C7000FFF7D8FAFA2B08D8251FD73B180022683F
:107C8000296808F0C9F9FFF7E9FA4C494C4820F097
:107C9000F4FC0400F8F796FA049B019A06339B0063
:107CA000D3185C60022054E55E2B10D1019B019A31
:107CB000DC680D98231DD3600EF014F9019B606001
:107CC0005B68019A059301335360FFF703FA0D9B3C
:107CD0003C4A934231D03C4A93422ED0019B0BA8A0
:107CE0001B6805930B9320F0BDFB04000BA820F04C
:107CF000B9FB05000BA820F0B5FB019B01005B68F8
:107D00000593019B1B680693069A059B9E1A1F23E9
:107D100001229C46361B0B9C2378002B09D058B2BD
:107D200000282EDB6046013418405B090B94864224
:107D300031D22B000D980EF065F90F23012106AA10
:107D40009B181A78002A29D10A9A039991422DD8B2
:107D500001221A700A9B0D991B680593059A019BD5
:107D600005915A6003220A9B5B6893430A9A9160CB
:107D7000164A5A600D9A9A6012680C331A60019A7A
:107D80000AE70F20E0271840FF001B011F4063781F
:107D900002343B43CAE7361AD218BCE70A9A526843
:107DA0000A401A700A9A0C3A0A92CAE7049B019A8E
:107DB00006339B00D3180D9A5A6073E726540300CC
:107DC000CC2F0300F82B0300082C0300D0DB0200AB
:107DD00010B50400002906D0044B8A6B03600968C3
:107DE00000230EF00FF92000F8F7F1F90431030039
:107DF000F0B587B0039202934718002A02D0023AE6
:107E0000222A31D80400BC423CD22078F9F74CFA3F
:107E1000009000282ED123782B2B2DD10134391B33
:107E2000200003AA1EF02DFD23181C00002501933D
:107E3000BC422BD226783000F9F74EFA039B00287B
:107E400022D032002F3A9A421EDC303E039928009D
:107E5000FBF73EF9002842D1039B5D43AD196B004F
:107E60006B403CD40134E3E72249234820F005FC71
:107E7000F8F7ADF90134C6E72D2BD0D101342C3BF6
:107E80000093CCE70023FBE7102B10D0009B002BC6
:107E900015D101236D001D43019B9C4212D117494E
:107EA000039A15480EF03EF80299FFF791FF202340
:107EB0001E433300613B052BE8D8573EC6E76D42B1
:107EC000E7E70134BC4205D22078F9F7EDF9002844
:107ED000F7D1E4E7BC42E2D1280007B0F0BD019B36
:107EE000009A0593F91A05A8039B1DF08CF9059CCF
:107EF0000500D1E79654030000320300B954030093
:107F0000F0B504008BB0069209934718BC4255D2D5
:107F10002078F9F7C9F90190002837D123782B2B65
:107F200036D1019B01340493BC4200D3D6E0202318
:107F300022781A43692A32D1A21C974200D8EBE07A
:107F400062781A436E2A00D0E6E0A2781A43662AC5
:107F500000D0E1E0E21DE61C974214D9E2781A4312
:107F6000692A10D122791A436E2A0CD162791A43F8
:107F7000692A08D1A2791A43742A04D1E2791343F9
:107F8000792B00D10536FF25ED052BE00134BDE747
:107F9000019A04922D2BCAD101342C3BC3E76E2ADF
:107FA00010D008940026644B3500079300230196F7
:107FB0000293BC4220D3002306937BE00023089465
:107FC0000493EFE7A21C974200D8A5E062781A4319
:107FD000612A00D0A0E0A27813436E2B00D09BE072
:107FE000564DE61C049B002B02D080231B06ED1887
:107FF000B44279D1524989E0631C039323781A0073
:10800000303A0592092A2CD8022D04D10A235E4366
:10801000B618039CCDE7012D15D1059814F0DEFBB1
:10802000079914F097F8011C029813F011FD0290C3
:10803000079816F069F9434A434B15F059FB16F0BF
:10804000B5F90790E5E74149029814F083F8041C5C
:10805000059814F0C3FB211C13F0FAFC00250290D4
:10806000D7E7002D03D12E2B03D10125D1E7022D17
:1080700018D020221A43652A14D1039B9F4204D9A9
:1080800063782B2B06D1A31C0393039BBB42B1D077
:108090000225BEE702252D2BBBD1631903930123D3
:1080A0000193F2E7069A002A04D0202213436A2B98
:1080B00081D1039C019B002B00D07642300014F04C
:1080C0003DFB011C214816F0DDFF029914F042F837
:1080D000069B2600051C0193089C83E70023089457
:1080E0000026029367E70136BE4205D23078F9F7E1
:1080F000DBF80028F7D17DE7BE4200D07AE7099B84
:10810000002B02D1019B002B0DD01149114820F00A
:10811000B4FA1099FFF75CFE049B002B00D169E7CD
:108120002600002561E7032302209D430A4B2843D4
:10813000C0180BB0F0BDC046CDCCCC3D0000C07F18
:108140007C5403009A9999999999B93F000020416C
:108150005F54030000320300000080800023820788
:1081600008D10068044A0133904203D0034BC01A7F
:1081700043424341180070477CED020040ED02008D
:1081800070B506000D000124B44201D3044870BD4F
:10819000A300E95828681CF0B4FE0134F4E7C04697
:1081A000D0DB020010B5040010201EF05EF9044B75
:1081B00084600360034B43600023C36010BDC0466E
:1081C000C4060300E14F020070B5050010201EF048
:1081D0004CF90400074B696808C01EF049F8AB6809
:1081E000E968A3606B68E0689A0024F0BEFA20009A
:1081F00070BDC0467CED0200F7B505000E000024FE
:108200008B0705D10B68224C1C1B62426241D4B221
:10821000B368002B0AD1002C03D01E4928001EF0A1
:1082200058F91D4928001EF054F9F7BD002C03D061
:108230001A4928001EF04DF9194928001EF049F985
:10824000002701237268974207D3164928001EF0C1
:1082500040F9002CE9D01449E4E7BA000192F26831
:10826000B9005258002A01D0042A01D10137E9E7A8
:10827000002B03D10D4928001EF02BF9F368B9003B
:10828000595801222800FAF7DBF90023EEE7C0462F
:1082900040ED02002F550300365503003C55030006
:1082A000FF470300CB830300C14A03003C4803009F
:1082B00010B5FFF753FF002805D1034903480DF01F
:1082C00031FEF7F784FF10BD03550300883103002A
:1082D00070B50D000400FFF7EBFF280007F010FE5B
:1082E0000500280007F058FE011E01D1054870BDA9
:1082F000231D002218001DF0C5FF0028F1D0024800
:10830000F5E7C046442403003C24030010B583076E
:108310000CD10368084A93420DD0084A934205D114
:108320000749084820F0A9F9F7F751FF064907481F
:108330000DF0F8FDF8E710BD7CED020040ED020005
:10834000E15403009C2C0300035503008831030013
:1083500070B50D000400FFF7D9FF280007F0D0FD2D
:108360000500280007F018FE011E01D1034870BD6A
:10837000231D032218001DF085FFF2E7D0DB020069
:1083800070B50D000400FFF7C1FF2900201D012278
:108390001DF078FF004870BDD0DB020070B50D0005
:1083A0000400FFF7B3FF2900201D02221DF06AFF21
:1083B000004870BDD0DB020010B50400FFF7A6FF37
:1083C000201D1DF0EAFF014810BDC046D0DB0200B1
:1083D00010B501221CF0CFFD004810BDD0DB02001B
:1083E00070B504000D00FFF791FF201D0222290047
:1083F0001DF048FF002804D1034820F031F9F7F7B9
:10840000E6FE024870BDC046942E0300D0DB020099
:1084100010B50400FFF77AFF201D1DF09FFF002814
:1084200005D10349034820F028F9F7F7D0FE10BD25
:1084300019550300942E0300F8B50D0001280BD048
:10844000002803D002280BD0002004E08B681448D9
:10845000002B00D11348F8BD8B685B001843FAE786
:10846000032400200C408442F5D10F4B0E682000FD
:108470009E42F0D14F68A74203D1012076003043DD
:10848000E9E7EA68A3009958002906D0042904D036
:10849000022007F0D3FB401036180134EBE7C0464A
:1084A000442403003C24030040ED0200F7B507001C
:1084B000102001911DF0D9FF05000A4B060008C5E8
:1084C000390028001DF0D4FE0024BC4201D1300048
:1084D000FEBD0199A3000122C95828001DF0D2FE5B
:1084E0000134F2E77CED0200F7B505000E00171E1F
:1084F00006D0FFF70BFF1A4CB5420AD12000FEBD93
:10850000FFF7D6FEB54204D128001CF00CFD040094
:10851000F4E700210800FFF7C9FF0400300007F06E
:10852000EFFC0190019807F037FD061E0CD1002FDB
:10853000E4D0E8681DF0C0FF63686B60A368AB60BF
:10854000E368074CEB60D9E7281D002231001DF0DD
:1085500099FE0028E6D031002000FFF711FFE1E787
:10856000D0DB0200F0B585B0170004000390029143
:10857000FFF7F4FD0026021E06D103AB01211F48C0
:108580001CF056FD01260400029D2800FFF7E6FDC1
:108590000023021E06D102AB012118481CF048FD41
:1085A000012305000193002F15D0A368AA68934208
:1085B00011D10027002E02D02000FFF7FDFE019B05
:1085C000002B02D02800FFF7F7FE0D48002F00D146
:1085D0000C4805B0F0BD2000FFF7E4FD07003800AF
:1085E0001CF0FEFC011E01D10127E3E72B1D002238
:1085F00018001DF047FE0028F1D1DAE77CED0200FB
:10860000442403003C24030037B50C0015000091FE
:1086100001921F284ED812F0E7FE10151A4D4D4D4D
:108620001F4D4D4D4D4D4D10151A4D4D4D1F4D4D7E
:108630004D4D4D242A2D393E4D43110020001CF094
:108640007CFC3EBD110020001CF085FCF9E7110008
:1086500020001CF0E2FCF4E7694602201CF0BBFCA1
:10866000EFE7012229002000FFF77CFFE9E7012264
:108670002800F9E70800FFF71BFE2800FFF76EFD52
:10868000002815D0A368AA68934211D129002000C0
:108690001CF000FDD5E7110020001CF0F3FCD0E732
:1086A000081D002229001DF0EDFD031E0248C8D15F
:1086B0000248C6E70020C4E7442403003C2403002A
:1086C00030B507240278084DA24314000222224349
:1086D00002707F22039C41602240D40002888360A4
:1086E0002A402243028030BD07FCFFFF10B50B007B
:1086F000072401782340A14319437F230170049983
:108700000A4C0B40D9000388426023400B4303808E
:10871000039B04685905064BC90A23400B430360B9
:10872000029B8360059BC36010BDC04607FCFFFF32
:10873000FF03E0FF10B510201DF097FE0400034B6F
:1087400008C020F0AAFF200010BDC046A0F0020023
:1087500070B50C00052804D812F046FE06030E047E
:10876000151E0024200070BD081D21F0C7F80E4C16
:108770000028F7D00D4CF5E7081D21F0E5FB01249A
:1087800040000443EEE7FFF7D5FF211D050004304C
:1087900021F0E7F82C00E5E7FFF7CCFF211D0500ED
:1087A000043021F0EEF8F5E7442403003C240300F4
:1087B00070B5050083070CD1104B02689A4208D1AE
:1087C000FFF7B8FF0400291D043021F0BFF8200096
:1087D00070BD2800FAF704F8C0231B06984205D1A3
:1087E00080200021C0051CF0D9FCF1E7C2178318D6
:1087F000012053405B001843EAE7C046A0F00200A6
:1088000070B544006408051C211C201C13F05EFF99
:10881000002820D11149201C12F0DEFF002814D1BD
:10882000281C1CF074FE002808D0FFF783FF04000A
:10883000291C043020F0B0FF200005E0281C13F0B4
:108840005DFF01244000204370BD054905480DF03F
:1088500069FBF7F7BCFC04490448F8E7FFFF7F7F9A
:108860009A55030044300300B3550300003203005F
:1088700007B5C30701D540100EBD043001A90EF0A5
:1088800001FE002801D00198F6E7034903481FF0D4
:10889000F4FEF7F79CFCC0466D550300443003001E
:1088A0000123F0B58DB006000C0000920B402ED0D5
:1088B0004B10022202A903A820F02DFF03AD009B5C
:1088C000DB072ED5009B02225B1002A903A820F033
:1088D00022FF03AC092E01D0162E3ED1200021F03C
:1088E0000DF8002867D1280021F084FB051C20002A
:1088F00021F080FB011C281C13F03CFA032302002A
:1089000002209A438D4B1043C0180DB0F0BD0320D8
:10891000084000D007E18A4B0A689A42F5D10D1D44
:10892000CDE70323009A1A4208D10099844A0968C6
:108930000191914202D1009B1C1DCBE7009A13408C
:10894000022B04D17F4B1340062B00D0EDE0009AA0
:108950002100300000F090FED7E7182E00D9BAE0D1
:10896000FFF7E8FE0700300012F03EFD6E74687AF3
:108970007A0D131A20DD4D8E946E74687A7A0D1379
:108980001A20DD4D8E0022002900381D21F090F8BC
:1089900004E0381D2200290021F0C4F83800B4E7B3
:1089A000381D2200290021F00AFAF7E7200020F004
:1089B000A5FF002805D0644964481FF05EFEF7F764
:1089C00006FC06A83E1D20F068FE23002A0006A92A
:1089D00030000EF0EBFB2B7822785340DB070ED5EE
:1089E00006A820F08BFF002809D1012109A84942DF
:1089F00020F087FE09AA3100300021F059F806A8BE
:108A000020F057FECAE7200020F078FF0028D2D1DE
:108A100009A83E1D20F041FE23002A00310009A8CC
:108A20000EF0C4FB09A820F044FE2B7822785340B6
:108A3000DB07B3D5220031003000A7E7381D220044
:108A4000290021F0B7F8A9E7381D2200290021F0FC
:108A500033F9A3E7381D220029000EF033FB9DE710
:108A60000098FFF705FF021E02DA39493948A4E7EA
:108A7000381D2900032E01D0102E02D10EF0B6FAB7
:108A80008CE720F0B5FF89E7381D2200290021F08E
:108A900019FA83E7200020F031FF00288BD1FFF77F
:108AA00049FE3E1D009023002A00043031000EF0E4
:108AB0007DFB2B7822785340DB0704D52200310060
:108AC000300020F0F5FF009B09A9022009930A97C6
:108AD000FEF79CF919E72100280020F014FF193E49
:108AE00003000020042E00D90FE7300012F07CFCB8
:108AF0000309160D12001848002B00DB05E7174884
:108B000003E71548002BFADCFFE61348002B00DDD5
:108B1000FBE6F4E71048002BF1DAF6E60E48002BEE
:108B200000D0F2E6EBE70020EFE6280021F062FA41
:108B3000009A011C30000CF085FCE6E60000808005
:108B4000A0F00200070080FF4755030048320300F1
:108B500058550300003203003C2403004424030062
:108B6000F0B50700443787B0040038000E00002538
:108B700020F0C7FB2069431C1CD00A2804D1200028
:108B80001CF06CFB0125F5E7F8F78EFB002803D0FD
:108B900020001CF063FBEDE72369232B08D12000A4
:108BA0001CF05CFB23695A1CE4D00A2BF7D1E1E7E7
:108BB0005C2B0ED0E369226AA363E263002E17D117
:108BC000636A002B1DDA2200072140321170013345
:108BD0001EE020001CF042FB23690A2BD8D0E36979
:108BE000A363236AE36304234034237007B0F0BD1A
:108BF000012BE5D1012AE3D00622230040331A706D
:108C000007E0002B1FD02200062140321170013BEB
:108C10006362200040300378082BE7D10023E56C25
:108C2000B24EA46C9A00915900228F18944200D140
:108C300070E28F5CBC46AF5CBC4500D168E201339A
:108C4000222BEFD1D2E7002D34D0A36A002B31D1F3
:108C50002100052040310870551E6362226BA44B31
:108C6000606BD3185B001B5A9D42BFD017D9E16AD5
:108C70008A4207D3083149001DF00DFCE36A6063A6
:108C80000833E362236B5A1C2263626B5B009D52C4
:108C9000636A9CE7013B2363636A013B6362236B66
:108CA000934A9A185200125A9542F3D39ED0022347
:108CB0000B70AEE72069431C1AD18D4A236B616BA0
:108CC0009B185B005A5A23004033002A97D0052294
:108CD0001A7000236362864A236B9A185200525A14
:108CE000002A00D182E7013B2363636A013BF1E77D
:108CF00027281FD022281DD0752804D01023020059
:108D00009A43622A04D16369272B0ED0222B0CD000
:108D1000722800D015E26369622B00D017E2A369C4
:108D2000272B02D0222B00D011E2752804D120007D
:108D30001CF094FA00234DE0622842D120001CF080
:108D40008DFA002302932369722B04D120001CF0BA
:108D500085FA0123029323000C2240331A70012369
:108D6000059323690393222B01D02723039320002B
:108D70001CF074FA0123039A0493236993420BD1E4
:108D800013006269934207D120001CF067FA2000AB
:108D90001CF064FA03230493002623690193013332
:108DA00000D1C9E0049B012B03D1019B0A2B00D108
:108DB000C2E0049BB34214D83100380020F03FFBDE
:108DC00027E77228B6D120001CF048FA2369622BED
:108DD000BCD00123029323000B2240331A700023DE
:108DE000BEE7019B039A934208D111003800013677
:108DF0000EF09EF820001CF031FACEE7019B5C2BB0
:108E000000D096E020001CF029FA029B2569002B77
:108E100004D05C2138000EF08BF85AE0622D00D1AE
:108E2000BEE130D84E2D78D01BD8222D53D0272D1F
:108E300051D000260A2DDDD0280030380728E8D888
:108E4000050003266369303B072B42D8013E002E04
:108E50003FD020001CF002FA2369ED00303B5D1981
:108E6000F0E75C2D37D0612D5AD0552DE4D1059B0C
:108E7000002B27D05C2138000EF05AF8E9B23800F8
:108E800020F094FA13E0742D13D008D86E2D00D181
:108E900088E1722D14D0662DCED10C250AE0762DF6
:108EA0000CD0E4D30226782D10D06B1CC4D1002640
:108EB000A0E70925059B002BE0D112E00B25F9E77F
:108EC0000D25F7E70826752D00D1043E0025013E4B
:108ED00012D26B1CEBD0074B9D4225D8059B002B73
:108EE00020D1290038000EF023F8E0E724EF02003B
:108EF000FFFFFF7FFFFF100020001CF0AFF9236988
:108F000018000193F8F7F4F9002800D113E1019853
:108F10001BF02CFB2D012D18D9E7A54807F09CFD6F
:108F20000725DBE7FF2DA9D92300012240331A7062
:108F3000BDE76B461979A2E7049BB34200D83BE733
:108F40002300032240331A7036E7F8F7C5F90028EA
:108F500007D02600216940362E291CD10A23337000
:108F600029E023692E2B04D16069F8F7B5F90028B0
:108F7000EFD121692E2954D0002602228D4D2F7861
:108F8000002F01D0B9426CD120001CF067F9002FEE
:108F900076D1012231E60923337030290BD1626981
:108FA00017331343623B162B03D8834DDD40012357
:108FB0001D4001231D4038000DF0BAFF20001CF0B9
:108FC0004DF914E0002D16D1652801D0452812D1A5
:108FD0000A236521337038000DF0AAFF20001CF031
:108FE0003DF9216902220B002B3B9343E3D020691A
:108FF000431CE7D10DE6F8F763F9002808D0216992
:109000002E29ABD00B00202293434A2BD3D1A5E7C6
:109010002069F8F761F90028F1D123692E2BEED0F1
:10902000F7E5260038000DF083FF20001CF016F94C
:10903000236940362E2B00D0B6E065692E2D00D076
:10904000B2E0290038000DF073FF290038000DF060
:109050006FFF20001CF002F920001CF0FFF80D2328
:10906000A3E03B00633B9343DBB2681C002B03D1BE
:1090700005000136013582E7452FFAD1013EF7E7B9
:10908000330001352A78652A09D16A7821690136C9
:10909000914212D120001CF0E1F8330001352A780A
:1090A000452A20D16B7822699A420AD120001CF00F
:1090B000D5F83300414AD25C04E01F0002353B0082
:1090C000E0E70122230040331A70230040331B786D
:1090D000042219009143422901D0442B10D1A36AE4
:1090E0000133A36295E5632AE4D16A782169771C8C
:1090F0009142DFD120001CF0B1F802353E00DEE7DE
:10910000432902D0452B00D083E5A36A013BE8E761
:1091100001328AE53A78002A00D090E5212B08D167
:10912000274BA8331A680E23002A00D1023303709C
:109130005CE50E33FBE72300012240331A70050083
:10914000B8E6622803D16369722B00D1E7E5F8F72E
:10915000B7F8051E206904D15F2802D07F2800D807
:10916000F3E62300082240331A70C1B2380020F021
:109170001DF920001CF072F82069431C00D148E55D
:10918000F8F79EF8002809D120695F2806D07F28CB
:1091900004D8F8F7A1F8002800D13AE5217CE5E7EA
:1091A000082587E60A2585E64A23337031E5C0465F
:1091B0000E560300CC550300012040008D560300DD
:1091C000380A0020F0B5050089B002AFB96016007A
:1091D0003B6005F0A3F8AB687B611423F8181FF01F
:1091E00041F914237860F8181FF03CF90323584321
:1091F0007B68C0188300FB602C2B29D86B46F8686D
:109200002A30C008C0001B1A9D46002302ACFB6038
:10921000AA687B6929009B1A63607B682000A361B0
:109220003B680093BA6833000BF0E0F91A4E002156
:109230007368200063616B687360FDF733FF6369D7
:10924000B860736000280AD0022819D0134D08E0D6
:10925000F8681C301DF016F9041ED9D1CEE7E3687A
:109260001D68FB68002B07D00023BB6020001DF0A9
:1092700023F9BB68002B0BD12800BD4607B0F0BD19
:109280007B6805339B00E3185D68FB68002BEDD11C
:109290002800F6F79CFFC046380A0020D0DB020009
:1092A0000122030030B5134085B004004510002BA7
:1092B00014D128491D00884210D0274988420DD07A
:1092C000264B1500984209D00323034009D1244AB4
:1092D0000168914205D11BF0ADFF0500280005B0E3
:1092E00030BD204A25002240062A05D0002B08D197
:1092F0001D4B22689A4204D101A92000FAF7B8FC5C
:10930000EBE72000F9F784F9184B984207D1FF23C7
:10931000DB05E0180323984313F0F0F9DDE7144B65
:10932000984206D101AA694620001BF0AAFD019DC2
:10933000D4E7104B984205D101AA694620001BF0E2
:1093400047FDF4E7022201A920001BF050FA002893
:10935000C4D0ECE7D0DB02003C240300442403002B
:10936000A0F00200070080FF84320300442B0300BA
:1093700090EC0200C0E90200F7B506000F00009271
:109380000193041E00D044683800431E9841201801
:10939000043080001DF069F80C4B050003600C4B95
:1093A0005B684360009B8360019BC360002E05D017
:1093B0003100A2000831103023F0D7F9002F02D07D
:1093C0000434A40067512800FEBDC046E8EF020047
:1093D000380A002070B5060010200D0014001DF0A2
:1093E00044F8034B466085600360C46070BDC046AE
:1093F000ACEF02007FB54B680E005C1021006846A0
:109400001FF060FF029D00212200280023F0C8F910
:1094100001213068014009D12B0022001BF0A4FE7D
:1094200069460748F9F740FF04B070BD43102000BB
:10943000042C00D904202A0000211CF003F9EFE7D6
:1094400008E00200F0B50C00002585B011002000F6
:109450001E00009502232A0005F078FB0120AC4293
:109460002BD0844231D13068204226D103230340DF
:10947000AB4203D11C4A016891421ED01B4A0240F4
:10948000062A06D0002B0DD10268194B92699A4228
:1094900008D103A9FAF7ECFB00231A000399FEF7A1
:1094A000A7FC0AE0032302001A40022A07D1FF2288
:1094B000D20580189843FFF7A3F905B0F0BDF9F77E
:1094C0008FF9012340001843F7E703A93068FAF742
:1094D000CFFB04007068039FF9F782F92B000200AC
:1094E00039002000DBE7C046A0F00200070080FF43
:1094F00029420000F0B58DB00A9214AA1278050036
:109500000B9215AA12780E000792DA0700D494E0A5
:109510001800F9F765F9002305900693002803DA8F
:10952000434205932D230693129B0027023B1E2BDB
:1095300016D84F4B129A2020995C11F073FF079BAD
:10954000C4B2BB4204D0601C032111F06BFF0700C2
:109550001398002801D023F089FA0334E7193F1843
:109560003368BB4204D238001CF07FFF28603760AC
:1095700000222C68E619731E1A70059A002A2CD056
:10958000099308930B9B0A3B0B930598129912F0D1
:10959000B9F80E000598129911F0CEFF330005902E
:1095A0003033092E01DD0B9B9B19089A561E337030
:1095B000079B002B30D0059B002B11D0B4420FD25B
:1095C000099B9B1B032B06D16B461B7F013E33700F
:1095D000B44205D209960896D7E73023023E33708D
:1095E000139B002B06D0180023F040FA0023301AFA
:1095F000844219D3069B002B05D0B44203D26B469C
:109600001B7E013E33702B68DF19BF1B0A9B013F95
:109610001F6030000DB0F0BDB442E1D2059B002BBD
:10962000D9D1DDE7C2540133139AD25C002AF9D1B3
:10963000069B0600002BE2D1E5E79A0711D10D4AFF
:10964000196891420DD1079A310003920B9A029248
:10965000139A0192129A00920A9A1BF05CFD06007E
:10966000D7E700232A6813700A9A2E681360D0E7A0
:10967000B8560300A0F002001300144A10B504000D
:10968000934204D10122200006F0C6FC10BD104A0E
:10969000934201D10322F6E70020072CF6D10D4AB0
:1096A0001A40062A0ED09A07F0D11A680A4CA24234
:1096B00008D00A4CA24205D0094CA24202D0094C63
:1096C000A242E3D10A0007201900DDE73C24030091
:1096D00044240300070080FF8432030008E00200F6
:1096E00090EC0200C0E90200074BDB68002B01D1BF
:1096F000180006E05A68824204D8801A04308000BC
:10970000C05870471B68F1E7380A002070B5114D4A
:109710000400EB689868DB6883420FD30230C00016
:109720001CF0A3FEEB685A68D96803609B68521866
:109730005B00836000234260C360E860EA68D3682E
:109740005068591C04339B000138D16040189C506C
:1097500070BDC046380A0020074B4118884204D328
:10976000D8B2002800D1013070475A01D3180278CE
:1097700001305340F2E7C04605150000034B044A90
:10978000DA60002294331A607047C046380A00201D
:10979000DCF00200F0B585B001900E00FFF7DCFFB1
:1097A000144B0290DC68002C01D120001EE0270041
:1097B00010373D00E3689B00FB180393039B9D4219
:1097C00001D32468EFE72868029A03789A420FD100
:1097D00043789E420CD102303200019922F0B6FF4C
:1097E000002805D1ED1B6068AD10281805B0F0BD4C
:1097F0000435E3E7380A0020F0B585B00290019106
:10980000FFF7C8FF002858D12F4C019B2700943741
:10981000DD1C3B68002B17D026002C4A98361268B6
:1098200031680392AA188A420ED9020069181800FA
:109830001CF03EFE0390002841D1244B3868196883
:109840001CF029FE039B3B60230094331B68002B14
:1098500017D12E00802D00D28026300027001CF06A
:1098600011FE94373860002804D128001CF0FDFD5B
:109870002E003860230098331E60230000229C33A2
:109880001A6023009C331A6894342468AD18019937
:109890000298A4181D60FFF75FFF6B461B792070CC
:1098A0006370019AA01C029922F05FFF0022019BC5
:1098B0002000E3189A70FFF729FF05B0F0BD336868
:1098C0005B193360C0E7C046380A0020D40A002084
:1098D0003E2803D040280CD03C2811D14239C9B2CF
:1098E0002F290DD8084B585C0123002A00D01360A3
:1098F0007047712904D8054B585C054B5B56F4E75B
:1099000001230020F1E7C0468E730300BE730300FD
:109910003074030010B551283DD011D849282ED0FD
:1099200007D8422803D0482826D0002806D18B5CCF
:1099300010E04F284BD017D84C2820D0002309E046
:10994000682816D00AD8642836D066282AD062281B
:10995000F4D18B5601205B00184314E06C2803D02F
:10996000712811D06928E9D1920050581BF025FCCC
:1099700009E05200535EEDE75200535AEAE79200C5
:1099800050581BF035FC10BDD2008A181068516881
:109990001BF004FCF7E7D2008A18106851681BF02E
:1099A00018FCF0E70323920050589843030002206C
:1099B0001843084BC018E6E7D2008A1810685168AF
:1099C00014F0F4FC032302009A431300EFE7920023
:1099D0005058D8E700008080F7B51700156801AA35
:1099E00004000E00FFF774FF402C05D1019B043CDE
:1099F0005A1EAA185D4215405A213E3C62426241FD
:109A0000B14289412B183B60D2B22B0049421BF076
:109A1000F0FD04000D004F2E08D0532E07D123F087
:109A200025F8002201002000F9F774FCFEBD662E27
:109A300006D1032302249843154B2043C018F5E7B1
:109A4000642E06D114F0B2FC0323040002209C43D0
:109A5000F2E75A2E0FD980220023D20512196B414A
:109A6000002B04D1002A02DB1BF0A7FBDEE7290054
:109A70001BF094FBDAE7002905D1064B984202D887
:109A80001BF0B6FBD2E729001BF0A3FBCEE7C046D4
:109A900000008080FFFFFF3FF0B587B0140003AAED
:109AA00007000E0001931D68FFF712FF0090402F82
:109AB00005D1039B043F5A1EAA185D421540009B26
:109AC000019AEB1813603E3F642E14D0662E0DD021
:109AD0004F2E2ED179424F410098F9B2042800D977
:109AE000042023002A001BF0ADFD30E02000F8F731
:109AF000DBFE0400EEE72000F8F7D6FE14F004FCCD
:109B00000490059139004B425941C9B28B0006AA15
:109B1000D318083B2A001B6804201BF093FD3B0070
:109B20005A1E934106AA9B00D318083B04351C68B3
:109B3000D0E7A3070DD10F4B22689A4209D1794291
:109B40004F412B00F9B2009A20001BF00DFB07B02B
:109B5000F0BD2000F8F744FE009B0400042BB9D9A7
:109B60005A2EB7D90028B5DA1A1F281DFF2122F076
:109B700017FEAFE7A0F0020070B505000E0014005C
:109B80001800642D0CD0662D04D04F2D11D19400F7
:109B9000A35104E094000E19F8F786FE306070BD02
:109BA000D4000E19F8F780FE14F0AEFB306071603F
:109BB000F5E720232B43712B0CD10321014009D160
:109BC000094B02689A4205D1E300F31808221BF002
:109BD000CBFAE4E7F8F704FE220003003100280086
:109BE0001BF043FDDBE7C046A0F0020005230200A6
:109BF00070B5094C094D2068434309489B189B00E8
:109C000018582B682260C0180F23194009012860DA
:109C1000FDF75CF870BDC04638030020C403002087
:109C2000D4FC0200A839030000B5080006292ED88C
:109C300011F0DAFB040A10161B2128009A18E223FF
:109C4000DB00D218107800BDC4329200D05C8006D0
:109C5000800EF8E7C4329200D05AC004400EF2E7FA
:109C6000C4329200D0580003F8E7C43292009A1828
:109C700090780009E7E7C43292009A18D07800077C
:109C8000000FE0E7C43292009A18D078F1E7024A58
:109C9000024B00201A60D6E7A27403007000002077
:109CA000A83910B504000800062949D811F09CFB1A
:109CB000040A141F2A343F00E221A218C9005218D6
:109CC000137010BD3F210B401800C4329200135D89
:109CD0008B4303431355F4E77F21C43292001940AC
:109CE0001948135B890103400B431353E9E77F21B4
:109CF000C432920019401059144B490303400B43DE
:109D00001351DEE70F20C4329200A2181901937894
:109D100003400B439370D4E70F210B401800C4326B
:109D20009200A218D3788B430343D370C9E70F2066
:109D3000C4329200A218D1781B0101400B43F4E712
:109D4000034A044B1A60BCE73FE0FFFFFF1FF0FF30
:109D5000C074030070000020F0B5D2B287B00F00CD
:109D60000593072113000B40013BDBB2042B02D902
:109D70002C4D2D4C25608A4319020291002A29D1CD
:109D80002A4BC55C2D09ED43EBB23D7801932C00C5
:109D90005B1BDBB204930826254B029A1B199B5CC4
:109DA0005A00D2B25BB20392002B38DA1A21032098
:109DB000013EF6B2FFF71AFF039B002EF0D10134EB
:109DC000049BE4B2E318DBB2002BE4D1019BED1A53
:109DD0003D701AE0D4431749E4B2CF5C0825144B18
:109DE000029A1B199B5C5E005BB2F6B2002B0FDA85
:109DF00005210220FFF7FAFE013DEDB23300002DF0
:109E0000F1D10134E4B2002CE8D1059807B0F0BDDF
:109E100039000120FFF7EAFE002FE9D0ECE7062128
:109E20000420C5E7AD74030070000020190700008E
:109E3000387A0300938003000022F0B505000F007C
:109E4000FF200F248BB008AB654EDA710100C431DE
:109E5000890069188B781A09B25C234012011343F8
:109E6000CA788B7013071B0FF35CA2432340134384
:109E70001A09B25C234012011343CB700138E5D2BA
:109E8000E223DB00EE5CB308F31ADBB20593554B1B
:109E90001B68002B0BD0E222C4218120D200890054
:109EA00000013B00AA1869182818F8F72DFA0024B9
:109EB0004823029403930194009481222B191201E8
:109EC0009B181B78180004930723984320D008A9F7
:109ED0002300049A07312800FFF73EFF0230C4B286
:109EE000023FFFB2002F78D02B780393013EF6B2E9
:109EF000002E47D1E2222B19D2009B181E78B308FE
:109F0000F31ADBB205930023029301930093D4E785
:109F1000354B009A9C469A5C2300C4339B00EB1897
:109F2000997809090A4331498A5C01990692624687
:109F3000DB78525C1907090F0A432C491B098A5C1C
:109F40002B490792029A8A5C07991343069A521882
:109F50002649C95C01238918FF2A00DC031CC918A3
:109F6000882309061B06C918090F0020FFF73EFECB
:109F7000039B013BDBB20393002BB7D10134E4B266
:109F8000013FAEE7059B013BDBB20593002B02D1FD
:109F9000049B002B18D12200C4329200535D00991B
:109FA0009B069B0ECB18DBB20093535B0199DB043D
:109FB0005B0ECB18DBB201935359029A1B035B0E65
:109FC000D318DBB2029378E708A92300049A07317B
:109FD0002800FFF7C1FE04008CE70BB0F0BDC046BF
:109FE000BC750300A4030020887F0300947703005E
:109FF00038790300064B1B5C002B05D0054B185C21
:10A000004843C011C0B27047034B185CFBE7C04621
:10A01000E47803005D7703001D760300064B1B5CAC
:10A02000002B05D0054B185C4843C011C0B27047E7
:10A03000034B185CFBE7C046E478030098800300FC
:10A040006D760300F0B5037A8DB004007F2B00D14C
:10A0500045E10300070000250933FF330837099362
:10A0600001953E787F2E00D086E000230693019371
:10A0700006998B00E31803931A7A481C1B7BC0B225
:10A0800006907F2B00D11DE19F49CE5C8D5C9F49DE
:10A09000AE4200D0F3E08D5CCB5C0493039B597A15
:10A0A000019B5918CBB20193049BEB18DBB20793C9
:10A0B000023B1B06DCD4A826019B5D1BEBB205937B
:10A0C000A82E00D0E3E0039BA8215F7A5A7B7F088B
:10A0D0005208BB180293019B20009A18D2B2DF1BD2
:10A0E000FFF7A0FDFFB205003A00A8212000FFF70E
:10A0F00099FD2D1AEDB27F222B006DB29343089388
:10A10000EB17E8185840029911F0FCFA2800CBB27E
:10A110000299099311F010FA0025C3B20A93059F22
:10A12000029BDB19DBB20B933A0031002000FFF7F2
:10A1300079FD0A9B01370B9A1818FFB2C3B29742F8
:10A1400000D1B9E0099AAD18029AEDB2AA420DD831
:10A15000AD1A20216A4652181278EDB252B2002A86
:10A1600000DAA7E0002B01D00133DBB23A00310066
:10A170002000FFF795FDD7E7012E7AD12B003100A3
:10A18000019A20001BF0B5FABA78614BA1789B18B0
:10A190005B7830000193FB780293FFF72BFF3F239E
:10A1A000E178034030000393FFF738FF7F22594BDB
:10A1B0009B5D1A40584B04929A5D0F231A400592FA
:10A1C000564A925D1A400692554A925D1A4007928D
:10A1D0003F22544B9B5D08937B78EB18DBB20A93CC
:10A1E000039B134003937F23184083019C462A005E
:10A1F0003F21C4329200135D0F268B4303990B431A
:10A200001355135B48490B4061460B431353049BA2
:10A2100010595903454B03400B430598190C314025
:10A22000000113510843A21890701B0E0698B34307
:10A230000799034309011E400E4320206946D6704A
:10A24000812209186319097812019A181170E22203
:10A25000D2009B180299019A013552181A700A9B74
:10A26000EDB29D42C3D1099B0437BB4200D0F8E652
:10A27000FBE6022E88D12B00019AFF2181E72C48B2
:10A28000AE4201D9C55C07E78D5C835C05E7049BA2
:10A29000019A31009A18D2B22000FFF7C3FC059A48
:10A2A000050031002000FFF7BDFC079B2D1AEDB221
:10A2B000029320E7013B58E70136F6B2AF2E00D0FB
:10A2C000FEE6D5E6023189006118019B49785918EC
:10A2D0006368C9B2002B04D02000FFF7ADFD0DB0BC
:10A2E000F0BDE2228025D200A0186D001A00C43211
:10A2F0009200125D06789206D20EB21A01330270F5
:10A300000130AB42F2D1E7E7CD750300947803004A
:10A3100088800300BD760300CC7403001C75030025
:10A320006C750300387F03003FE0FFFFFF1FF0FF65
:10A330000D77030070B50C0005000B6805495A68DD
:10A340001CF092F9216828004031220003F000FD42
:10A3500070BDC046749F0300136870B5002B12D106
:10A360000568EE6BB34200D170BD9C002C19246CC3
:10A37000A14201D00133F5E7591CF5D002339B000F
:10A380001B581360F0E7034903481EF076F9F5F710
:10A390001EFFC046CF8003009C2C0300F0B585B0A3
:10A3A0000C000325F8F7D8FF25400700002D03D146
:10A3B0001E4B22689A4205D01D491E481EF05DF9C9
:10A3C000F5F705FF03AA02A920001AF001FD029E7D
:10A3D000039B30001030800001931CF046F804000D
:10A3E0003C22290022F0DCF9134B67602360134BF9
:10A3F000E663A360124BE360124B6361124BA361EF
:10A40000124BE361124B2362124B6362124B636384
:10A41000AE4202D1200005B0F0BD019BAF00D8597B
:10A42000F8F79AFFE71938640135F1E7C0E902004F
:10A430006C810300883103005035030035A3000010
:10A440005DA400008D6D00004D6E000059A300005A
:10A45000416F0000E96D000044FD0200F0B51D00F1
:10A4600085B0C36B00AFFB607A608B18FA6806009A
:10A470000C009A4205D02B492B480BF053FDF5F701
:10A48000A6FEFB688B424AD09A00130069460E3341
:10A49000DB08DB00CB1A9D4618000021BB6022F0D0
:10A4A0007FF90023A200934210D1F9687A688C46A4
:10A4B00062447A60ED187B689C420CD3B968F868F6
:10A4C000FCF7A4FCBD46066005B0F0BDE858B968CD
:10A4D000C8500433E7E72868F8F73EFF0021020080
:10A4E000F36B3B603B68994204D110490E480BF076
:10A4F00019FDC4E78B00F018006C824201D00131D5
:10A50000F0E70131F1D0B968CB181968002901D002
:10A510000749EBE76A6802341A600835CBE7BD608B
:10A52000CCE7C046E3800300883103001C810300B0
:10A530003D810300F7B5244900250B000833DA6F8D
:10A54000224B94461B785488981C80001618805A19
:10A55000883144430968A4120195F078002823D07B
:10A56000B07801268640A1273000A026FF00F6051E
:10A570000133F051DBB2981C80001618805A070096
:10A58000508878438012001BE7D0104A1370019B5B
:10A59000002B02D00C4B88331960002D03D062468B
:10A5A000094B0833DA67FEBDA024094B5668E40561
:10A5B000E650002902D10B000C00DCE701258C4697
:10A5C0000A0001950100F6E7380A0020380900204A
:10A5D0000C050000044B05491A000832D16700221F
:10A5E00088331A607047C046380A002050FD0200C8
:10A5F00010B578220249022002F072FC10BDC0465C
:10A6000035A50000421E104BFF3A70B59A4218D88B
:10A61000061172B60D4C00212300220088331D68FC
:10A620000832196062B68D4200D1D56F29782800B2
:10A630001BF083F86B6888344360468020600020FC
:10A6400070BD01204042FBE740410F00380A002066
:10A65000054B1A0088331B680832002B00D1D36FDA
:10A66000588800017047C046380A0020F7B5414AB3
:10A6700007000B00914200D913008022D200D21AA9
:10A68000019272B63C4A00201100883214680831E9
:10A69000106062B6844200D1CC6F0126BE40626871
:10A6A000324207D13A00A0210320C132FF3292008A
:10A6B000C9055050002521788D421CDB002B19D094
:10A6C000013120001BF039F86A46636892881E4306
:10A6D000466023789B00C3181A8101229F72DA72A8
:10A6E00001216388021D4380037899421CDB224BC1
:10A6F00088331860F7BDAA00A218927A97422CD02E
:10A700000135D9E7013920001BF017F86368B3431E
:10A71000436023785A1EAA42E2DD01339B000235D2
:10A720001B59AD002B50DBE71700D37A1489967ABA
:10A7300001934B1EBD88A54204D97D68043FFD608E
:10A74000013BF7D203339B00C3181C806C4624796D
:10A750009E70DC7001310432C6E7002BD2D020009D
:10A760001AF0EBFF6368023543606B469B88AD00CF
:10A770002B52B5E7FF030000380A002010B5002176
:10A780000400FFF773FF0D4B0833DA6F00231078D6
:10A79000834200DB10BD99005118897A8C4201D0A8
:10A7A0000133F5E702339B00D3181F229A7001236F
:10A7B000A021A340024AC9058B50EBE7380A0020CC
:10A7C0000C050000F7B54F4B4F4E504F3360002340
:10A7D0003B707B70BB70FB703B71A0238500DB0579
:10A7E000E022ED180323D200AB50023B8340A024AB
:10A7F0000093009A464BE405E250122010F0BAFC98
:10A80000A123009ADB00E25028200138C046C04650
:10A81000C046C046C046C046C046C046C046C04608
:10A82000C046C046F1D1E0220C23A221D200AB5099
:10A83000384BC90062580098024202D1013B002BFC
:10A84000F8D1A222A024D2001100324BE405A05876
:10A85000009D284202D0013B002BF8D1A12000220C
:10A860003368C0001A500920585080210224F83063
:10A87000C902FF30195028481A5028481C50C120DE
:10A88000A2248000E4001950A44610000721244CA3
:10A89000A0256646ED05AD59009E354201D1013C2B
:10A8A000F6D2002A01D101251D600125DD601D00C1
:10A8B0000026FC350195AE64A0266546F60576595E
:10A8C000009D2E4216D1019CA46C012C03D18C401A
:10A8D0003D5C2C433C54002911D10130C0B20731FA
:10A8E0000132282AD3D1FA20273A5A60800010F08A
:10A8F00041FCF7BD661E002CE5D03400DCE70139D1
:10A90000C9B2EDE7009000401C0000209B0B002026
:10A910000C0500001127000004050000440500009C
:10A9200010270000254B13B51A780400244B002A89
:10A930001CD0244A24491278002A12D1234A20002C
:10A940001A60F7F74DFF012812D02000F7F748FFF3
:10A95000022830D02000F7F743FF1D4C102808D004
:10A960001C491D481DF089FEF5F731FC1B4AE6E73E
:10A970001B4C200009F0B6FA1A4988420AD0200080
:10A9800009F0F2FAA02204216379D205C133FF3322
:10A990009B0099506079FFF715FF134CA0781AF0CF
:10A9A0000CFC009020781AF008FC69460190022007
:10A9B000FCF72CFA16BD0D4CDBE7C046990B0020C6
:10A9C0001C0000209A0B00207A81030000A00040A8
:10A9D00004E60200B68103008831030000900040C5
:10A9E00014E60200E42803009B0B002024E602008A
:10A9F00070B5137804000A3BD8B20F2809D90A00B1
:10AA0000104811490BF08EFA0025A3681860280041
:10AA100070BD002552781B021A43E3689D420AD19B
:10AA200023880025042BF2D1084906480BF07AFA56
:10AA3000A3681860EBE72069A90009589142E6D0A5
:10AA40000135EBE704310300558303006A830300FB
:10AA5000F0B585B004000D00100003A91E0019F028
:10AA6000BDFC002809D12A000B490C480BF05AFA0A
:10AA7000A3681860002005B0F0BD0398F7F7DCFE6E
:10AA80000300B343F7D0030000962A0004490348AB
:10AA90000BF048FAECE7C0461183030004310300D1
:10AAA00029830300F7B51E0013780D000A3BD9B2C5
:10AAB00004001B480F2904D850781B0218431AF0D1
:10AAC0008BFD03780193174B5A1C002317780199CB
:10AAD0008F421BD141785778B94217D18178977846
:10AAE0008F4213D1002F0ED10E4A9B00D05CB04292
:10AAF00008D933002A000C490C480BF013FAA3685C
:10AB000018600020FEBDC778002FEDD0013304325D
:10AB1000152BDBD12A00064904480BF003FAEEE7B7
:10AB2000C8CB0300CD8303008183030004310300FD
:10AB30009A830300F0B5137887B005000E000193E7
:10AB4000992B47D103A9100019F06CFC039B984284
:10AB500040D003781A000A3A0F2A0AD802000F23BD
:10AB600031002800FFF79EFF01248440200007B039
:10AB7000F0BDAE2B2ED119F050FC040019F048FCAA
:10AB800004900378B22B25D10127A33B220031008A
:10AB90002800FFF787FF3C0005A98440049819F0BE
:10ABA00041FC059B04909842E0D0019904A819F05B
:10ABB00048FC049A059B9A42D8D00F233100280004
:10ABC000FFF770FF3B00834004981C4319F020FC02
:10ABD0000490EEE73200044904480BF0A3F9AB6897
:10ABE00000241860C2E7C046B283030004310300AA
:10ABF000F0B50E0087B0040004A930001F000192D8
:10AC00001AF0EFFC019B0500002B0CD1322E05D170
:10AC1000BF21090260691DF03EF916E0482E00D000
:10AC200078E0B549F6E7019B012B00D089E0412E81
:10AC30000DD101003A682000FFF7DAFE01006069DB
:10AC40001DF07FF9002800D1C7E107B0F0BD422E0A
:10AC500009D101003A682000FFF7CAFE01006069CF
:10AC60001DF0C7F9EEE7432E0AD101000F233A6821
:10AC70002000FFF717FF8E21C000C9010143C9E77B
:10AC80000378622B32D1049B032B07D0052B2DD1E7
:10AC9000C3785F2B2AD103796E2B27D1012600239D
:10ACA00068787642954AD1184A78824205D1AA78C6
:10ACB00089788A4201D1914A9E5C03332A2BF1D1D3
:10ACC000731C27D03A6829002000FFF791FE0499F1
:10ACD000020000236069052904D12B79773B5D428E
:10ACE0005D41EBB231001DF048F9ABE7462E01D1D2
:10ACF00083498FE7472E01D182498BE7442E12D139
:10AD000029003A682000FFF715FFFF231B02B4213A
:10AD1000184214D0019B2A007B497C480BF002F9B1
:10AD2000A368186091E7452EF4D13A682900200005
:10AD3000FFF700FFFF231B021842EBD1BC210902E1
:10AD40009CE7019B022B00D0E8E07B681B780A3B64
:10AD50000F2B48D8332E12D13A6801000F23200060
:10AD6000FFF7A0FE7A68060029000F232000FFF7F6
:10AD700099FE3100020060691DF0CCF865E7002300
:10AD80000293342E1AD18026F6013A68290007234F
:10AD90002000FFF787FE7A68019029000723200032
:10ADA000FFF780FE019A0300310060691DF0ABF8E7
:10ADB0004BE7029B013302930F2BABD0029B032284
:10ADC0009E00534B711C5918280021F056FE002894
:10ADD000EFD1EB78002BECD14D4BF65C80233601A4
:10ADE000DB011E43D1E7332E19D1802607233A68B1
:10ADF00029002000FFF756FEFF23019029007A6802
:10AE00002000FFF725FE019BB601190206433143DE
:10AE100000E7A026EAE7C026E8E7E026E6E7352EC9
:10AE2000F7D0362EF7D0372EF7D00023394A9900C5
:10AE30005018408886425BD18B5A200002933A68B2
:10AE400007232900FFF72EFE7E6803903378982BA6
:10AE500031D1300019F021FB00282CD1300019F03D
:10AE6000DCFA03789A2B26D105A919F0DBFA0599AB
:10AE7000060019F0C1FA02281DD1300019F0C8FAF5
:10AE800007233200070029002000FFF70BFE029B7A
:10AE90000600DB0417D51F233A0029002000FFF726
:10AEA000D7FDF100039B029E80011E433143F8262B
:10AEB000F6003040E2E62A00174914480BF032F859
:10AEC000A368186026E76B4608229B5E002B07DA12
:10AED0003E233A0029002000FFF7BAFD4008E0E7D2
:10AEE0007C233A0029002000FFF7B2FD8008D8E754
:10AEF0000133062B9BD10DE730BF0000D281030048
:10AF000072B6000062B600008C82030004310300B8
:10AF1000D5820300BE45030061820300019B032B21
:10AF200000D0F7E6382E21D100263A680723290001
:10AF30002000FFF7B7FD7A68019007232900200061
:10AF4000FFF7B0FD1F230290BA6829002000FFF729
:10AF50007FFD019F029B374381013943DE0056E7A5
:10AF600080263601E1E780267601DEE7392EF7D02C
:10AF70003A2EF8D0362E2BD1C02607233A68290066
:10AF80002000FFF78FFD072301907A682900200039
:10AF9000FFF788FDBA687601137802900A3B0F2B01
:10AFA0000DD8072329002000FFF77CFD029BD90064
:10AFB000019B194331430F00810139432AE6802365
:10AFC000DB001E43290007232000FFF741FDEDE7CA
:10AFD000372E00D09EE6D026CFE703490348A46869
:10AFE0001DF04BFB206030E6C182030004310300FA
:10AFF000F7B506000D0000240192019B9D420AD086
:10B00000631C0093052B08D1B468124912481DF047
:10B0100034FB206000242000FEBD28780A38C3B22B
:10B020000F2B02D9B4680D49F0E76B780002184382
:10B030001AF0D2FA0235070021F018FD0228F1D1EA
:10B040003B78722BEED17B783034A342EAD1009C5E
:10B05000D3E7C046FC810300043103002F820300C4
:10B060000300203B5E2B00D93F20052320384343BB
:10B07000014A1068C01870477800002070B50500BC
:10B08000080068430130401008300C001BF0EDF957
:10B090000122044B8571036003794471934303716A
:10B0A00070BDC0467403030010B5040010201BF0EF
:10B0B000DCF9044B036063684360A368C36000234A
:10B0C000836010BD4800030070B5050020201BF010
:10B0D000CCF905210B4B040003600800FFF7CEFFFD
:10B0E0006B68EA68A060236162602A7C2000A27617
:10B0F000AA689B1863616B7CE3761AF092FC2000CF
:10B1000070BDC046BC030300037910B5DB0705D54D
:10B11000034904481DF0B1FAF5F759F810BDC046CF
:10B12000218403008831030070B50D000400FFF78F
:10B13000EBFF2800F7F754FB0100092805D9054962
:10B1400005481DF09AFAF5F742F820001AF0CBFCFA
:10B15000024870BDBF84030000320300D0DB020050
:10B16000F0B50C000B6889B0070018000493FFF7D6
:10B17000CBFF65682800F7F74BFA1F4B1F49984231
:10B1800002D1072F05D11E491E481DF076FAF5F7AA
:10B190001EF8A068F7F724FB0690E068F7F720FB9D
:10B1A00007902069F7F71CFB05906069F7F718FB1B
:10B1B000059B0600002B01DB002802DA1249134828
:10B1C000E3E7062F14D0A069F7F70AFB0700E06950
:10B1D000F7F706FB059B0390009328000297019662
:10B1E000079B069A04991AF02FFD094809B0F0BD93
:10B1F00000200700EEE7C046740303004E840300FE
:10B2000061840300883103007B8403000032030063
:10B21000D0DB020070B5040008001600F7F7E0FA72
:10B2200005003000F7F7DCFA0600002D01DB0028EE
:10B2300005DA0D490D481DF020FAF4F7C8FF20008B
:10B240001AF0EDFC854204DA20001AF0F6FC864282
:10B2500001DB0749EEE73200290020001AF0D1FC9B
:10B2600043000120184370BDD9840300003203005D
:10B27000F2840300F8B50D000C682000FFF744FFCE
:10B280006868F7F7ADFA0600A868F7F7A9FA0700AB
:10B29000002E01DB002805DA104911481DF0EDF9F8
:10B2A000F4F795FFE868F7F79BFA0500092801D93C
:10B2B0000C49F2E720001AF0B2FC864204DA2000C2
:10B2C0001AF0BBFC874201DB0749E6E72B003A0096
:10B2D000310020001AF0E0FB0448F8BDD9840300D7
:10B2E00000320300BF840300F2840300D0DB0200BD
:10B2F000F7B50E002649040001921BF0B5F9019B39
:10B30000002B03D1234920001BF0AEF92249200075
:10B310001BF0AAF9002530001AF08FFC854221DAD3
:10B32000002730001AF07BFC87420CDA39002A0033
:10B3300030001AF066FC194B19491A5C20001BF00A
:10B3400093F90137EDE7174920001BF08DF9019BB8
:10B35000002B05D130001AF070FC0138854211DB5A
:10B360000135D8E70C4920001BF07EF9019B002B2A
:10B3700003D10D4920001BF077F90C4920001BF088
:10B3800073F9F7BD0A4920001BF06EF9E8E7C046E3
:10B390008185030088850300968503009885030056
:10B3A0001C5003008E85030049490300C14A030075
:10B3B00090850300F0B50F00110000228BB01E0035
:10B3C00000920323380003F0C1FB032F00D9D5E01E
:10B3D000380010F009F8020C949405210800FFF7DA
:10B3E0004DFE04001AF08DFB20000BB0F0BD30685C
:10B3F000654B0340062B07D0830700D0C1E0634BA9
:10B4000002689A4200D0BCE007A9F8F731FC079B1C
:10B4100003900593012B04D1039B18781AF014FEB6
:10B42000E3E700231E00039A029303990598511A3B
:10B43000814218DA11780A2901D03A2908D19E42AE
:10B4400000DA1E00029B0133029300230132ECE775
:10B4500001332029FAD03929F8DD4D494D481DF036
:10B460000CF9F4F7B4FE002B05D0029A01320292D7
:10B470009E4200DA1E0002993000FFF7FFFD002512
:10B4800007002C00039B0493039A049B9B1A059AC4
:10B490009A4223DD049B1B780A2B01D03A2B0FD153
:10B4A000A64207DD210000232A0038001AF0F4FA32
:10B4B0000134F5E700240135049B01330493E3E7ED
:10B4C000202B07D1002321002A0038001AF0E4FACB
:10B4D0000134F1E7392BEFDC303BF4E7029B380015
:10B4E000AB4200DC81E7A64207DD210000232A00F1
:10B4F00038001AF0D1FA0134F5E7380075E7306802
:10B50000F7F76EF905007068F7F76AF90290010025
:10B510002800FFF7B3FD0390022F03D11AF0F1FAD0
:10B52000039862E7012207A9B068F7F713FB002D23
:10B530001FDB029B002B1CDB6B43089A934218D144
:10B5400000242700029B9C42EAD03E00EB190493A2
:10B55000049BF11B9E420ED0079B9A5D131C092A87
:10B5600000D90923DBB2220003981AF095FA0136BC
:10B57000EEE7094972E77F190134E3E70749084814
:10B580006DE70849FBE7C046070080FF84320300EF
:10B5900002850300003203002C8503004985030067
:10B5A0008831030068850300F0B585B0019105007E
:10B5B0000021019810F0FCF8041E05D0234924480E
:10B5C0001DF05BF8F4F703FE28001AF028FB0600D4
:10B5D00028001AF032FB01003000FFF74FFD070092
:10B5E00028001AF01CFB84422CDA002628001AF0EE
:10B5F00016FB864224DA3200210028001AF001FBF3
:10B6000011F09CF8019910F0A5FD12F07DFE0022CA
:10B61000104B11F029F9104B00220290039110F009
:10B620008DF80923002804D00298039912F0F6FD42
:10B6300003003200210038001AF02EFA0136D5E757
:10B640000134CDE7380005B0F0BDC0469384030057
:10B65000003203000000E03F00002240F0B587B058
:10B660000700039105921AF0E8FA040038001AF076
:10B67000D6FA019003981AF0E0FA84422DD1210005
:10B680000198FFF7FBFC0025029006E0049B1B1AC3
:10B69000DA43D217134019E00135019B9D4222DAAB
:10B6A0000026A642F8DA3200290038001AF0A9FA7A
:10B6B00032000490290003981AF0A3FA059B002B8E
:10B6C000E4D0049B1B18092B00DD0923320029005C
:10B6D00002981AF0E1F90136E3E7044904481CF046
:10B6E000CCFFF4F774FD029807B0F0BDA38503000A
:10B6F00000320300F8B5040008000D001600F6F74C
:10B7000087FF164FB84201D000200FE0053C042C03
:10B71000FAD820000FF05EFE141403F80B0030007E
:10B72000F7F7C2F8011C2800FFF73EFFF8BD300014
:10B73000F7F7BAF8011CFE20800510F01BFBF1E7BB
:10B740003000F6F765FFB842DED162426241310057
:10B75000D2B22800FFF782FFE8E7C0467403030077
:10B76000F7B507000193142008AB0E0015001C78F4
:10B770001AF07BFE044B476003606B461B798660C2
:10B78000C56003744474FEBDF803030070B5050082
:10B790000C201AF06AFE0521044B0400456003608A
:10B7A0000800FFF76BFCA060200070BDFCFF0200EA
:10B7B00070B5060008001DF0E8FD050018F09CFCBF
:10B7C000041E06D12A00084908480AF0ABFBF4F72A
:10B7D000FEFC30001CF056FE012102000300200098
:10B7E00005F0F0F870BDC046C1850300E02D0300F0
:10B7F00010B504001DF0C9FD1CF0CFFC01280BD0D2
:10B80000064920001DF0DBFD20001DF0BEFD1CF0F0
:10B81000C4FC022800D0002010BDC04612860300E0
:10B82000F0B59DB000AF0C68032859D9CB6800254E
:10B83000FB60042801D00D696D101C232000F9184D
:10B84000F8F716FA7861002D5BD0A04C6E21606885
:10B85000F6F792FC0600606800229621043000F0A2
:10B86000DBFC1823FA18D11804003000F8F700FAAE
:10B870003B6B013D0100C318002C05D1994203D256
:10B88000013B1A782E2AF9D1013D31D2FE695C1AAA
:10B890002500002E01D0751C65192B006A460E3359
:10B8A000DB08DB00D31A9D46220018003B6120F024
:10B8B0005CFF002E08D02E233A69601C1355101827
:10B8C0007969320020F051FF29003869FDF794FFB3
:10B8D000012810D17E497F481CF0CFFEF4F777FC99
:10B8E0007D4B0025FB60A8E7013B1A782E2ACBD0C0
:10B8F0009942F9D3C8E706243B69C0000443FD61BF
:10B900007B612000F7F728FD09F050F8061E15D0DE
:10B910002E21786921F092F800280BD06E4BFA683E
:10B920009A4207D17B69C11A1800FDF765FF09F03B
:10B930003DF806003000BD461DB0F0BD18231820AC
:10B940000125FA18D2183818103B4021C0181DF0F4
:10B95000C1FCBE603E61FB699D4205D95E4BFA6841
:10B960009A42E7D1BE68E5E79D4204D07B695B5D02
:10B970002E2B00D097E029007869FDF73DFF1822B3
:10B980000823BA183860D0181DF0CDFC002817D154
:10B990002A000823796918303818C0181DF05AFC9D
:10B9A00018220823BA18D018FFF722FF78607B68A6
:10B9B000002B14D13A68494946480AF0B3FA8DE79A
:10B9C00018220823BA18D0182F210BF0B1FA3B69BE
:10B9D0003969EA1A7B69182059180823DCE73868A6
:10B9E00008F0E4FF041E48D1386808F0A5FFFB69A1
:10B9F00004009D4208D13A4BFA689A4204D15E2273
:10BA00006E21806818F064FE7B68012B55D11822E6
:10BA10000733BA18D0181DF07FFC18220823BA1873
:10BA20007860D0181DF07FFC002201007868F7F7DD
:10BA300071FC12210200200004F03EFA18220823B3
:10BA4000BA18D0182F210BF073FA18220823BA184D
:10BA5000D01824491DF0B3FC18220823BA18D018B6
:10BA60001DF093FC1CF099FB02281ED0182208231D
:10BA7000BA180C21D0181DF0E2FC002E0CD07A6907
:10BA80003B699446E91A63441800FDF7B5FE2200AD
:10BA90000100300004F010FABB68002B00D1BC603C
:10BAA00026006B1C3B61013555E718220823BA18A4
:10BAB000D1182000FFF77CFED8E718220823BA1817
:10BAC000D1182000FFF774FED7E7C046380A0020DF
:10BAD000D6850300E02D0300D0DB0200F5850300CE
:10BAE0003C2403000A86030030B58DB0050068468B
:10BAF000F4F752FB011E10D12A1D01201BF09EF805
:10BB00000122EB6804005B1001335B001343EB6020
:10BB1000F4F758FB20000DB030BD0198054A0368CA
:10BB2000934205D0044A00249342F3D0F4F74FFB2C
:10BB30000024EFE7C8300300582E030010B50400BE
:10BB400010201AF092FC044B036023684360636882
:10BB500083600123C36010BD4004030010B5034A95
:10BB6000034904481AF080FD034810BDEE86030027
:10BB700001CD0300F8100300D0DB020010B5034A2A
:10BB8000034904481AF070FD034810BD16860300EF
:10BB900001CD0300F8100300D0DB02000023FA21DE
:10BBA000084A89001360084A1370084A1360084A5B
:10BBB0001160084A1370084AD36613670122074BC5
:10BBC0001A70704740030020390900203C03002010
:10BBD000200000203A090020380A00203B090020FC
:10BBE00010B5084B084A1978002907D1116B0029B4
:10BBF00002D0FFF7D3FF10BD30BFF4E700221A7068
:10BC0000F9E7C0463B090020380A0020837F02483C
:10BC1000002B00D101487047442403003C2403005A
:10BC2000A02010B50F49C0054B7F5A1C002B09D12D
:10BC30004C8C0D4BA3430D4C03510D4B4A775200D6
:10BC4000D05A0DE010335B00CB185C88A123DB00D9
:10BC5000C450092AF1D1012001F076F901204042B7
:10BC600010BDC04624000020F01F00000C0500009D
:10BC7000D64503000023E021A02210B583770C4BAA
:10BC80000902D205D1500B4808F058F90A4808F0CB
:10BC900055F90A4808F052F9094808F04FF90948DF
:10BCA00008F04CF9084808F049F9084810BDC046AA
:10BCB0000C0500002CE6020034E6020044E6020017
:10BCC0004CE602005CE60200D4E50200D0DB020094
:10BCD00073B5041E09D1194D2B78002B2BD01849B0
:10BCE00018481AF0C7F92C7073BD174EF56EF6F7A9
:10BCF0008FFC164B2100984214D0154B2340062B85
:10BD000005D0A30712D1134B22689A420ED101A984
:10BD10002000F7F7ADFF019B012B0CD100781AF042
:10BD200093F9010028001AF0A5F9DDE70A490B484C
:10BD30001CF0A3FC3063FFF731FFD5E73A09002080
:10BD4000F402030024000020380A002074030300DA
:10BD5000070080FF843203006888030088310300F5
:10BD6000034B1878013843425841C0B27047C0466F
:10BD700039090020F7B5A123A024224AE405DB00FD
:10BD8000E250C37F012219000D318A4001331E4960
:10BD9000DBB262500191032B31D0C3770200030064
:10BDA000002122333632198002339A42FBD1C47FFC
:10BDB000164A63000133D318052204259446012155
:10BDC00067465A1E12781E787A43114F0633BA1806
:10BDD0000F00AF4092191279013552008218568C2B
:10BDE0003E4356840D2DEBD10D34A023A122A1405A
:10BDF000DB05D2009950828E01995A50F7BD00237D
:10BE0000CBE7C046F01F00000C050000328803009D
:10BE10002400002070B5304D8CB0AB7F002B1FD0BC
:10BE20002800FFF7A7FF2D4A2D491368096806333C
:10BE300013608B4207D300242A4B14601B78012B1C
:10BE400010D0022B43D000232A8C6B77FF33FF33B3
:10BE50001A4205D0E1222449D200012001F040F825
:10BE60000CB070BD214EF36E002B02D0336F002B4F
:10BE700002D1FFF793FEE6E7F5F77CFC6846F4F79E
:10BE80008BF900280CD11A4B186804F05FF80400F5
:10BE9000F4F798F9F5F778FC2000FFF719FFD2E7DF
:10BEA000F5F772FC019B134918680AF0AFFF0028F0
:10BEB000F2D10198F6F7ACFB0F4B984203D10F4932
:10BEC0000F481AF0D1FB019B00243363E4E70D49CE
:10BED00028001AF0CFF8CCE7240000203C03002013
:10BEE000200000203909002021BC0000380A002071
:10BEF00040030020C8300300542F03008B88030048
:10BF0000F8100300F4020300F7B50024009308AB17
:10BF1000124D1B780600080017000193EC662C6791
:10BF200003F0EEFF6A460E4B127818600D4BEE667A
:10BF30001F600D4B28671A700C4B1C7004F006F83C
:10BF4000FFF7C6FE01220A4B1C600A4B1A70019BC8
:10BF5000A34201D0FFF744FEF7BDC046380A0020D7
:10BF600040030020200000203A0900203B09002067
:10BF70003C03002039090020F0B500242B4B8DB084
:10BF8000DC661C672A4B07AC40C90138009301945A
:10BF9000052302F00DFE0798636805900293237B4A
:10BFA000257A0393234B277C0340062B05D0830778
:10BFB0002ED1214B02689A422AD106A9F7F758FEE2
:10BFC000069B002B21D0012B0CD1002D0AD1002F74
:10BFD00008D100781AF038F80590059930001AF069
:10BFE00049F812E00598FFF7D1FB0590237C002B60
:10BFF00003D00598FBF71EF80590039B029A009367
:10C0000005992B003000FFF77FFF0C480DB0F0BD05
:10C01000F6F7FEFA0A4B9842E8D1002D01D1002F25
:10C02000DBD005A90120FAF7F1FEDEE7380A00208F
:10C0300054050300070080FF84320300D0DB0200B8
:10C040007403030030B5104B89B003AC20C901382C
:10C0500000930194052302F0ABFD02A90398F7F7C2
:10C0600007FE227C237B02990092039AFFF778FB5C
:10C07000237A01000093280000236268FFF744FF41
:10C08000024809B030BDC04690050300D0DB020075
:10C090000022074B10B51A70064B02321A70064B7D
:10C0A000064A1B68063B1360FFF79AFD10BDC046A9
:10C0B0003B09002039090020200000203C0300201B
:10C0C00010B5FFF7E5FF014810BDC046D0DB020008
:10C0D00010B5042901D8042A05D90A490A481CF0D8
:10C0E000CCFAF4F774F8092B01D90849F6E70524CE
:10C0F000614341188A18137101229A40038C13433B
:10C10000038410BD7688030000320300BF8403005F
:10C11000F8B548680C000D68F6F762FB0600A068E9
:10C12000F6F75EFB0700E068F6F75AFB3A000300FB
:10C1300031002800FFF7CCFF0048F8BDD0DB02003B
:10C1400010B5042901D8042A05D9064906481CF06F
:10C1500094FAF4F73CF80523594340188018007905
:10C1600010BDC0467688030000320300F7B51B4FB0
:10C170000190380007F0D4FE194E300007F0D0FED1
:10C18000184D280007F0CCFE174807F0C9FE1748E5
:10C1900007F0C6FE164807F0C3FE164C3800210013
:10C1A00007F0E2FE3000210007F0DEFE280021004B
:10C1B00007F0DAFE21000C4807F0D6FE21000B48FC
:10C1C00007F0D2FE21000A4807F0CEFE19F0D9FF91
:10C1D0000123019A08489377FEBDC0462CE6020071
:10C1E00034E6020044E602004CE602005CE602008F
:10C1F000D4E50200F4280300D0DB020070B505008E
:10C200000C200C001AF031F9024B45600360846089
:10C2100070BDC0462C060300F0B587B000920278CE
:10C2200004000E00930703D5009B002B00D0E0E034
:10C23000D307DB0F0ED0704B3340062B43D00323C4
:10C24000334003D16D493068884203D0009B012BF5
:10C2500000D0CEE00193530749D52368A568DF08D5
:10C26000FF00EF19BD4230D3009B012B00D0C0E08E
:10C270002368D9086368994210D104316160A068CD
:10C28000C9001AF008F923686268DB08D21ADB00DB
:10C29000A060D200C018002120F082FA0721236894
:10C2A000DD086A1CD2000B4013432360A368ED0035
:10C2B0005D19514B2E601E40062E4ED00122237870
:10C2C0009343237049E00123C4E72868864204D1E0
:10C2D000009B022B41D104237CE0019B002B04D165
:10C2E0003100F6F72BFA0028F2D10835BAE7636877
:10C2F000002B06D1009B012B00D07AE0200000F03B
:10C300007FF83D4B33400593062B29D1F00819F0F7
:10C3100059F90390616803980FF00AF90027049116
:10C32000049B0293029BDD00A3685D192868002826
:10C330001DD1009B012B5CD107212368DA08013253
:10C34000D2000B4013432360002F00D03D00002398
:10C350006B60059B2E60062BB0D1280007B0F0BDA6
:10C360003100022003F06AFC43100393D2E7042853
:10C370001DD1002F00D12F000298616801300FF00D
:10C38000D7F8049B02918B42CCD1009B012B30D17A
:10C39000002F2AD023683D000833236000237B60F0
:10C3A000059B3E60062BD8D02378009A88E786420A
:10C3B00012D1009B022BD0D123680298083B236046
:10C3C000013061680FF0B4F8A368C900CB58002BA6
:10C3D00000D080E72B60C0E7019B002BCCD131005F
:10C3E000F6F7ACF90028C7D0E3E7200000F008F822
:10C3F00090E70025B1E7C046070080FF84320300C4
:10C40000F7B54368040001935A1C002316495D5890
:10C41000AA4204D904335C2BF9D101251543E80065
:10C42000A7681AF034F807232268656013400122D8
:10C430003D000026236013432370A060019B9E42B1
:10C4400003D138001AF038F8F7BD2968002907D061
:10C45000042905D001222000FFF7DEFE6B6843604F
:10C4600001360835EAE7C04668060300F8B505005E
:10C4700000230768866811497A1C5858824204D9FB
:10C4800004335C2BF9D101201043002428606C6038
:10C49000800019F0FCFFA860BC4203D130001AF004
:10C4A0000BF8F8BDA300F158002905D0042903D0EA
:10C4B0000122280019F0E6FE0134EDE768060300CA
:10C4C00001220020074B08495A600860A821DA6061
:10C4D000064AC9005A5006495A5004315A50054973
:10C4E0005A507047009000400C9C0040FCFF000038
:10C4F000440500004C050000034B04481B78002B4A
:10C5000000D103487047C0463D0900204424030081
:10C510003C240300F8B5A826324A334BF6001968CC
:10C5200013680420CB18C9181160304A8C46127861
:10C530001B11170009112E4A2E4C2F4D002F47D0EA
:10C54000002B39DA9051C31AA920C000135081235F
:10C550009B00002936DA591A135151510123274CF7
:10C56000D3602378002B21D03F222548254B01683A
:10C570009B6F01310A409D5C1C4B1B78002B01D046
:10C58000803D6D001C23026062466B4308339B1A9A
:10C59000154A9B1013601F23194007D11A4B1A78B4
:10C5A000002A03D01948197000F000FD01232278F9
:10C5B000042053402370F8BDA9270433FF00D05155
:10C5C0009351C4E7535181239B00C9181151C5E70A
:10C5D000043390515351A9208123C0009B00135074
:10C5E000F3E7C046440300205403002076020020F5
:10C5F000009000404C050000440500003C0900206C
:10C6000048030020380A002077020020136402004B
:10C6100030B585B001220400080001A9F6F79AFAA6
:10C62000029A202A00D920220023019D934204D09F
:10C63000E85CE11808710133F8E7014805B030BD46
:10C64000D0DB020070B5040008001500F6F7C8F84A
:10C650000E491F2815D8002D05D10D490D481CF095
:10C660000CF8F3F7B4FD2418042D04D1012023792C
:10C670005B00184370BD2800F6F7B2F8FF2802D916
:10C6800005490648EBE720710548F3E7BD8803003C
:10C69000D188030088310300F688030000320300CC
:10C6A000D0DB02000123A022834010B5134CD20539
:10C6B00013510300C133124CFF339B009C50114BAC
:10C6C0008900C918A223DB00CA580F4C000222407F
:10C6D000CA50F82252011040C022CC589202224384
:10C6E00010430322C850CC58084822432043C85066
:10C6F000C046C046C046CA5010BDC0460C0500002A
:10C700000303000000600040FFE0ECFF031F000097
:10C71000A0221E21114BD20070B59C58104D8C43A5
:10C720009C50A324E4001D510E4C0F4D0F4E5C5144
:10C7300004355E510E4D80005C51A5240D4DE40082
:10C740001D51084C0C4D00190C4C185104341D514E
:10C750000B4C185198580143995070BD00F001409E
:10C7600040910040006000401C05000044910040E2
:10C7700024050000489100404C9100402C05000029
:10C780003405000070B50D00040007F0C9FB134E1E
:10C790002800310007F0E8FB3100200007F0E4FB3F
:10C7A0000F4BA0221C600F4BD2051D606079012445
:10C7B0002100814026000C4BD15069798E40002128
:10C7C000D650FFF76FFF68792100FFF76BFF20005D
:10C7D000FFF79EFF054B1C7070BDC0460C2903007F
:10C7E0004C030020500300200C05000076020020BE
:10C7F00010B504000A4907F0B7FB0A4BA0211C60E2
:10C8000001236079084A8340C9058B500021FFF756
:10C8100049FF0020FFF77CFF0022044B1A7010BD77
:10C820000C2903004C0300200C05000076020020B8
:10C83000F8B50025FFF744FE214B2800DD6700F026
:10C8400083FBA0221E201F4B1F491D701F4BD200CF
:10C850001D601F4B1F4C1D608B581F4F83438B5017
:10C86000A223DB00E2581D4E3A40E250E2581C4938
:10C870003243E2500122E5501A4B186843799A403E
:10C880001300A022D205535007F058FB164B1B781B
:10C89000AB4213D0154B1249E2581740E750E2580B
:10C8A00016430122E650E550114B186843799A402F
:10C8B0001300A022D205535007F040FBF8BDC0463C
:10C8C000380A00203D09002000F001404403002008
:10C8D0005403002000600040FFE0ECFF001F030055
:10C8E0000C0500004C030020760200201405000017
:10C8F00050030020F0B53A4E8DB0F36F0500002BC9
:10C9000003D1FFF795FF0DB0F0BD002801D0F4F77B
:10C9100031FF6846F3F740FC00281DD1F06F03F0AB
:10C9200015FB0400F3F74EFC002D01D0F4F72CFFAB
:10C9300020222C4B1D68B36F6D1101356D01154020
:10C940005D19002C2CD121002800F4671FF028FF6E
:10C950000122254B1A70D6E7002D01D0F4F714FF01
:10C96000019B224918680AF051FA00240500A042F0
:10C97000DED1019F3800F5F74BFE1D4B98420BD1DD
:10C9800029000120FAF742FA2A000400F8601F216A
:10C990001848F6F7BFFCA060019B00243363C7E78B
:10C9A0002000F5F735FE144B984207D000231349B9
:10C9B0001348F3671BF061FE3063A4E763682B60E4
:10C9C000A3686B60E368AB602369EB6063692B610C
:10C9D000A3696B61E369AB61236AEB61B8E7C046A9
:10C9E000380A00204803002077020020C8300300E6
:10C9F000542F03008B880300C8070300AB88030093
:10CA00008831030010B5FFF713FF014810BDC04681
:10CA1000D0DB0200F0B589B00493704B03901B7813
:10CA20000E001500002B01D0FFF702FF6C4B1A78A7
:10CA3000002A07D16B4C4020E26701321A7019F0CE
:10CA400014FDA06780270122674BBF00674CDF679A
:10CA5000674BE250FFF734FD0023664AF021A350F4
:10CA60000432A3500832A350C22209039200A150FD
:10CA7000E351614F0594BE4200D09FE0B54200D023
:10CA800096E05E4D07AC280007F062FA002805D05A
:10CA900001235B492800237007F066FA594D2800EE
:10CAA00007F056FA002805D0012355492800637085
:10CAB00007F05AFA544D280007F04AFA002805D02A
:10CAC00001234F492800A37007F04EFAA027002445
:10CAD000FF0507ABE35C002B33D10134022CF8D106
:10CAE0004648F8F7C5FBFFF783FE002601240398AC
:10CAF00003F006FA3F22454B3A4D1E70444B80210D
:10CB00001C70444BE8671A60A86F12191FF048FEAA
:10CB10003000FFF7EFFE404B304F1C60059B50226A
:10CB20001C603E4930003C7000F0DAF9049BB342CF
:10CB300052D03B78002B4FD02B6B002B4CD120BF19
:10CB4000F7E7374BA200D65803227379651CC1332F
:10CB5000FF339B00DA5107ABEB5C002B24D0304B4A
:10CB6000AA00D358019304230093012273799A40B9
:10CB7000A123DB00FA50019B05331800029319F042
:10CB800028FC012810D173799840264BF850029860
:10CB900019F01FFC002807D1009B013B0093002BDC
:10CBA000E3D10199300014E00135032DD3D194E78E
:10CBB0001D491E481BF061FDF3F709FB3000F8F733
:10CBC00057FB0400BD428ED02800F8F751FB01004E
:10CBD0002000FFF7D7FD88E709B0F0BD3D09002030
:10CBE0003E090020380A002004E100E000900040E7
:10CBF000FC0F000004050000D0DB0200CCE50200C1
:10CC0000DC28030014E6020024E602003C090020B0
:10CC100077020020480300200C9C004015C500004E
:10CC2000800703000C050000098903008831030018
:10CC300010B5084B86B002AC00930194042301F0B8
:10CC4000B7FF02982379E268A168FFF7E3FE024884
:10CC500006B010BD8C070300D0DB0200014B187832
:10CC6000C0B270473D09002010B5242019F0FDFB2B
:10CC70000400044B202208C080211FF091FD2000F9
:10CC800010BDC046C8070300F8B5050008000E0037
:10CC90001700F5F7BDFC324B984201D00020F8BDDB
:10CCA000681F0F28FAD80EF095FB080835F9F9F936
:10CCB000F9F9F9F9F9F9F9333358FFF7D5FF0423F6
:10CCC0000400F25CE2540133242BFAD13800F5F76A
:10CCD0009FFC234B9842E1D10121052D05D0123D47
:10CCE000691E8D4101216D4229430422FF20BB5C56
:10CCF000A55C803B4B435B19FF2B03D90500DB1779
:10CD00009D432B00A3540132242AF0D12000C6E712
:10CD10003400DBE7FFF7A8FF04230400F25CE254D1
:10CD20000133242BFAD13800F5F7BEFD0F2119F09D
:10CD300075FB2100FF25221D24311378803B4343DE
:10CD4000DB138033FF2B03D92E00DB179E43330008
:10CD5000137001329142F0D1D8E73400E3E7C046C6
:10CD6000C80703008022044B52001A600123034AC3
:10CD70001360034A1360704700E100E00C8C004030
:10CD8000008000408022054B5200DA67044BFF3AD6
:10CD90005A600022034B1A607047C04604E100E06D
:10CDA000008000400C8C004070B501251D4B1E4CCE
:10CDB00018601E4BE550C046FFF7E4FF1C4A1D4BB0
:10CDC000E560E250002303211B4AFF20A3500432F8
:10CDD000A15049190832A1508021C12209039200B3
:10CDE000A150053AFF3AA350C224144BA40019598C
:10CDF000C13A8143FF3A0A4380211A510C341A592F
:10CE000009061202120A0A431A51C022043419599F
:10CE100081430A431A51802212041A60802252046C
:10CE20001A6070BD6803002000800040FC0F000005
:10CE3000701700004C0500000405000000E100E050
:10CE400070B51F4C1F4D636C002B0AD00023636428
:10CE50001D4B1B689847A823DB00EA580001801887
:10CE6000E850A36C002B09D00023A364164B5B6829
:10CE70009847164B0001EA588018E850E36C002BE5
:10CE80000AD00023E364104B9B689847A923DB007A
:10CE9000EA5800018018E850236D002B0ED00023C3
:10CEA0000B4A2365AB580B495B18AB500A4A136811
:10CEB000063313608022094B12045A6070BDC046CD
:10CEC000FC800040008000405C0000204405000021
:10CED0004C05000070170000D8080020FCE100E0BD
:10CEE000F7B50191032823D8134B8000C758C223FC
:10CEF000124D9B00EF50012344192364A8230F21F6
:10CF00000F4EDB009C46E358AE59921BD218D31744
:10CF10000B409A1801990B4B1211C150C1239B0071
:10CF2000EF5063460020013212019619E650FEBD13
:10CF300001204042FBE7C046EC10030000800040A7
:10CF40004C0500005C00002003280BD8074B800034
:10CF5000C158C223064A9B00D150064A064BC25014
:10CF60000020704701204042FBE7C046EC10030060
:10CF700000800040C16402005C00002010B5024B3C
:10CF80001B68984710BDC0466803002010B50024F8
:10CF9000054AA358002B02D00021A1509847043421
:10CFA000102CF5D110BDC04658030020074A890057
:10CFB0008B58002B06D1885080211800044A490460
:10CFC0005160704701204042FBE7C04658030020F3
:10CFD000FCE100E0F0B587B0039205910D9A03994A
:10CFE0000500521A0CA9097820200C00844339D07E
:10CFF00030293BD00CA902910121802401911C40D1
:10D0000036D0D40FA4186410171B002C37DD26006F
:10D01000019B0493B34200DD04966B68049A029965
:10D0200028689847049BF61A002EF1DC039B002B1E
:10D0300006D01A0005996B6828689847039BE41886
:10D04000002F0CDDE419019EBE4200DD3E003200DF
:10D05000029928686B689847BF1B002FF3DC2000FB
:10D0600007B0F0BD074902911021C6E70649FAE76B
:10D0700001271F4001D11400C7E71700D6E700249D
:10D08000D4E7C0463D8903004E890300F0B593B054
:10D09000069318AB20CB04901B780F001600079363
:10D0A000CB070BD48B0703D1854B0A689A4205D076
:10D0B0003800F5F795FB01274000074381231D4207
:10D0C00009D1079B302B06D11A9B1B9A934200DA99
:10D0D0001A9200231B93380018F04BF80AAA130089
:10D0E000002806DDAB070FD52B231370123B04AAD3
:10D0F0009B18EA0616D5022E0DD130221A70069A18
:10D1000001325A7002330DE013006A07F1D5202274
:10D110001A701923EBE7082E3CD130221A70AA05A9
:10D1200035D4013300220AA91A705B1A0593AB06A5
:10D1300000D52C320EAB0B93102300210C931B9BBC
:10D140000D91012B01DD40231D4304ABD9756B46C6
:10D1500040241B7E2C400392029322D03B0001917D
:10D1600000960DAA0CA90BA8FCF7C4F903780700D8
:10D170002D2B2DD104AAD3750D9B1B9A013B013792
:10D180000D93012A00DD95E0002634004AE0069A5E
:10D190000E32B6E7102EC5D130221A70069A173219
:10D1A000AFE70AAB019300963B000DAA0CA90BA8B0
:10D1B000FCF7A0F91B9B07002600012B32DD0D9B1D
:10D1C0001B9C9C4215DA1C0013E00026340019E079
:10D1D0001B9B012BD8DD0D9B1B9C9C4200DA1C0085
:10D1E000172304AA9B181B78002B00D00134059B41
:10D1F000E4181A9BA342E8DD01261C1B2E4001D037
:10D200002600002401239D432F330793002C09D0CF
:10D21000103B0093002301941A002A490498FFF759
:10D22000D9FE04006B0621D5172104ABC9180B7871
:10D23000002B0AD000230122009301920498FFF7EB
:10D24000C9FE1A9B2418013B1A93059B002B0DD095
:10D25000012301930023059A00930AA90498FFF77C
:10D26000B9FE1A9B059A24189B1A1A931B9B012B33
:10D2700000DD1A931A9B0D9A0193079B39000093C6
:10D2800004982B00FFF7A6FE2418002E09D02023B7
:10D290000093002301961A000A490498FFF79AFEAA
:10D2A00024180B980EAB984201D019F005F9200014
:10D2B00013B0F0BD1B9C9C4298DA1C0096E7C04658
:10D2C000A0F00200C8CB0300F0B506001400002750
:10D2D0008DB00D002B78002B1ED1A94208D26B1AFD
:10D2E00004931A003068736898472900049BFF185C
:10D2F0000B78002B00D13EE14B1C0493202300252A
:10D300003022082104200893049B1B78002B07D1AE
:10D310000693013B079355E0252BDED00135D9E775
:10D320002D2B05D12C3B1D43049B01330493EBE7CC
:10D330002B2B01D1293BF6E7202B01D10543F3E745
:10D34000212B01D10D43EFE7302B23D000230A21FD
:10D350000693049B1B781A00303A092A1ED92E2BFB
:10D3600050D1049A049B527801332A2A1FD0049387
:10D3700000230A210793049B1B781A00303A092ADC
:10D3800020D8079A4A43D318303B0793049B0133B4
:10D390000493F0E7402308921D43C5E7069A4A43E9
:10D3A000D318303B0693049B01330493D1E7049BCD
:10D3B00002330493236804340793DB43079ADB1793
:10D3C0001A400792049B1B786C3B59425941049BBD
:10D3D0005B1804931B780593002B00D1CBE0642BE2
:10D3E00000D1A1E022D8502B29D00ED8453B022BEA
:10D3F00000D8A9E001220499306873689847013782
:10D40000099452E001235B4284E7059B622B3CD0E8
:10D4100057D8582BEED1231D0993069B01950393F2
:10D42000089B029341230093313B7BE0059B712BCA
:10D4300053D00FD8672B00D886E0702BDAD1231D8C
:10D440000993069B01950393089B02936123009324
:10D45000513B67E0059B752B5AD0782BEFD0732B8F
:10D46000C8D1231D24680993002C49D0079B0133A0
:10D4700003D120001FF0FAFA0790069B079A019348
:10D48000089B210000932B000BE0231D09932368C8
:10D49000002B0ED0069B04220193089B3749009372
:10D4A0002B003000FFF796FD3F180499099C0131CD
:10D4B0000FE7069B05220193089B314900932B003F
:10D4C000EFE7231D099323680BA90B70069B01222C
:10D4D0000193089B00932B00E3E7231D0BA9206811
:10D4E000099318F07EF8079B0100013301D10B9BD3
:10D4F0000793069B079A0193089B00932B00D0E7A4
:10D50000069B06220193089B1E4900932B00C8E747
:10D51000231D0993069B01950393089B02936123A6
:10D520000093573B00220AE0231D0993069B01222A
:10D530000393089B0195029361230093573B216855
:10D54000300018F0D5FFAFE7072307349C432300D2
:10D55000206861680833099310F028FF079B011CBD
:10D560000293069B059A0193089B300000932B00C1
:10D5700019F032F898E738000DB0F0BD2B890300A0
:10D580003089030036890300034B04481B78002BC5
:10D5900000D103487047C04600D002004424030075
:10D5A0003C24030010B5DA2018F05FFF002303705D
:10D5B000024B8C331860024810BDC046380A002068
:10D5C000D0DB0200F0B507000E001500094C87B053
:10D5D0002000019317F081FC02AB1F70019B102209
:10D5E00002A92000039604950593F9F731FD07B0D1
:10D5F000F0BDC04600D00200F0B5784B99B08C3336
:10D600001A680192002A02D1002019B0F0BD00244E
:10D610001C60019B1B78A342F6D00126019B704F32
:10D6200002331093019B109DD233119302933B0060
:10D630002341334211D01A2302991B1B2800039364
:10D6400019F04FF8BB235B00984206DC3300A3407F
:10D6500032009F43039B9A409743029B0134083B4F
:10D66000083502930D2CE2D10A230893002302937C
:10D67000029810F049FE089B12901391013B089309
:10D6800014AA39000198002B00D188E0002618F078
:10D69000F6FF109B0E93119B0D93524B0F931A2381
:10D6A0009B1B0B930E9B09960C930D9B0A934D4B62
:10D6B00004930C9B4B4C07930B9B16AD05930A9B55
:10D6C0000693099B03933B00039A134101221342E3
:10D6D00025D014AB0F9A1B882900D3182B8014ABCC
:10D6E0005B88049A0798D3186B8014AB9B8814AAA4
:10D6F000E318AB8019F024F8011C02980EF06CF8C6
:10D70000002862D114AA2900069819F019F880227D
:10D71000029B120699180EF05FF8002855D1039B62
:10D7200001330393069B083B0693059B013B05933E
:10D73000FA23DB00E418079BA4B208330793FA230B
:10D740001B019C42BFD1FA22D2009446099B0333AD
:10D7500009930A9B183B0A930B9B033B0B930C9B6F
:10D7600018330C93049B63449BB20493A342A0D14F
:10D770000D9B0936483B0D930E9B48330E930F9B30
:10D7800063449BB20F931B2E89D112981399164AAA
:10D79000164B0FF069F810F009FE029068E718F0D8
:10D7A0006EFF040014AB04229B5E14AA0221525E99
:10D7B00014A90020095E1B01120109010120FFF7D5
:10D7C00001FF200017F0F9FC1FE70122059B0399D8
:10D7D0009A4001238B4013439F43A0E7380A00205F
:10D7E000FFDFFF0730F800009A9999999999B93F9E
:10D7F000F0B5584C8BB00390A37F002B05D1564950
:10D8000056481AF03AFFF2F7E2FC0398FFF7CAFE17
:10D8100000225349200018F08AFCFEF7A1FA0028E4
:10D820000BD0504800F0A6FB002804D14E4800F071
:10D83000A1FB0028F1D0FEF72BFC202018F004FCFF
:10D8400000230700190007AA995401330C2BFBD1C0
:10D850000224002325000293019306AB05AA04A924
:10D8600042481AF05FFD002322002900380018F01A
:10D8700013F9049B3E4A002593420CDB1900013545
:10D88000C83108DBC821033589008B4203DC013D28
:10D89000C82B00DC013D059B002493420CDB1A00E1
:10D8A0000134C83208DBC82203349200934203DCFF
:10D8B000013CC82B00DC013C0422029B134205D131
:10D8C000092322002900380018F0E6F80023294E29
:10D8D0000093009A07ABD25C002A2AD00923727801
:10D8E0003178380018F0D8F8009B023601330093E5
:10D8F0000C2BEED1174E3900300018F0BBFB642022
:10D9000006F0D6FA029B01330293019B0B2BA4DD98
:10D910001949300018F0AEFBFA20800006F0C8FA72
:10D920000398FFF769FE0400FEF7B2FB20000BB07E
:10D93000F0BD3278AA42D7D17278A242D4D1012167
:10D94000009AD154019B220001330193290009233D
:10D95000C7E7C04624000020778903008030030019
:10D96000A3890300CC140300D81403004427030048
:10D97000E0FCFFFF5F8903005CFE0200002310B59E
:10D9800018001A001900FFF71DFE014810BDC0461F
:10D99000D0DB020070B500210320F9F737FA084DFB
:10D9A0000400686817F009FCA060A86817F005FC7F
:10D9B000E060E86817F001FC2061200070BDC046FF
:10D9C00000D0020070B548680C00F4F709FF0500AC
:10D9D000A068F4F705FF0600E068F4F701FF3200E5
:10D9E000030029000120FFF7EDFD014870BDC0468E
:10D9F000D0DB0200F8B50B4E3378002B10D10A4D66
:10DA00002C78E4B2002C0BD1012700682F7003683A
:10DA10005B689847054A2C7013683770DB191360F0
:10DA2000F8BDC0463F090020400900206C030020DB
:10DA3000F0B53E4B87B01B780400002B01D1FFF7F7
:10DA4000D7FE201DFFF7D6FF394D28000CF090FBC4
:10DA5000002160681DF0B9F8344E0490736800210D
:10DA6000606805931DF0BEF8B368002102906068FD
:10DA700003931DF0C4F8F368C01A0EF05FFE041C97
:10DA800028001EF0AAF8061C28001EF09DF8051CB0
:10DA9000301C11F02BF8071C301C10F0A3FE019075
:10DAA000281C11F023F8061C281C10F09BFE029B7A
:10DAB000039A051C981A0EF041FE291C0EF04AFB31
:10DAC000311C051C201C0EF045FB011C281C0DF010
:10DAD000BFFF80231B06059AC518049B981A0EF0F9
:10DAE0002DFE01990EF036FB211C061C381C0EF091
:10DAF00031FB011C301C0DF0ABFF80231B06C0184E
:10DB0000291C11F063F90B490EF024FB10F0FCFB0B
:10DB1000094A0A4B0FF0B8F910F080FB002801DA2F
:10DB20006930FF3017F049FB07B0F0BD00D00200AC
:10DB3000CC0600200000B443EA2E4454FB211940D7
:10DB400010B504000430FFF755FF002160681DF098
:10DB500056F8034BDB68C01A17F02FFB10BDC04608
:10DB600000D0020010B504000430FFF743FF00218D
:10DB700060681DF02AF8034B5B68C01A17F01DFBA4
:10DB800010BDC04600D0020010B504000430FFF7FD
:10DB900031FF002160681DF025F8034B9B68C01A17
:10DBA00017F00BFB10BDC04600D0020070B500217D
:10DBB00005000320F9F72AF90400281DFFF71AFFD2
:10DBC000002168681DF001F80C4E7368C01A17F048
:10DBD000F4FAA060002168681DF004F8B368C01A68
:10DBE00017F0EBFAE060002168681DF008F8F368B0
:10DBF000C01A17F0E2FA2061200070BD00D00200C8
:10DC0000F0B54C4B89B08C331B680293002B4CD081
:10DC100049480430FFF7EEFE484C002120001CF07C
:10DC2000D4FF00210311200003931CF0DBFF00212F
:10DC30000311200001931CF0E2FF03110493029BE7
:10DC4000039A1B785242002B31D1019B0321D31A36
:10DC50009C4649420800654609380124032664426F
:10DC60000319029FDB00FB186A461F0092896A377E
:10DC70003A806A46928870337A806A46128A013EF8
:10DC8000BA80049F67437F191F800134002EE7D1BB
:10DC9000019B0330ED188142DFD1039B09319C4485
:10DCA0001829D7D10123029A137009B0F0BD019B46
:10DCB000D71A032252421100059709390120032681
:10DCC0004042049C059B4443E3180693029C0B18B6
:10DCD000DB00E3181C00703407940025645FA44641
:10DCE000069C644515DD6A24A4466D469C44644642
:10DCF000AD8925806C24A4466D469C446446AD885D
:10DD00006E3325806C46248A1C806C46079B248BCE
:10DD10001C80013E0130002ED3D10598019B0331B8
:10DD2000C31805938A42C9D1039B0932FF18182AE8
:10DD3000C1D1BAE7380A0020A81203000807002062
:10DD400010B54A68014918F08FFC10BD749F03009C
:10DD5000F7B50191114904001700002518F0B9FB2F
:10DD60007B689D4204D30E49200018F0B2FBF7BD3A
:10DD7000002D03D00B49200018F0ABFB019BAE0037
:10DD80009A5909492000BE1918F06EFC0122B168A9
:10DD90002000F4F755FC0135E2E7C046018A030094
:10DDA000C14A03003C480300B1890300F0B5114BA0
:10DDB00087B003AD40C9013800930195032300F0FB
:10DDC000F7FE68680C4C1E27A04202D016F02BFF0D
:10DDD0000700A8680022A04202D016F024FF02002B
:10DDE000706803990771427109F03CFC200007B08C
:10DDF000F0BDC046D0130300D0DB020030B5124B9B
:10DE00008BB003AC20C9013800930194032300F0C8
:10DE1000CFFE616806A81BF055FA039B089A5900CB
:10DE2000237A00936868079B0AF09EFD021E05D0C6
:10DE30000649074808F076F8F2F7C9F906A9054837
:10DE4000F5F732FA0BB030BDF4130300B5890300C7
:10DE50000830030008E0020030B5114B89B002AC75
:10DE600020C9013800930194032300F0A1FE012290
:10DE700005A96068F4F76EFE029B059A5900237AA3
:10DE800000936868069B0AF0B9FD021E05D005499B
:10DE9000054808F047F8F2F79AF9044809B030BD90
:10DEA00018140300D889030008300300D0DB0200F7
:10DEB00010B50124037A05499B005A5804482242B0
:10DEC00000D10448A243CA5010BDC04670030020D0
:10DED000442403003C24030070B5037A064C05007B
:10DEE0009B001859400817F068F901222B7A9B0013
:10DEF00019590A401A5170BD7003002070B5A22252
:10DF0000A025D200ED05AA580723CA401100174CDE
:10DF10000340E056421EC90700D5421C022A0BDC12
:10DF200000218A421CDB124DEE5C30008E4201D093
:10DF30000220E954E25470BD072A09DD0C2A12DCE4
:10DF40000B490320CD5C002DF4D10238C854F1E711
:10DF500007490320C95C4D1EA94149420840E9E731
:10DF60000A000800E6E703200C22E3E78002002015
:10DF7000780200200722436801201B791340024ADF
:10DF8000D35C58407047C0467802002010B5FFF7B8
:10DF9000F1FF034B002800D1024B180010BDC04612
:10DFA000442403003C2403001D4B70B559791879B3
:10DFB000FFF7A4FF022805D11A490B689A1C012318
:10DFC00013430B60184B59791879FFF797FF022814
:10DFD00005D114494B689A1C012313434B60134C21
:10DFE000200005F07FFF124DA84203D1617920790E
:10DFF000FFF784FF0F4C200005F074FFA84203D107
:10E0000061792079FFF77AFF0B4C200005F06AFF59
:10E01000A84203D161792079FFF770FF70BDC04637
:10E020003CE6020070030020DCE50200CCE50200C3
:10E030001429030014E6020024E6020007220379F3
:10E040001340014AD05C70477802002070B504008C
:10E050000D00104918F03DFA696801222000F4F71C
:10E06000EFFA0D4E2000310018F033FAA9680122B2
:10E070002000F4F7E5FA3100200018F02AFAE968E8
:10E0800001222000F4F7DCFA0449200018F021FAFC
:10E0900070BDC046FC8903003C480300C14A030030
:10E0A00070B5060010200D00140018F0DEF9034BC7
:10E0B000466085600360C46070BDC04608150300FB
:10E0C000F7B5040005200D000DF054F82000F4F71A
:10E0D00087FB694C20702800F4F782FB674BC0B2C5
:10E0E00018702378012B14D0022B1CD0102B1CD0BD
:10E0F0000F2B1CD0052B1CD00E2B1CD00D2B1CD095
:10E100005F490B2B06D05F495F481AF0B6FAF2F769
:10E110005EF85E49012812D0022855D05C4C1028C8
:10E120000ED05C49F0E75C49F4E75949F2E75B49F6
:10E13000F0E75B49EEE75B49ECE75B49EAE7534C04
:10E14000A02604224B79F605C133FF339B009A5178
:10E150006079013A0300C133FF339B009A51023AC0
:10E16000130083401800A123DB00F0500A2001387F
:10E17000C046C046C046C046C046C046C046C0466F
:10E18000C046C046C046C046F1D1100063790024A5
:10E190009840464BF050A920454BC0001B689A643C
:10E1A0001D5844480560100049790196884042494D
:10E1B00000900868A227019EFF00F759009E3E428A
:10E1C00004D0002C0ED00CE0334CB9E70120986449
:10E1D000A920C0001858394F441BA4461400BC4560
:10E1E000E8D9086001229A64A9220026D200985832
:10E1F000334C344A10602268A027A225FF05ED00A9
:10E200007F59009D3D4202D1002E0CD00AE0012230
:10E210009A64A922D2009A58284F161AB4460126A9
:10E22000BC45E9D9226001229A64A922D2009B58F8
:10E23000254D181A0B60254B421E2860244C9A422B
:10E240000DD9244814F080FF2968234814F0B8FE43
:10E2500000232360012023685B001843FEBD0EF0FD
:10E26000BDFA1E490DF076FF1D490DF083FD0EF03D
:10E2700045FA2060EEE7C04641090020420900202F
:10E28000DCE50200038A03008831030014E6020083
:10E2900004E60200428A030024E60200FCE50200D4
:10E2A0003CE60200F4E50200ECE502000C0500008B
:10E2B00068000020C40200202C0A0020C8AF000023
:10E2C000300A0020280A0020340A0020C6AF0000CF
:10E2D00078030020618A03006A8A03000000084274
:10E2E0000000FA44034B82B001AAA0331A6002B0C6
:10E2F0007047C046380A0020014BA43318607047AD
:10E30000380A002010B5034903481AF0AFF9F1F7B5
:10E310005EFFC046FE08000080300300064B07B5D4
:10E320001A00A033A4321B68126801A95B1A9A4232
:10E3300001D8FFF7E7FF07BD380A00200139C9B24D
:10E34000054B401880301970044A03781370044A52
:10E35000D25C044B1A707047440900204509002024
:10E36000479C0300430900200131C9B2054B401806
:10E3700080301970044A03781370044AD25C044B4D
:10E380001A7070474409002045090020479C03008B
:10E3900043090020074B984206D9074B1818074B32
:10E3A0004118C91808787047054B18184118054BD3
:10E3B000F7E7C046A4920000889A03005B6DFFFF58
:10E3C0009C8A03000083FFFF030020228033F0B506
:10E3D00004001A707F2000224F255F2689B0A15CBF
:10E3E000531C0A00DBB202406F2A28D90A003240CF
:10E3F000E11880310A701A007F2BF0D1BB4A1370EC
:10E4000023001B22FF331A70E4320192531CDBB24B
:10E4100003936B46B6481B7BB6490370039BE31816
:10E4200080331B780B705B2B0ED19B22019B0A70F3
:10E430000133DBB20370E254012009B0F0BD5F2A62
:10E44000D6D90A002A40D3E72E2B13D10232D2B2FA
:10E450000270A21880321278A4480270A648825C2A
:10E460000120024206D1019A0B701218D2B2019219
:10E47000A3546FE202209D4A13709F4AD25C104061
:10E4800000D0ADE0002A19D19948203203780A70F3
:10E49000E31880331A70019B0133DBB201936B46A2
:10E4A0001B790370019B782B01D8E25452E29B2325
:10E4B000019AA3546B461B7B0B70BDE716007F25AA
:10E4C00052B2AE430E70002A03DB8C4A8C4B1A60AA
:10E4D000B3E7413B8B4ADBB28B49D25CCB5C120287
:10E4E00013430293029B002101339BB21800029355
:10E4F000FFF750FF0306F5D50123012700267B4DCA
:10E500002B7039000298FFF745FF7B1CDBB22828EF
:10E5100068D1002E00D02F702B780133DBB2059329
:10E5200005990298FFF736FF059B0133DBB22928D6
:10E53000F5D17F25049304990298FFF72BFF049BE4
:10E5400028400133DBB23D284FD16A46694B127B2C
:10E550001870674B00261A706A467B1CDBB200936A
:10E560001278624B039D1A700695631980331B78ED
:10E57000009902980793FFF70DFF079B8342B1D1E3
:10E58000009B05990133DBB20093009A6B1CDBB250
:10E590008A422CD1002E01D0554B1D70039D013FA6
:10E5A000FFB2524B390002981F70FFF7F3FE514E35
:10E5B000030600D504E14E4B7F2118704E4B1B5CC7
:10E5C0001A005BB28A433270002B14DA484B013DCB
:10E5D000EDB21D70631980331B789842DFD081E75C
:10E5E0004A4B7EE71F0001268BE70493A3E71D003B
:10E5F00001260693B9E7307020281BD0232825D0A8
:10E600002E282CD0262832D040284ED05E2856D036
:10E610002B285CD03A2800D00EE1202629002000CB
:10E62000FFF78CFE334A137833401370B7D0304B6A
:10E630001D78F3E729002000FFF780FE0023F35642
:10E64000002B00DA4EE72A4B1D78A8E729002000AE
:10E65000FFF774FE402233781342F4D142E72900D9
:10E660002000FFF76BFE33781B07ECD43AE7290054
:10E670002000FFF763FE1022337813403370E2D19D
:10E680001B4B1B78E118803109783170482900D084
:10E6900028E7013B1649DBB20B70E31880331B7887
:10E6A0009343432B00D01DE7CDE729002000FFF75F
:10E6B00045FE0422337813403370C4D112E7290099
:10E6C0002000FFF73BFE33789B06BCD40AE7084BDB
:10E6D000013DEDB21D70651980352B78452BB2D008
:10E6E00010229343492B00D0FCE6ACE745090020FB
:10E6F0004409002043090020479C0300888A030046
:10E7000070000020CD9C0300B39C0300A592000084
:10E710006B1C934ADBB21370E31880331B7891496A
:10E720000B70452B36D1A81CC0B2231880331B7840
:10E730008D4E33708D4EF656002E02DB884B1D78C1
:10E740003FE010700B70522BF8D0532BF6D0442BB7
:10E75000F4D04C2B08D10335EDB215706519803516
:10E760002B78592BEAD0BDE6462B00D0BAE6EB1C3D
:10E77000DBB21370E31880331B780B70552B00D07D
:10E78000B0E60435EDB21570651980352B784C2B49
:10E79000D4D0A7E6492B00D0A4E6AB1CDBB21370A3
:10E7A000E31880331B780B704E2B00D09AE60335AC
:10E7B000EDB21570651980352B78472BBED091E6E8
:10E7C000069D6A46009B0133DBB200931278664BCC
:10E7D0001A70009B049A934200D19CE019000298A1
:10E7E000FFF7D8FD614B7F211B5C5D4F1A005D4E2A
:10E7F0008A435BB238703270002B08DA0135EDB213
:10E80000631980331B783D709842DAD06AE6307025
:10E81000202816D023281ED02E2826D026282DD0FA
:10E82000402848D05E2851D02B2858D020263A289E
:10E8300064D0252800D16BE74D4A4E4B00201A606A
:10E84000FBE529002000FFF78FFD0023F356002B86
:10E8500000DB73E746E629002000FFF785FD402234
:10E860003378134200D069E73CE629002000FFF727
:10E870007BFD33781B0700D560E733E629002000D5
:10E88000FFF772FD102233781340337000D055E744
:10E890003B78E118803109783170482900D021E6B1
:10E8A0000133DBB23B70E31880331B789343432B77
:10E8B00000D017E642E729002000FFF755FD0422AB
:10E8C00033781340337000D038E70BE6290020007E
:10E8D000FFF74AFD33789B0600D52FE702E60135A6
:10E8E000EDB23D70651980352B78452B00D125E7B9
:10E8F00010229343492B00D0F4E51FE729002000A4
:10E90000FFF732FD174A13783340137000D158E7F0
:10E91000134B1D78F2E700257F272E0000990298FF
:10E92000FFF738FD03003B403D2B04D0019A013234
:10E93000D2B20192A354009A0132D2B201060BD591
:10E94000002E03D06946084A09781170054A1370F1
:10E95000069B0393039A59E500920126DEE7C04621
:10E96000440900204309002045090020479C03007A
:10E97000928A03007000002030B585B003AB05001B
:10E980001400080002AA01A917F0B8FF019A16495D
:10E9900000238A4200D0531002984210884200D1CE
:10E9A0002A00002B15DA5B19D843C0170340002A50
:10E9B00013DA52192360934200DA13006360039B59
:10E9C0008B420ED0032B0CD000205B10A36005B04F
:10E9D00030BD9D42EBD22B00E9E79542EAD22A00F6
:10E9E000E8E70120A060F2E7D0DB0200F0B5060006
:10E9F00085B017001B2805D10A9A974209D000203C
:10EA000005B0F0BD19281AD01C281AD00A9A0A9706
:10EA100017001A000B0011000A9A0192BA4200D99D
:10EA200001971D000C0000230093009B019A934264
:10EA300009D10A9BBB4220D0E1D30120E0E71A268E
:10EA4000EAE71D26E8E70295039401CD02CCF3F72F
:10EA500075FE002802D0009B0133E5E71B2ECED0C7
:10EA6000039B30001A68029B196801F0D5FA044B29
:10EA7000C01A43425841C0B2C2E71A2EDDD1BEE7E8
:10EA800044240300F0B51E0085B0039018680D0003
:10EA90001700F3F7BDFD7368019002930024022F65
:10EAA0000ED90123B2682900F3F772FF0400032F87
:10EAB00006D029000123F2680198F3F769FF0500E9
:10EAC000A54205D80A490B4819F0D7FDF1F77FFB9D
:10EAD000039AA3000299D058F3F730FE002801D121
:10EAE0000134EDE701206400204305B0F0BDC046CD
:10EAF000E79C030000320300F0B50D00002785B04D
:10EB0000110003901E0028000F4B0222009700F016
:10EB10001DF8A81C800017F0A8FC039B04000360EC
:10EB20006B1E3D000393436033688360039B9D42EB
:10EB300002D3200005B0F0BD0135AF00F05901F05F
:10EB4000DFF9E719B860F1E7FFFF000010B51C001E
:10EB500002AB1B78002907D0002B05D10F491048C4
:10EB600019F08BFDF1F733FBA24207D1824213D09B
:10EB700003000C490A4807F0D5F9F3E7824205D9AA
:10EB8000121A0949064807F0CDF9EBE7844203D28F
:10EB9000030022000549EDE710BDC046FE9C0300BE
:10EBA00088310300E3800300279D0300599D030083
:10EBB000F0B50025170087B00C9C0D9E03900491C2
:10EBC000059302950195059B9D4208D1019B039AEF
:10EBD000934241D22449254819F04FFD26E0039B7A
:10EBE0009D4211D263689B05F4D4019B049A0133C2
:10EBF0000193AB00D058FF2263681340012B22D150
:10EC0000F3F72CFF307015E023680022D9000623AB
:10EC100038001943FDF700FB00280FD16368DB05BE
:10EC200006D522681249114807F07CF9F1F7CFFAAE
:10EC3000A368336001350C340436C4E7029B406896
:10EC400001330293D7E7022B03D1F3F7C9FD3060FC
:10EC5000F0E7032BEED1FAE73B68029ADB0805499F
:10EC60009A42B8D307B0F0BD9F9D030088310300DE
:10EC7000889D0300C09D0300014B58687047C04643
:10EC8000380A0020014B18687047C046380A002037
:10EC9000F0B5194E87B03368050000200C000193D1
:10ECA00015F0DEFC30600090206817F0AFFF019B8C
:10ECB00007003360114E022D03D0A068F3F7A8FCC3
:10ECC0000600210063680831A81E0393F8F79EF838
:10ECD000009B04900593002203AB0321300001F058
:10ECE00015F8074B04009F4203D00100380019F0CB
:10ECF00091FB200007B0F0BD380A0020503503001A
:10ED0000D0DB0200F8B50326050007003540022DD0
:10ED100016D10E4B0340062B12D0FF23DB05C4187F
:10ED2000B443201C00210CF043FD002806D08023B2
:10ED30001B06E418B443064B2C43E7183800F8BD13
:10ED40003800F9F735FD0700F8E7C046070080FFF7
:10ED50000000808010B501F0D3F80400200001F01D
:10ED60001BF9002801D1044810BDF3F777FE0028F5
:10ED7000F4D10248F8E7C046442403003C240300D1
:10ED800010B501F0BDF80400200001F005F90028DD
:10ED900001D1044810BDF3F761FE0028F4D0024809
:10EDA000F8E7C0463C2403004424030007B5044BA5
:10EDB00001900022694602200093F5F7AFFC0EBDDA
:10EDC0000604000010B5F3F7A7FC034B002800D1A0
:10EDD000024B180010BDC046442403003C2403002D
:10EDE00037B5F3F7FDFC01AB7F2806D80121187079
:10EDF00001221800F4F78EFA3EBD1F4982098842AD
:10EE00000BD8402149420A431A703F220240802019
:10EE10004042104358704231EAE7184C010BA042BF
:10EE20000ED8202464422143197080215F34494266
:10EE3000224020400A43014399705A700321D7E7CA
:10EE40000F4CA04212D81024850C64422C431C7035
:10EE50003F258024294064422A4028402143224300
:10EE6000204359709A70D8700421C1E705490648BB
:10EE700019F003FCF1F7ABF9FF070000FFFF0000FA
:10EE8000FFFF1000DE9D03000032030010B50200FA
:10EE900002490A2001F0C0F810BDC046BE040000BF
:10EEA00010B5020002490A2001F0B6F810BDC046B4
:10EEB0003E050000F0B585B0019202900D000022E1
:10EEC000314901980393FDF7A7F90090002801D07C
:10EED00043680093029B012B10D00026340001965A
:10EEE000029B9E421FD0009B002B3DD12F68002C1F
:10EEF00040D12C68019701360435F1E700242868D9
:10EF000000F0FEFF27000290029801F045F8051E70
:10EF10000CD1002C07D122001C490198FDF77CF987
:10EF200000281BD04468200005B0F0BD009B2E00D7
:10EF3000002B04D02900180017F06FFE0600002CEB
:10EF400009D03A003100039801F066F8104B98425E
:10EF500001D025003E002C003700D5E70D490E48B2
:10EF600019F08BFBF1F733F92968009817F055FE7B
:10EF70000700BCE7019A3900039801F04DF8044BF3
:10EF80009842B8D1B5E7C046D60600001E0500007D
:10EF900044240300FF9D03000032030037B501A99C
:10EFA0000500F4F765FE1E4B04002B40062B05D030
:10EFB000AB072AD11B4B2A689A4226D1019920001F
:10EFC00015F0B2FA0190012822D1207843B2002B2B
:10EFD00004DB012023785B0018433EBD7F2301340E
:10EFE00018403F3B034208D13F2223781900914348
:10EFF000802905D016F0E1F8EFE798435B10F1E7C0
:10F000008001134001341843EFE7019B012BE0D04E
:10F01000019A0549054806F085FFF1F7D8F8C04682
:10F02000070080FF84320300189E0300883103002C
:10F03000F0B5140087B0029003910022234920000C
:10F04000FDF7EAF80022050021492000FDF7E4F869
:10F0500001230400049305931E4F002D07D0686818
:10F060001D4B984203D004A9F4F702FE07001B4E83
:10F07000002C07D06068184B984203D005A9F4F71C
:10F08000F7FD06000024029B154D9C420AD1002387
:10F09000059A0193009331002800FDF79BFF0E486D
:10F0A00007B0F0BD002C07D00023049A0193009311
:10F0B00039002800FDF78EFF0399A3000022C958EC
:10F0C0002800F3F7BDFA0134DDE7C046EE05000085
:10F0D000F60500008C850300D0DB020049490300DF
:10F0E000F81003007FB50D4D0400A84213D00C4E5C
:10F0F000012201003000F3F7A3FA0A49300017F0AB
:10F10000E8F904230293084B0394DB6902AA032164
:10F11000064801939847280004B070BDD0DB020078
:10F12000F810030049490300082B0300C817030027
:10F1300010B5040086B06A4602A8102107F0ECFE64
:10F14000012221006846F3F77BFA02A90248F4F78E
:10F15000ABF806B010BDC0468432030070B50C6831
:10F16000E30726D4A30703D1254B22689A4220D077
:10F17000012820D94868F3F733FB06002000F3F795
:10F1800093FB051C30000DF0D9FA011C1D480FF04F
:10F1900079FF011C041C281C0CF0DCFF0FF01EFC86
:10F1A000211C0CF0E7FD032302249843164B044373
:10F1B000E418200070BD2000F3F776FB051C0FF06B
:10F1C0000DFC061C0DF09AFA311C0400281C0DF0F1
:10F1D000E1F8FC218905051C0CF0E4FA002803D0B5
:10F1E000013401239C4306E0BF21281C09060CF0D2
:10F1F000D9FA0028F5D1200015F0DFFF0400D8E788
:10F20000A0F00200000020410000808013B504003F
:10F210000800F4F7A1F86A460100200000F0F4FDB0
:10F22000009B0248002B00D1014816BD4424030076
:10F230003C24030037B50024022800D98C684868B4
:10F240000D68F4F789F80A4B0100002C00D0094B37
:10F2500028006A4698470098002806D001990400C3
:10F26000002902D0FCF7CAFF040020003EBDC046C2
:10F2700069FE000009FE000070B5040008001500DA
:10F28000F4F76AF82A000100200000F015FE01489A
:10F2900070BDC046D0DB020010B500F057FE00285C
:10F2A00004D1034819F0DCF9F0F791FF10BDC04616
:10F2B000C830030030B50B0085B01400012805D913
:10F2C0000A490B4819F0D9F9F0F781FF09480121E3
:10F2D000C2680192019D0022A8472200039003A961
:10F2E0000120F6F7B3FA039805B030BD529E030033
:10F2F00088310300C0E90200F8B50E0000280FD1E4
:10F300000400294B1D680021080015F04AFD002764
:10F310000600002D34D10025002C40D13000F8BD6E
:10F320000868830715D10268204B9A420DD119F065
:10F33000A9F805003068F3F76BF91D4BC26800248B
:10F340009A42E0D134680434DDE71A4903008A4266
:10F3500002D0F3F75DF903009D6B002DEAD0164B48
:10F360002A689A42E6D00025E4E7EA68FB0099584B
:10F37000002904D0042902D03000F6F705FA01373D
:10F38000AB689F42F1D3C6E7A268EB009958002909
:10F3900004D0042902D03000F6F7F6F9013563688D
:10F3A0009D42F1D3BAE7C046380A0020082B03007B
:10F3B0007D6A01005035030084DE020010B5034869
:10F3C0000968F3F761F9024810BDC046F810030060
:10F3D000D0DB0200F7B50125284B070001911D7015
:10F3E000F3F7FEF9102805D02549264819F045F90C
:10F3F000F0F7EDFEA1220021234BD200A226995066
:10F400000922F6009A51802080228000D2021A50F0
:10F410001E481F4C1950A9211F20C9005850C12156
:10F4200089005A508023C022C220DB005200A35022
:10F430008000225817491140C02212040A4322506A
:10F44000C0225200A35038002360F3F7C9F903002B
:10F45000A0220C21C133FF339B00D20599504023D9
:10F46000C12223600C4B000218430C4B92009851B0
:10F470009D500B4B019A0B481A60FEBD9A0B002061
:10F48000839E03008831030000A0004004050000B3
:10F4900000E100E0FFFF00FF01000200006000400B
:10F4A000D0090020D0DB02000B4B0C481A68C16C5D
:10F4B000013210B51A600A4B012907D1C124A400FA
:10F4C0001C59640302D50024C464D960C82A02DD33
:10F4D00001225A60DA6010BD84030020FCA00040C5
:10F4E00000A00040F7B5474B5A680193012A22D18A
:10F4F000C12345499B00CB5813421CD0434C444D7B
:10F5000023683C2B09DD002342490B8042494A60B5
:10F51000CA60424A23602B7013702B78002B0BD1EA
:10F5200001223D492A702360CA600A603C4A136088
:10F530000023019A5360F7BD3A4E226833783A4F60
:10F540000133337000230D2A35D1337023603349E2
:10F55000314B0C3A0A70DA603B78012B06D13278D5
:10F560003249013A93400A6813430B603378202BE9
:10F57000DED1002301212E4A1370274A5160D16049
:10F580002A4A23601068234C010C218029492B70E2
:10F59000088080B2136015F010FE274D2860208887
:10F5A00015F00BFE254B02001860254B29681868E2
:10F5B00017F03BFBBCE7012A04D117492360CA605E
:10F5C0003B70C9E7022A04D123600123124AD360A9
:10F5D000F6E70B2AC0D101210F4A23605160D160A8
:10F5E000134A2B7013785B18DBB21370052BB3D959
:10F5F000124B1A68104B1968114B186817F015FB5D
:10F60000AAE7C046FC600040006000408403002080
:10F61000490900202209002000A0004047090020DD
:10F6200080030020460900204A0900207C030020B6
:10F630004809002020090020840B0020880B0020AE
:10F64000D0090020F7B5CC1CA400070020000E0054
:10F65000019216F00AFF22000500054B4760866004
:10F6600003600C3A01990C301DF07FF82800FEBDB4
:10F67000A01B0300F8B5224E3568686801281DD923
:10F68000AA68431ED15C0A2918D1002B03DD591E3C
:10F69000545C0A2C13D11C00844202D2115D202933
:10F6A0000FD0002B0FDC1218023AE31A14789B08D3
:10F6B0003A3C614261415C18002C11D1F8BD0B004D
:10F6C000E3E70134E8E7611C8842ECD1591E0029C8
:10F6D000E9D00139575C0A2FF0D0202FF7D0E2E7AC
:10F6E000084F04223900280019F0B4FD0421380025
:10F6F00004F086FB3369013C04333361DCE7C04628
:10F70000880300208985030010B5202200210248CB
:10F710001DF046F810BDC046800A0020084B10B509
:10F72000426818600020986018750138D860080099
:10F730005A601A61996118F06FFEFFF79BFF10BDC8
:10F7400088030020F8B503780400002B1DD00F4E6D
:10F75000B06C002804D021001DF07EF9002814D0E0
:10F7600020001DF083F9471C380016F08BFE051EA3
:10F770000BD03A0021001CF0F8FF054B054A196830
:10F78000043B99609A42FAD1B564F8BD380A00206A
:10F79000980A00207C0A0020F0B5B64C06002068CC
:10F7A000A568436885B00193002D00D010E1731E59
:10F7B000042B0AD819F0B7FD6368984200D1A3E082
:10F7C000012E00D140E1022E10D0032E00D19BE08B
:10F7D000042E13D1206821694368994200D32AE19D
:10F7E000012219F038FE0025012726E1236962680D
:10F7F000934200D94EE10126764285E0052E00D1E4
:10F800000EE1062E0FD123685D682369AB42AD413E
:10F810006D42002DEFDD2368290098682369C01828
:10F8200004F0EEFA20E00B2E22D1019B2269206821
:10F83000991A19F004FE2368019A5B689A4204D968
:10F8400013002269981A04F013FB22682369516897
:10F850009068C91AC01804F0D3FA2368586823695D
:10F86000C01A401B04F0F2FA23695D192561C2E752
:10F870000E2E13D1E368002BBDDB2068013BE36053
:10F8800062684368991A19F0DAFDE368002B17DB08
:10F890001233794A9B00995820680FE0102E16D138
:10F8A000E368062BA7DC5A1C734913339B00595895
:10F8B0000029A0D020686368E260436019F07FFDF2
:10F8C00063682269D61A22685568ED1A0BE0152E76
:10F8D0000DD12369626861689A1A206819F0BBFD2E
:10F8E000236962689E1A0127002E30DCA3E70D2EE3
:10F8F0000DD1624818F090FD206819F046FD63684C
:10F900000026C018FFF71EFF300005B0F0BD012330
:10F910001B2E66D0082E01D07F2E21D1216962686E
:10F92000914200D867E7002320688668B618F75C24
:10F93000202F13D101339F188F42F8D30126032BB8
:10F9400000DD0336891B320019F085FD01273000E8
:10F9500004F07CFA23699E1B26617FE00126F1E713
:10F96000092E29D163682269D11A22689068444A15
:10F97000C01803AB04F0A0F8061E00D13BE7002737
:10F98000431C0BD1A06918F047FD63682269D11AA6
:10F9900022689068C01804F033FA4CE723692068A5
:10F9A000F918039B01375A1C03921A7819F035FD98
:10F9B000BE42F3D135003EE73300203B5E2B00D939
:10F9C00019E732002169206819F030FD012532E77E
:10F9D000012D08D104234F2E03D002235B2E00D02B
:10F9E0000023A36007E7022D21D13300303B092B10
:10F9F00003D803232675A360FDE60023A360412EF0
:10FA000000D14DE7422E00D134E7432E00D1FAE673
:10FA1000442E00D1EAE6482E16D0462E00D0EAE663
:10FA2000002723683E005D682369ED1A11E0032D6D
:10FA300028D17E2E03D000252F002E0009E0237D43
:10FA4000312B01D0372B0DD100252F00236962689F
:10FA50009E1A0023A3609E4200DD78E7002F00D1AC
:10FA6000D7E6E8E61A00FB21343A0A42D8D0332B15
:10FA7000E1D1AFE688030020380A0020484903009E
:10FA8000F81003000023042DABD1462EC8D0482E19
:10FA9000DAD0A6E7002501262F0058E7F0B50E00C2
:10FAA000002485B011000700039322000C4B3000A6
:10FAB0000094FFF74BF8B01C800016F0D6FC050050
:10FAC00007604660B44202D1280005B0F0BD039B38
:10FAD000A700D85900F014FAEF19B8600134F1E723
:10FAE000FFFF000070B5F9F749FE0B4C002623001C
:10FAF000A8331E60266304F043FF084D012128004F
:10FB0000F2F74EFB28005E226E2114F0E1FD6560E5
:10FB10002560666470BDC046380A00206C0A00206B
:10FB200070B50624134EC3001C4373680022050001
:10FB30002100181DFCF770FB021E18D1706C002804
:10FB400007D004302100FCF767FB002801D0406893
:10FB500070BD002221000848FCF75EFB021E06D1A2
:10FB60002A000649064806F0DDF9F0F730FB506838
:10FB7000EEE7C046380A0020D8170300969F03001E
:10FB8000902F03000A4B10B5040018685B68984278
:10FB90000AD00621E300194304300022FCF73CFBA5
:10FBA000002801D0406810BD2000FFF7B9FFFAE738
:10FBB000380A0020074B10B5586C002801D10648C0
:10FBC00010BD043000222621FCF726FB0028F6D0C9
:10FBD0004068F5E7380A0020541603000A00C10007
:10FBE000062010B5024B0143186814F071FD10BDDA
:10FBF000380A0020062110B5034BC00001431868E5
:10FC000014F070FD10BDC046380A00200A00C10083
:10FC1000062010B5024B0143586814F059FD10BD81
:10FC2000380A0020062110B5034BC0000143586874
:10FC300014F058FD10BDC046380A002070B505000C
:10FC40000C00062806D10800F2F708FF00280ED0A5
:10FC5000274870BD012001421AD04B10042D08D056
:10FC6000052D13D00800002DF3D1002BF0D0214832
:10FC7000EFE7C0221206934204D18020C00515F0A0
:10FC80009CFAE6E75B425B001843E2E7DB43FAE7F6
:10FC9000022D12D1184B0B40062B08D08B070CD12C
:10FCA0000A68164B92699A4207D1486802E0C80870
:10FCB00015F088FC43000120E6E72000F2F7A8FCDD
:10FCC0004369002B0DD10E4BAD002000ED5814F010
:10FCD00078FD2A0003000B490B4806F023F9F0F7E2
:10FCE00076FA2100280098470028B2D1EBE7C046F9
:10FCF0003C24030044240300070080FF2942000045
:10FD00008C35030022A0030088310300F7B50400FE
:10FD1000019116001F00F2F77BFC0569002D09D147
:10FD2000200014F04EFD06490200064806F0FAF8DD
:10FD3000F0F74DFA3B00320001992000A847FEBDC4
:10FD4000299F030088310300F8B504000D00170057
:10FD50001E0000290BD01868F2F75AFC636898421D
:10FD600005D00649064818F088FCF0F730FA330051
:10FD70003A002900A068FFF7C9FFF8BD959E03006F
:10FD800088310300F8B506000F0014001D0093072A
:10FD900014D11368174A934202D163682B60F8BDEF
:10FDA000154A934207D1002802D0F2F731FC070030
:10FDB000636888C5F3E7114A934201D12C60EEE7EE
:10FDC0005B681A00F23A012A01D9F02BF6D1002E15
:10FDD0000ED12000F2F71CFC094B984208D10C20F0
:10FDE00016F043FB074B4760036084602860D6E74A
:10FDF00050C5D4E7D83403009C34030050350300C9
:10FE000024F00200241C0300F8B5002313605360A3
:10FE100006000D001400F2F7FBFB0700102D05D1C2
:10FE2000836A002B02D00F4B48C4F8BDFB69002B3E
:10FE300004D02200290030009847F6E7B86B00286C
:10FE4000F3D00621ED00294304301A00FCF7E4F951
:10FE50000028EAD04268230039003000FFF792FF03
:10FE6000E3E7C0465017030070B5160004000D000C
:10FE7000FFF7CAFF3368002B15D10B4EA3070BD138
:10FE80000A4B22689A4207D12B0062680849300069
:10FE900006F048F8F0F79BF9200014F092FC2B00D4
:10FEA00002000449F3E770BD9C2C030050350300A9
:10FEB000AF9F0300D69F030073B504000D0016002A
:10FEC000F2F7A6FBC369002B09D004220196009229
:10FED00029006A4620009847009B002B0AD020008A
:10FEE00014F06FFC2B0002000349044806F01AF8D6
:10FEF000F0F76DF973BDC046D69F03009C2C03003C
:10FF000013B50400F2F784FB436A002B11D16A4653
:10FF10001A212000FFF778FF009B002B0ED1200054
:10FF200014F04FFC07490200074805F0FBFFF0F70B
:10FF30004EF9200098470028E9D016BD6846FBF727
:10FF4000FDFDFAE7459F03008831030037B5040043
:10FF5000F2F75EFB856A002D02D02000A8473EBD67
:10FF60006A4610212000FFF74FFF009B002B05D0B1
:10FF70006A462900280016F061FEF0E7200014F020
:10FF800020FC03490200034805F0CCFFF0F71FF9FD
:10FF9000779F03008831030030B505008FB0FEF76E
:10FFA000BDF92800F2F734FB846A002C05D0280044
:10FFB000A047040020000FB030BD6A461021280081
:10FFC000FFF722FF009B002B16D002A8F0F7E4F801
:10FFD000002807D16A46010016F030FE0400F0F751
:10FFE000F1F8E7E7039B0949186806F00FFF0028BE
:10FFF000E0D10398F0F7EBF8280014F0E2FB044995
:020000040001F9
:100000000200044805F08EFFF4E7C046C830030044
:10001000779F030088310300F0B585B003900F008F
:100020001600202804D1914210D0B14805B0F0BD8F
:10003000039B1B2B01D01E2B0DD131003800F2F792
:100040007DFB039B002803D01B2BEED1A948EDE7D5
:100050001B2BFBD1E9E7039B212B28D1100005F0D6
:10006000A9FF002806D03100380018F010FB002846
:10007000ECD1DAE70324344000D05EE19E4B3268D5
:100080009A4200D059E173689C42CED2A300F31883
:100090009D68280005F08EFF002800D14CE1290062
:1000A000380018F0F4FA0028D0D10134EBE701232E
:1000B000194200D1FCE013404D100293002B00D1F7
:1000C000EEE0039B54101D2B00D936E118000BF015
:1000D0009FF91E0028002A002D0047004E00510005
:1000E00053005E0067007D008500BA001E002800F6
:1000F0002A002D0047004E00510053005E006700AB
:100100007D008500D300D7003401DB00DF002543EC
:100110000295029B5C00634000D5BDE001202043B6
:1001200084E76540F4E72C400294F2E7002C04DAFF
:100130007249734818F0A1FACFE01F2C08DC714B0C
:1001400023419D4204DCC0231B0623419D4205DA66
:10015000E917280015F022F807004BE0A540D7E783
:10016000002CE5DB1F2C00DD1F242541D0E72B19D7
:100170000293CEE72B1BFBE721002800F2F7A8FF34
:100180000028E5D1012065436D0028434EE7002C8F
:1001900000D1E5E02100280014F0ACFB0290B8E7A4
:1001A000002C00D1DCE028000CF0C8FA051C20006F
:1001B0000CF0C4FA011C281C0BF0DCFD0323050025
:1001C00002209D43504B2843C0182FE7002C00D13C
:1001D000C6E02100280014F07DFBDFE72F00002C93
:1001E0002EDA28000CF0AAFA032302279843464B84
:1001F0000743FF183800F2F70BFA8369002B00D190
:100200009BE03200390003989847002800D00DE7A2
:1002100093E001231C4208D039000298F2F758FFFE
:10022000002895D1029B7B430293012C00D170E7FB
:10023000390038006410F2F74BFF002888D17F4363
:10024000002CE6D165E7002C00D189E000210220D6
:10025000F6F7DCFD21000600280014F04BFB012717
:1002600040003843B0602100280014F033FBB84050
:100270000743F7603000D9E6A54200DAE6E6D4E6A7
:10028000A54200DDE2E6D0E6A54200DCDEE6CCE6F3
:10029000A54200DBDAE6C8E6029814F08EFFC5E658
:1002A00003231340022B03D1184B1340062B5AD1C2
:1002B000039B1F2B9ED13000F2F7AAF9836904003B
:1002C000002B0CD1636A002B26D1300014F079FA90
:1002D0000F4902000F4805F025FEEFF778FF3A00BE
:1002E000310003989847002800D09FE6EAE7C0460F
:1002F0003C2403004424030090EC02005855030002
:1003000000320300FFFFFF3F00008080070080FFF6
:10031000459F0300883103003000FFF7F1FD040022
:100320002000FFF739FE002800D17EE63900F2F701
:1003300005FA0028F4D089E62E00039B38009A00C5
:100340000D4BD45814F03DFA0500300014F039FA82
:100350002B00009022000949094805F0E3FDBCE7A5
:1003600008490948E6E628000CF0E8F93200011CCB
:10037000039805F067F848E7FC330300049F030087
:10038000883103004755030048320300F0B5136875
:100390008DB00693002800D06CE00400131D039379
:1003A000FF220B00090A1340114001934B000593F3
:1003B000059A019B04919B18039A9B00D558D3186A
:1003C0005F68381E09D00020BB0706D1844B3A680D
:1003D0009A4202D1380014F078F9049B1E18002DBF
:1003E0004DD1019B76000133F3189800009316F06D
:1003F0003CF825000600002C01D001250460019B7B
:10040000A8009A00301803991CF0AFF9019B5B1902
:100410000293029B9800049B3018DA00019B99001C
:10042000039B59181CF0A1F9029A059B944663445A
:100430001C00002F0FD003253D4000D09CE0684BEE
:100440003A689A4200D097E0380014F054F94168B5
:100450008D4200D07FE0029B0299E21A52083300DD
:100460000698FFF753FC0400300016F025F8200032
:100470000DB0F0BD130008330393546890E7AB0749
:100480002FD12B68574A934202D0574A934228D122
:1004900028000AAA09A9F2F745FA099B019A013333
:1004A0009B1876009B199800009315F0DEFF25003D
:1004B0000600002C01D001250460019BA8009A00D1
:1004C000039930181CF051F9019B0A995819099B9E
:1004D00080009A0030181CF048F9019B099A9B187B
:1004E00095E7019B7600181D33189800009315F0CE
:1004F000BCFF02940600002C02D00123046002938A
:10050000029B03999800019B30189A001CF02DF96A
:10051000019A029B9446280063440293FFF7F0FC83
:10052000029B07909C000798FFF736FD051E00D13F
:100530006FE7009B029A934207D8D900300015F06C
:10054000AAFF0600009B5B000093029B355101331C
:1005500002930434E7E78368EF00DA59002A09D0F0
:10056000042A07D0A300F2508268F318D219526807
:1005700002345A6001356BE70AAAC5213800FFF73B
:1005800073FC00210AAA080016F058FBFFF7B8FC1C
:10059000A50001900198FFF7FFFC071E00D15AE764
:1005A000009A631C9A420BD853000093042B01D28B
:1005B00004230093009B3000990015F06CFF0600A7
:1005C00009AA02213800F2F7CFF9099B02341B680F
:1005D0007351099B5A6873195A600835DAE7C046A7
:1005E00084DE020090EC0200C0E9020073B50C004A
:1005F000150083071ED10368204A934207D0204A82
:10060000934217D101AA694614F0E2FB03E001AA64
:10061000694614F036FC009B9C4228D817D3019BF6
:10062000A4001C19043B043C9C4200D173BD226809
:1006300004C5F8E7FFF764FC002306000093009B65
:100640003000A34206D3FFF7A7FC0028EED022001B
:100650000C490EE0FFF7A0FC002808D0009A0A49D8
:10066000A31A5B189B00013258510092E7E7009AE9
:100670000649074805F056FCEFF7A9FD90EC02008B
:10068000C0E9020063A00300FFFFFF3F40A003009A
:1006900000320300F7B514000A0AFF230E0015000C
:1006A0001E401D4083073BD107683D4B9F4208D049
:1006B0003C4B9F4234D1FF231143194224D1206087
:1006C000F7BD01AA694614F0DCFB009B72199A423F
:1006D0005ED89A009446002001998200A84218D161
:1006E0009B1BB5004919181AA41814F05AFB019B5A
:1006F00020605D190023013601339E42E0D09A004C
:1007000051426958A150F7E701AA694614F060FB0D
:10071000DBE76746BF1A043FCF590130A750DCE73B
:10072000FFF7EEFB002307000093009B9E4217D8C3
:100730000021080014F035FB06003800FFF72CFC00
:10074000011E1AD1B1688D4222D8AB00E3181E6099
:1007500088009C4215D1491B300014F03EFBAFE7E6
:100760003800FFF719FC002812D0009AB31A5B1961
:100770009B00013218510092D7E73000F5F704F8DA
:10078000DBE7F268C71AA218D259043B1A60E0E707
:10079000009A0549054805F0C5FBEFF718FDC0466E
:1007A00090EC0200C0E9020040A003000032030008
:1007B000F0B587B01D0006000C000192F1F728FF8C
:1007C0002E4B984207D12B00019A2100300002F0F5
:1007D000D9FD07B0F0BD876A294B002F08D09C4295
:1007E00021D13000B84728600028F2D00120F0E77E
:1007F0009C4218D103AA10213000FFF705FB039B90
:10080000002B0CD103AACD213000FFF72DFB05945E
:1008100003AA0021012016F011FA2860E6E703AAD6
:1008200039003800F7E7002CECD1019B2000002BA9
:10083000CFD01800F1F7ECFE124906F0E7FA0028D5
:100840000FD003AACC213000FFF7DEFA039B002B68
:1008500007D003AA2100200016F0F0F9286020003C
:10086000B7E703AACE213000FFF7CEFA039B01AA17
:10087000002BCED1019B02202B60AAE77425030038
:10088000D0DB0200A42D030010B5040005F092FB9C
:10089000002808D0002320001A001900FFF736FABC
:1008A0000400200010BD200017F0EBFE0028F8D156
:1008B0000249034817F0E1FEF2E7C046F89F030043
:1008C000883103007FB5C30006201843054B019013
:1008D0000491052001A9029303930592FAF7A0FF62
:1008E00007B000BDD0DB02001423F0B58DB000AF1F
:1008F000FA1805000C00FFF787FABB69002B06D039
:1009000022002C492C4805F00DFBEFF760FC7869BC
:1009100000284BD1280015F0A3FB0028F0D01423A9
:100920002800FA180D21FFF76FFA10237869F918DB
:10093000F3F79EF9B860200014F049FE6A463E695C
:10094000B968731C7B60C318FB600E33DB08DB00E7
:10095000D31A9D46320068461BF007FF6D462E23D2
:10096000AB557B682000EB18BB6014F035FE060029
:10097000200014F02CFE31000200B8681BF0F5FED8
:10098000F9686846F8F738FFC300062018430B4B98
:1009900010223B627B620A4BBA18BB620123FB62E6
:1009A0000B33F861D1180520FAF73AFFBD460DB0B8
:1009B000F0BDC046619F0300E02D0300D0DB0200C4
:1009C00044240300F0B5174C0F00616895B0039103
:1009D0002168060008A8049162602360EFF7DCFB41
:1009E000051E06D0039B09986360049B2360EFF704
:1009F000EEFB33683A00310005A80193F0F73CFAAA
:100A00002B002A00019905A801F0ECFB16F0FEF876
:100A10000500EFF7D7FB2800039B6360049B23606E
:100A200015B0F0BD380A002010B50400F0F7B6FE8E
:100A3000031E064804D0064917F01FFEEFF7C7FB58
:100A40002200044905F06EFAF8E7C046542F03006F
:100A5000AD9E0300D69E0300010010B5024817F0BA
:100A60000CFEEFF7B4FBC046CC2F030010B5437962
:100A7000012B03D1C06A13F0D3FE10BD0B00C26A74
:100A80000249006B13F008FFF7E7C046A0330300EC
:100A900010B54379012B03D1C06A13F0E1FE10BDFC
:100AA0000B00C26A0249006B13F0F6FEF7E7C0467E
:100AB000B033030010B54379012B03D1C06A13F0A2
:100AC000CFFE10BD0B00C26A0249006B13F0E4FEBA
:100AD000F7E7C0469033030010B5024B3F2216F0F3
:100AE0006EF910BDAF77020010B5024B912216F0DF
:100AF00066F910BD4D1C0100F7B50F0011001A007A
:100B0000C38AC579868A019300230400C371838256
:100B1000C382104B16F053F9A368002B18D1E18A59
:100B2000002908D0A38A002B05D1206B18F036F9D4
:100B3000206B17F0C6FFA38AE28A3900200016F066
:100B4000EEF86B1E9D416B469B88E571A682E382A1
:100B5000F7BDC0465D180100836870B504000D0044
:100B6000002B09D11100054817F087FDA060200077
:100B700029000C3016F08AF970BDC046043103001C
:100B8000F0B58DB06B4601921B79040043710123CF
:100B9000E16203610B780D00012B06D00021954A1C
:100BA0002000FFF7D9FF0DB0F0BD019B012B07D945
:100BB000836B0A001E68030001990833406BB0473D
:100BC000AB681800049313F023FC63790490032BA3
:100BD0000FD109900C2109A813F033FCA36B02007C
:100BE0009B680999606B9847A3686883002B00D0C5
:100BF000BCE0049813F00CFC04900378002B3AD06E
:100C00000A3B0F2B32D809A916F05DF8099B772B08
:100C10002AD006D803220292312B08D0764A0499B2
:100C2000BEE7812B1DD002220292992BF6D10498A7
:100C300013F0EEFB5A21049004A813F002FC049D6B
:100C40000390039B9D4218D16379012B04D9A36BB8
:100C500002995B68606B9847A368002B00D085E021
:100C6000A1E701230293E2E70023FBE70100634AC7
:100C70002000FFF771FF0223F4E704952B78432B44
:100C800004D1280013F0C4FB0500DAE7392B01D0AA
:100C90005B4AC4E705A9280013F0C4FB03780600EB
:100CA000912BF5D113F0B4FB059B9842F0D105A927
:100CB000300013F0B7FB037807000A3B0F2BE7D88F
:100CC00013F0A6FB059B06009842E1D00378A02B09
:100CD000DED113F09DFB059B9842D9D106A93800BF
:100CE00015F0F1FF300013F098FB9C21079007A846
:100CF00013F0A7FB0100079813F07EFB069B06008C
:100D00002E2B1BD1012804D1079803780A3B0F2B07
:100D100001D93C4A83E72669731C2361019B012B9F
:100D200021D909A915F0CFFFA36B099ADB6831001F
:100D3000606B9847002816D1334A70E72F2B1BD1E0
:100D4000012803D107980378032B01D02F4A66E7C7
:100D5000019B012B07D9A36B676B1E6913F038FB4E
:100D600001003800B047A368002B8AD02000049906
:100D70000C3016F08BF816E7302B23D1012803D95D
:100D800007980378032B01D0214A48E7019B012BE8
:100D9000E9D908A913F00DFB0127079007980378FC
:100DA000032B01D01B4A3AE709A913F002FBA36BFE
:100DB00007905B69099A0899606B01379847BE42B2
:100DC000ECD1D0E7019B012BCDD9032800D95FE7F7
:100DD000079B1800099313F01BFB0A9013F018FBF4
:100DE000A36B0B909F69320009AB0699606BB84703
:100DF000B9E7C046B0A20300D4A20300E1A20300F9
:100E000009A303002CA3030048A3030058A3030075
:100E100074A3030099A3030010B5024AFFF79CFED8
:100E200010BDC046BBA303007FB50B7804000D00C6
:100E30004E1C002B0AD0032B0BD103A9280013F062
:100E4000B8FA03990600206B17F0D2FD300004B009
:100E500070BD012B07D18E1C49780529F6D0006B97
:100E600005F0D4FBF2E7042B0BD14B788978006BAB
:100E70000902194317F004FE280013F0C9FA06000E
:100E8000E4E7052B15D14379042B04D02A49006BE4
:100E900017F002FEF0E788784B780002184303A9A8
:100EA00014F09FFB0399246BF2F74CFA0100200029
:100EB000EEE71A000A3A0F2A09D803A9280015F00C
:100EC00002FF039906002000FFF7D0FDBEE7082BC4
:100ED0000CD103A9280013F062FA039B226A9B003D
:100EE00006009958206B17F0D7FDAFE703AB02AAB5
:100EF00001A9280013F0BDFA02990500206B05F046
:100F00003BFB019B0D4A9B009B58002B06D10C4AD2
:100F100029002000FFF720FE039E97E7039A29008F
:100F200020009847A368002BF6D0E368002BF3D18C
:100F3000029BE360F0E7C046D0DB0200601C0300C8
:100F400001A20300F0B587B000920A000493531E7B
:100F50009A410D00060004990098059213F04CFA8E
:100F60002C1E019009D02B780024842B05D102007F
:100F70002100306B17F090FF2C00019B009F013B7C
:100F80000393059B0293049B9F421ED1002C39D1F1
:100F9000019A059B944663441900306B17F070FF6B
:100FA000002D3CD1009B9F422AD0009B9C4239D10E
:100FB000200013F032FA00220100300000F038F86F
:100FC000009813F025FA0090ECE73B78842B07D1CA
:100FD000002C10D1039A0299306B17F05DFF3C0092
:100FE000380013F015FA029B070001330293039BAC
:100FF000013B0393C7E70D4A39003000FFF7ACFD12
:1010000007B0F0BD002DCDD0AC4208D1200013F0C8
:1010100004FA00220100300000F00AF8C2E70022C2
:101020002900F8E700220099C7E7C046F5A00300B1
:10103000F0B50B7817001A000A3A85B004000D00CD
:101040000F2A10D803A9280015F03DFE03992000AF
:10105000002F01D0022F03D1FFF71AFD05B0F0BD1C
:10106000FFF704FDFAE76A4A192B00D8CBE01A3BD8
:101070007C2B00D182E005DC252B08D0772B11D00A
:10108000644AC0E07E2B00D194E0912BF8D1002F70
:1010900000D0B7E003A9280013F0C4F90200039BB5
:1010A00000219BE002A9280013F0BCF90600022FE2
:1010B00003D001002000FFF7B7FE300013F0A8F9BD
:1010C0000299060015F0F6FD0028D9D13378922B4D
:1010D00013D1300003A913F0A5F90600300013F076
:1010E00097F9039A0190904207D2022F03D0310062
:1010F0002000FFF799FE019EF0E73378A12B21D164
:10110000022F06D1206B17F061FD206B17F01DFD3B
:101110000EE0300013F081F901002000FFF784FE9B
:10112000206B012FF2D117F025FD206B17F0F5FC95
:10113000300013F06DF9029915F0BCFD002800D0C5
:101140008CE79DE7A22B9BD1300013F066F903A931
:1011500015F0B9FD012F07D1206B17F001FD0399A0
:10116000206B17F0B8FCE3E7022F02D1206B17F0D9
:1011700016FD0399206B17F0DBFCD9E703A92800C3
:1011800013F050F90399060015F094FD002800D0E3
:1011900076E7002F36D1350003A9280013F042F975
:1011A000060013F035F903789D2B1BD100231A009C
:1011B000310013E0002F25D103A9280013F032F9E4
:1011C0000399050015F076FD021E02D03B003A009F
:1011D00066E72B789A2BDFD0030029002000FFF769
:1011E000B1FE3BE79E2B05D103A913F01BF9039B2E
:1011F0000200DDE7BE2B00D142E713F009F932000F
:1012000003004DE7044A29002000FFF7A5FC25E76D
:1012100096A00300AEA00300C9A00300F0B50B78B0
:101220008FB00A3B0400019103920F2B00D9E6E036
:10123000080013F0EDF80378912B00D0DFE001985F
:1012400013F0E6F80BA913F0EDF8037842780A3BA7
:101250001B021343AD2B00D0D1E013F0D9F8037873
:101260000500A02B00D0CAE013F017F9002800D029
:10127000C5E0280013F0CCF80B9B984200D0BEE0EC
:10128000280013F0CAF89C210C900CA813F0D9F890
:1012900001230C9E070030000D9313F0B9F80500F0
:1012A0000C90874200D1A0E013F0B2F80C90874276
:1012B0000AD00378032B00D0A1E00DA913F079F830
:1012C0000C90874200D09AE033784833DBB2022B8F
:1012D00000D894E02B784833DBB2022B00D88EE0A4
:1012E0000B9B1800049313F093F8039A029090421A
:1012F00001D1002302930D9B27690593238B27833C
:101300000693638B0793E38B08937B1C0393BB1CAF
:1013100009936B469B896383A38BE3833B1D236106
:101320002B780393032B03D029002000FFF77CFDCB
:1013300031002000FFF778FDF91C206B17F05BFCF3
:10134000B91C206B17F020FB206B17F009FC002262
:1013500001992000FFF76CFE04992000FFF764FD5F
:10136000791C206B17F010FB0599206B17F040FBE0
:101370001221206B17F0F0FC206BF91C17F004FB16
:10138000039B206B032B33D017F0F4FB206B17F07B
:1013900006FC059B1921002B00DA1A21206B17F09F
:1013A000DBFCBA1C0121206B17F031FC6B461B8B58
:1013B00023836B469B8B63836B461B8CE383029B6F
:1013C000002B03D019002000FFF72EFD3900206B01
:1013D00017F0DAFA206B17F0D7FB039B032B02D030
:1013E000206B17F0D1FB0FB0F0BD35002E4E6BE730
:1013F00017F0B6FB29002000FFF716FDC9E7238B85
:1014000025690293638B6F1C0493E38B67830593B9
:10141000AB1C0693A38B0198E383244B2B432383BC
:10142000EB1C236112F0F4FF01002000FFF7FCFC2D
:101430000600206B17F03CFC3900206B17F0A4FA73
:10144000A91C206B17F03EFC002201992000FFF739
:10145000EFFD31002000FFF7E7FC0600206B17F0DE
:101460008AFA002803D13900206B17F0C4FBA91CAD
:10147000206B17F089FA206B17F030FC6B461B8944
:1014800023836B461B8A63836B469B8AE383039BA0
:10149000B34203D031002000FFF7C6FC2900206BC7
:1014A00017F072FA9FE7C046534703000080FFFF22
:1014B000F0B5170085B0040008000D0012F0A8FF79
:1014C0003900060015F0F6FB019000281ED02379A4
:1014D000002B16D0E36A1E78002E12D113212000B3
:1014E000FFF7C4FA29002000FFF79EFC330032000A
:1014F0000121206B17F00FFD206B17F045FB05B0A5
:10150000F0BD29002000FFF78FFCF5E733783B2B77
:101510001DD1290001222000FFF78AFD300012F0C2
:101520007CFF4378811C4E3BDBB218260A2B01D886
:10153000224AD65C2000FFF777FC3100206B17F0C1
:101540000BFC022229002000FFF772FDD7E73C2B9D
:101550002ED1300003A912F065FF06000700039B9F
:101560009F421FD101992000FFF75EFC206B17F00E
:10157000F7FA002229002000FFF75AFD019BB34231
:10158000BDD0300012F044FF019B0500834202D021
:10159000206B17F0E5FA310000222000FFF748FD2C
:1015A0002E00EBE7380012F033FF01970700D6E773
:1015B00031002000FFF738FC019AC3E78BA003003D
:1015C000F0B589B0040005910492009302910029BE
:1015D0002AD1A379002B2CD0E36A1D78012D28D1C4
:1015E00005212000FFF742FAE16A029B088D834241
:1015F00006DB0021554A2000FFF7AEFA09B0F0BD26
:10160000CE6ADA00B21856782E420BD052880121E9
:10161000206B17F02EF9002302211A00206B17F01F
:101620007AFCEBE70133E2E79C2105A812F009FF01
:10163000029000273E00059D03970197029BAB4255
:1016400016D1002E0AD0039B002B70D1206B17F00F
:1016500038FA002F70D1206B17F033FA049B002B5F
:101660006FD03300019A0099206B17F05DFCC5E73D
:101670002B78B82B10D1B73B1E4202D0344A290038
:10168000B9E7012328001E4312F0C7FE039028008B
:1016900012F0BEFE0500D1E7B92B0BD1B73B1E42BD
:1016A00001D02C4AEBE7022328001E4312F0B5FEBE
:1016B0000700ECE7BA2B2CD1280012F0AEFE050093
:1016C00012F0A6FE0378BE2B0BD1200006222900C3
:1016D00015F019FC009B28000133009312F098FECE
:1016E000D6E72B780A3B0F2B01D91B4AC7E707A97E
:1016F000280015F0E8FA05000799206B17F0C0F9EB
:1017000029002000FFF790FB019B050001330193A6
:1017100094E7019B002B01D0104AB0E7290020007C
:10172000FFF782FB009B05000133009386E70399D6
:101730002000FFF779FB8CE739002000FFF774FBEE
:101740008CE73300019A009968E7C046D8A30300EC
:10175000F6A303000DA4030025A4030046A4030080
:10176000F0B589B00400039103A8072112F069FEC7
:101770000027E36A02905E7E0398029B834215D1A4
:10178000180012F04AFE029B03901B780100320001
:101790002000242B4CD115F04DFB0500013F4AD20F
:1017A00029002000FFF774F909B0F0BD05A912F077
:1017B00039FE4021039003A812F043FE06A905005C
:1017C000039815F080FA069B01902A2B3CD18542A4
:1017D00007D8214A00212000FFF7BEF9059B03939B
:1017E000CAE7019812F014FE8542F2D107A90198C8
:1017F00015F069FA079B2B2B24D02D2BE9D1042659
:10180000ECE707A915F05FFA07990390206B17F032
:1018100062F903988542F4D10599280015F04AFA37
:101820000028DBD1A07129002000FFF7FDFAD5E7E1
:1018300015F077FDB1E7002301211A00206B17F0A6
:101840006AFBABE70126C9E703992000FFF7ECFA32
:1018500001370390DDE7C04696A10300F7B50A788B
:101860000E0013000821293B8B43DBB20400002B40
:1018700002D10133C371F7BD13002A3B8B43DBB2A6
:10188000002BF8D013000A3B0F2B2FD9282A11D197
:1018900001A9300012F0C6FD070012F0B9FD019B4E
:1018A000984205D012F0B4FD019B0500984208D182
:1018B000002506E0300012F0B0FD070012F0A8FD90
:1018C000050001A9380015F0FEF9E379002D02D0DA
:1018D0002A78002A0CD1002BCDD1E38A002BCAD064
:1018E000184A31002000FFF737F9C4E73700DFE777
:1018F000002B1ED0A38A01339BB2A382012B09D1F6
:10190000E18A206B002911D017F048FA0021206BE2
:1019100017F06BFA29002000FFF786FA206B019977
:1019200017F0AEF8206B17F06CFAA4E717F0C9F8BF
:10193000ECE7E38A29000133E3822000FFF774FA21
:1019400099E7C046B4A10300F0B504000E00056994
:1019500087B002936B1C0393AB1C03612900006BDF
:10196000170017F082F9200015F0B5F931002000BA
:10197000FFF75AFA206B17F0B7F9691C206B17F0C4
:101980003AF92900206B16F0FFFF206B17F010FBCF
:101990002669731C2361029B9F4218D1A38B206B85
:1019A000013BA38317F079F9206B17F005FB03992E
:1019B000206B16F0E9FF0C9B002B03D019002000D0
:1019C000FFF732FA3100206B16F0DEFF1BE0380023
:1019D00012F023FD002305932369050001930133D1
:1019E00023610378002B10D112F012FD12F010FDCC
:1019F000029B834224D03F4A29002000FFF7ACF825
:101A0000A38B013BA38307B0F0BD07006A2B07D16E
:101A100012F003FD070012F0FBFC05A915F053F9C5
:101A2000206B17F09DF839002000FFF7FDF9212108
:101A3000206B17F091F9019A0021206B17F0E7F85D
:101A4000280012F0E5FC0700206B17F09DF80599BF
:101A500000294BD1206B17F097F80025206B17F069
:101A600093F8059BAB4209D02569206B6B1C236161
:101A7000290017F006F9200015F02DF93900200093
:101A8000FFF7D2F9059B0700002B02D0206B17F05F
:101A90002BF9206B17F049F9059B002B19D00F216A
:101AA000206B04F0B3FD2900206B16F06DFF0F21B1
:101AB000206B04F0ABFD05992000FEF7E9FF200044
:101AC0000599FEF7F7FFA38B206B013BA38317F06B
:101AD000E4F83100206B17F08EF80199206B16F0B6
:101AE00053FF0321206B16F04BFF54E72000FEF755
:101AF000CFFFB2E768A40300F0B587B00391437944
:101B00000400012B06D1C36A1B78002B04D11E4AA6
:101B1000FFF722F807B0F0BD039B432103A8019310
:101B200012F08FFC02900398029B8342F2D005A929
:101B30000B2715F0C8F802AB059DFF1803903A007B
:101B40002900E06A13F0EAFE3B780600002B03D17F
:101B500003780E4A042B0AD12900E06A13F00BFF28
:101B6000002803D00378023B022B05D9084A0199CB
:101B70002000FEF7F1FFD6E7042333702900E06A66
:101B800013F00CFFCFE7C04619A203003EA20300EA
:101B90005FA20300F0B587B0039144790500012CE2
:101BA00009D1019103A8432112F04BFC0290039844
:101BB000029B834201D107B0F0BD05A90B2715F0A8
:101BC00082F802AB059EFF1803903A003100E86AE4
:101BD00013F0A4FE3B78002B08D10378012B05D02D
:101BE000074A01992800FEF7B7FFE0E704703100CB
:101BF000E86A13F0B7FE0028D9D00470D7E7C046D2
